:109C6A00414952434F544543004256332E33342020
:109C7A00504F52004241542000532F4E2146414931
:109C8A004C555245005245454E54455221532F4E8C
:109C9A0000434F4E5441435420414952434F544587
:109CAA004300475053004032444000403344400090
:109CBA004F464621564F4F404D454E55000A160015
:109CCA000180000300007E0000FE00001E00003636
:109CDA000003E60001C4000000000FFFE050524FED
:109CEA0043555240534154530043414C4940414C1F
:109CFA00542020230053454C4543414F20005445EE
:109D0A004C4153202020004D41504120202020006A
:109D1A0043454E54524F202000564152494F20206D
:109D2A0020004241524F4752414600524F5441533C
:109D3A002020200050524F58494D20200050494CB5
:109D4A00614F202020004D4152434F532020004FA5
:109D5A00524947494E414C00202020214D4544217B
:109D6A00202020204449530020545241434B214C87
:109D7A004947200020545241434B21444553200077
:109D8A004D41524B00545241434B2D4143494D20C2
:109D9A00004E4F5254482D4143494D200021534112
:109DAA0049522020200153454C4540524F5441010D
:109DBA00414A55535420414C545501564F4F532054
:109DCA00202020686901564F4F5320544F44686938
:109DDA000150494C614F202020686901524F54417B
:109DEA005320202068690141495253504143456834
:109DFA006901434F4E4649475552686900414A55E1
:109E0A00535420414C5455004241524F4740414C13
:109E1A0054550047505320414C5455524100514E1D
:109E2A004820202020402148504100464C004C4FF9
:109E3A0047564F4F2056415A494F20003E21534121
:109E4A00495220202000534149522020014D4F53AE
:109E5A00545241015452414E5346014150414741E7
:109E6A005200215341495220202001434F4D3A20AC
:109E7A00202020202001544E432031232035374B07
:109E8A0001544E4320312320392E360101505743C5
:109E9A00403130234035374B01505743403130234E
:109EAA004031394B01014D5850403130234035374C
:109EBA004B014D58502034232035374B014D585013
:109ECA002031232035374B014D5850403130234043
:109EDA0031394B014D58502031232031394B002163
:109EEA0053414952202020014E4F564F2050494C91
:109EFA00614F014D4F44492050494C614F01415037
:109F0A0041472050494C614F0101434F4D3A01529C
:109F1A004543452050494C614F01454E5649205012
:109F2A00494C614F01454E564940544F444F5301E5
:109F3A00014449532050492D50492001415041477D
:109F4A0040544F444F53200044495220214449531E
:109F5A0054004752415620004C4F43414C40414324
:109F6A005455414C0047524156415220202020006E
:109F7A002053544F52452157505420002046554CE7
:109F8A004C20002140415041474152200053455244
:109F9A0020004952202000555342200055534220A8
:109FAA00004C49535400454E564900204552524FE1
:109FBA00205452414E534D495420200021534149C7
:109FCA00522020200153454C4540524F54410149EB
:0D9FDA004E532050494C614F20014D4F4423
:109FE700494620524F544101494E56455220524F3F
:109FF700544101415041472050494C614F01415064
:10A0070041472020524F54410143594C205241446B
:10A0170049555301434F4D3A01524543454220525A
:10A027004F544101454E56494120524F5441014337
:10A037004845434B20524F0053454C4521524F54FE
:10A0470041004E4F564F0020414C54404F52444020
:10A05700210021494E5645525445524000494E561B
:10A06700455254002140415041474050545300212C
:10A077004150414720524F54004D454D20434845DC
:10A08700494120002140454E5640524F544100203F
:10A0970020524144495553002153414952014341FC
:10A0A7005240435452215043200156455240435495
:10A0B70052202020014150414740544F444F5320E4
:10A0C7000101434F4D3A0152454345424520435410
:10A0D7005201454E5649415220435452005645526B
:10A0E7002043545220004D4F5645522020004D4FDB
:10A0F700564552205041524100455343414C41205F
:10A1070020582F592053414952004150414720447C
:10A117004953004155544F204C4947004445534C3F
:10A127004947414E444F002020205A4F4F4D00448D
:10A13700495354204B4D0044495354204E4D002160
:10A147005341495220202001564152494F20202097
:10A1570068690158432D434F4E4649686901525477
:10A16700412D434F4E46686901474552414C2020D7
:10A177002068690154454C4120202020686901016D
:10A18700014D4F442E464143494C01434F4E462013
:10A19700464142524901544553544520564F4F01B9
:10A1A70041504721544F4421564F4F0021534149B5
:10A1B7005220202001534F4D4445534301444553FA
:10A1C70043212D014D4F44404445534301494E56C9
:10A1D70040444553430153454E5641524020204089
:10A1E7002301564F4C554D450143414C492056419B
:10A1F70052494F01544F4E4520014652455155454E
:10A207004E4301564152204D4440203040230154D3
:10A2170045432020204030304025015445535441C8
:10A227005220534F4D0053444553434C4947005325
:10A2370044455343444553004E414F204455414CF8
:10A247000043414C4920564152494F004553504520
:10A25700524152203130204D494E202000414E546A
:10A2670045532043414C494252415220002153411A
:10A2770049522020200143414D494E484F2001417A
:10A2870055544F43454E5401014D45442F444953BE
:10A29700200146494E4553534520014C2F440101A7
:10A2A70056454E5421542D55500143454E54215483
:10A2B7002D555001574159505421425247002153BF
:10A2C70041495220202001484F5240494E494349B5
:10A2D7004F015052494D45014652455155203A01CB
:10A2E7005154444520202020202001554C54494DED
:10A2F7000143594C53494740202040230153454CC3
:10A3070040524F5441200101010143594C5201432E
:10A31700594C20542D55500021534149522020209B
:10A327000101554E495401434C49434B40302C40A1
:10A33700202301434F4E5452415354014E4D454142
:10A347002131383301494D502F41475053010143C3
:0DA357002D564152494F014D454D4F525971
:10A3640044554D50004D454D4F525944554D5000A4
:10A3740040574159504F494E542045584953542051
:10A384004000574159504F494E54002053414952BF
:10A39400202020210052454345424552004C495655
:10A3A4005240003C2D204C495354202D3E20204542
:10A3B4005849540053454C004E4558540054505489
:10A3C4002050524F580054505420414E544500419F
:10A3D400504720404C4547004150472040534F4D83
:10A3E40000444553202020202020202000204445E4
:10A3F400530046414C4841475053202000204752C7
:10A4040041564152202000524F544120004D4150AA
:10A41400524F58004C495354410045544500414C57
:10A4240054403000524F54412056415A4941002073
:10A43400544F4F404D5543482000214053454C4014
:10A444004C495354002053454C405750544021002C
:10A4540021405245434542455240002020404F2070
:10A464004B40202021004F4B005641520046495892
:10A474000047415445215800504F4E544F504152CB
:10A48400544900535443594C20004044455300540C
:10A49400502000406A40494E20004067404F5554C8
:10A4A400002046414C48412020210020534149527C
:10A4B400004D4F4449005940454053004D4F4449D5
:10A4C40020204E4F56204752415641520050524F81
:10A4D4005820202053454C202053414952005843D2
:10A4E400542D464C49474854200055534544004593
:10A4F4004E54455220004D4D2E4D4D4D20004D4D96
:10A504002753532E530057475321383400204055C6
:10A514004054404D402000554054404D0020555477
:10A524004320004C4F43414C005357495353474435
:10A5340000414C540053554940580041564740206F
:10A5440030402300353030003136343000205D2077
:10A554003130404B632F70005D2020203140632F49
:10A564002300205D202035404B5453005D203230C1
:10A57400304046504D00406340204B630046542019
:10A584004B6300406340204E4D004654204E4D0026
:10A594004D2F53003230305E003530305E003122B2
:10A5A40000322200332200352200382200464C3784
:10A5B40000464C313600464C333300464C363500A9
:10A5C4004631303000463136300046323630005E97
:10A5D400252640534F47005E2526405441530041F1
:10A5E4004C540056415200225E2F24004B54530019
:10A5F400532F4E002224004B5400225E004E4D0087
:10A60400302C3500312C3000322C3000302C360008
:10A61400312C3200322C3500332C3800372C3500E5
:10A624004031350040333000403630005441534B04
:10A6340000464C2D4441544500545000544F4600AC
:10A644005354410046494E004C414E00534554205A
:10A654004F464653455400495341204845494748CD
:10A6640054004155544F2D474F20005354415254E8
:10A674000020434845434B40414C4C005241442048
:10A6840044495354004053454C4048454947485475
:10A694003A00475053404241524F40414C4C0053C2
:0CA6A400494E4B40312D3221632F230022
:1064F400304D2475A7049005C2E0F51CE0F51DE0BD
:10650400F51EE0F51FE0F56DE0F56EE0F56FE0F5E2
:10651400541270B6126AF42275C70375C6E475B9CD
:1065240001E5BCB481431270B61256DC8E628F63EF
:106534007568F97569001265CA203C2D203B2B1241
:1065440066FF1266D3856D1C856E1D856F1E85548E
:106554001F126636203C12203243201D231266FF90
:10656400126AF4E532242850DC22126636203CF903
:10657400203DF6203205201DBD80EF301DB880EA95
:106584001266FF126AF4856D1C856E1D856F1E856B
:10659400541F1266E9126AF4203DCE8099126922D2
:1065A400201D0D7553107400126885203DBB808634
:1065B400E553540FC553C4540F20350512679A8010
:1065C40003126885808BC23CD23B126686FD12663C
:1065D40086FC126686C39573F565EC9574F564EDD7
:1065E4009575600504600A800EE56424E05011800E
:1065F40006E56424204009126686126686026686D1
:10660400126686FD126686FC126686C39576F56769
:10661400EC9577F566ED9578600904600122E566EE
:10662400F48002E5668562F0A474E025F04002C2BD
:0D6634003B22C23C126686A2E7923DA2E620
:10664100921DA2E592324026A2E492E592E692E7FB
:10665100FC1266862565F565EC3564F5641266867F
:10666100FC1266862567F567EC3566F56622A2E4BD
:106671009235540F79C6F712668609F7301D051257
:106681006686F55322E5697023E56860302404408D
:106691002CE56875F004A485F0C7F5C675B901E568
:1066A100BCB4811985BD68756902801E54037010E0
:1066B10005C675B901E5BC056953690F22D23C22B3
:1066C100147004E5BD80F0147004E5BE80E9E5BFF7
:1066D10080E575A7009006F6E56DF0A3E56EF0A3E1
:1066E100E56FF0A3E554F02275A7009006F6E0F5FA
:1066F1006DA3E0F56EA3E0F56FA3E0F55422E56428
:10670100B2E7F56D85656EAB67E566FC30E707C3FB
:10671100E49BFBE49CFCAA62A9631253DCE56630AE
:10672100E707C3E49DFDE49EFEEEB2E7F56F8D54ED
:106731002275380C12698B1269D6D553012275382E
:106741000C12695C1269CCD55301227538001269AB
:0E6751007412699BD553012275380012695CE1
:10675F0012699BD553012275380312698B126A0790
:10676F00D553012275380312695C1269FDD55301A7
:10677F002275380F126974126A2CD553012275389D
:10678F000F12695C126A2CD553262290679F2373D0
:10679F008091807780688059804A803B802C801D53
:1067AF00800E80DA80CB80BC80AD809E808F808011
:1067BF0075381512698B126A4ED55301227538152B
:1067CF0012695C126A43D553012275380912697434
:1067DF00126A14D553012275380912695C126A14B2
:1067EF00D553012275380612698B1269BED5530134
:1067FF002275380612695C1269B3D55301227538B8
:10680F00121269741269E4D5530122753812126994
:10681F005C1269E4D553012202673275381512698B
:10682F008B126A4ED553012275380F12695C126AAA
:10683F002CD553012275380F126974126A2CD55357
:10684F00012275380312695C1269FDD55301227557
:10685F00380312698B126A07D5530122753800125B
:10686F00695C12699BD55301227538001269741245
:10687F00699BD553262290688A2373809E80A980B6
:10688F00B480BF80CA80D580E08010801B802680B6
:10689F0031803C80478052805D806875380C12696A
:1068AF005C1269CCD553012275380C12698B1269B1
:0E68BF00D6D553012275381212695C1269E4B5
:1068CD00D55301227538121269741269E4D553013A
:1068DD002275380612695C1269B3D55301227538D9
:1068ED000612698B1269BED55301227538091269DA
:1068FD005C126A14D5530122753809126974126A33
:10690D0014D553012275381512695C126A43D5539B
:10691D00012202682A78C686040886037AED12538E
:10692D009A78CAA60408A60378C686040886037A50
:10693D006212539A78CCA60408A60378C68604087A
:10694D0086037AB512539A78C8A60408A603227551
:10695D001A6A751B0A78CA8618088619126B9F78F1
:10696D00CC86060886072278C88618088619E4F5AD
:10697D001AF51B126B9F78C886060886072278C603
:10698D008618088619751A00751B01026B9FE51D87
:10699D002519F51DE51C3518F51CC3E51F9FF51FC1
:1069AD00E51E9EF51E22C3E51F9FF51FE51E9EF5F4
:1069BD001EC3E51D9519F51DE51C9518F51C22E561
:1069CD001D2FF51DE51C3EF51CC3E51F9519F51F83
:1069DD00E51E9518F51E22C3E51D9FF51DE51C9EB0
:0969ED00F51CC3E51F9519F51F07
:1069F600E51E9518F51E22E51F2FF51FE51E3EF52F
:106A06001EE51D2519F51DE51C3518F51C22C3E5E7
:106A16001D9519F51DE51C9518F51CE51F2FF51F8D
:106A2600E51E3EF51E22E51D2FF51DE51C3EF51C57
:106A3600E51F2519F51FE51E3518F51E22C3E51DB0
:106A46009FF51DE51C9EF51CE51F2519F51FE51E86
:106A56003518F51E22E51A7009E51B70058C068DA2
:106A66000722ED851BF0A4A2F792D5ED851AF0A4B6
:106A7600AEF0FFEC851BF0A4A2D53FEE35F0FF92F9
:106A8600D5EC851AF0A42FFFE435F030D50104FECD
:106A960022E4F51AF51BEF4E7003051B22EF65196C
:106AA6007006EE65187001227808C3EF33FFEE33E7
:106AB600FEEF9519F5F0EE95184003FEAFF0E51AD6
:106AC60033F51AD8E5F4F51A751BFF7805C3EF33CD
:106AD600FFEE33FEEF9519F5F0EE95184003FEAF85
:036AE600F0E51BBD
:106AE90033F51BD8E5F4C403F51B22E51D9511E523
:106AF9001C9510500BE56E9511E56D95105001220E
:106B0900E51F9511E51E9510500BE5549511E56F9C
:106B19009510500122E51D9513E51C9512400BE5D2
:106B29006E9513E56D9512400122E51F9513E51E3B
:106B39009512400BE5549513E56F951240012253C8
:106B49002CF8C3E51F9554FFE51E956FFE92605022
:106B590007C3E49FFFE49EFEC3E56E951DF519E5A5
:106B69006D951CF5189261500BC3E49519F519E45C
:106B79009518F518C3E5199FE5189E9262500AE524
:106B890018CEF518E519CFF519126A97E52C5407AF
:106B990075F003A4F538E538906BA573026BBD0257
:106BA9006BD1026BDF026BF7026C0A026C1D026C7F
:106BB9002B026C43851C16851D17C3E4951FF5151B
:106BC900E4951EF514026C56851C16851D17851E45
:106BD90014851F158077C3E4951DF517E4951CF5F9
:106BE90016C3E4951FF515E4951EF514805FC3E4FB
:056BF900951DF517E4F5
:106BFE00951CF516851E14851F15804CC3E4951F34
:106C0E00F517E4951EF516851C14851D158039851E
:106C1E001E16851F17851C14851D15802BC3E49524
:106C2E001FF517E4951EF516C3E4951DF515E495AD
:106C3E001CF5148013851E16851F17C3E4951DF5CC
:106C4E0015E4951CF5148000C3E5179513E516950C
:106C5E001210D70122E5159513E514951210D701E0
:106C6E0022E519F92517FFE518F83516FED3EF952D
:106C7E0011EE9510500122E5119517FDE5109516B0
:106C8E00FC402A4D6027126A5BE5152FF515E514B9
:106C9E003EF514E5159513E514951210D70122E56E
:106CAE00199DF9E5189CF8851016851117E5172919
:106CBE00FFE51638FEE5139FE5129E500BC3E51354
:106CCE009517F9E5129516F8E51A700AE51B700688
:106CDE00AA00AB018013E9851AF0A4E5F0FBE88564
:106CEE001AF0A42BFBE435F0FAE5152BFBE5143A6C
:066CFE00FAE5119BE51010
:106D04009A10D70122EB9515FDEA9514FCC3E515FD
:106D14009511E514951010D717E5139BE5129A50B9
:106D240036E5139515FFE5129514FE126FD38027EF
:106D3400EB9511FFEA9510FEAA00C001126FD3D0A3
:106D440003E5172BFBE5163AFAEB99F517EA98F5E4
:106D540016851115851014C2D5E5466002D2D5AA50
:106D640056E98AF0A4ABF0E88AF0A42B30D5047578
:106D7400F00384F8700122E5172513FDE51635129A
:106D8400FCED8AF0A4ABF0EC8AF0A42B30D50475AA
:106D9400F00384FEE5152513FDE5143512FCED8A98
:106DA400F0A4ABF0EC8AF0A42B30D50475F0038486
:106DB400F9E538906DBB73026DD3026DDF026DE8A7
:106DC400026DF1026DF7026E03026E0A026E0FC3CA
:106DD400743E9EFFC3743E99FE8032C3743E9EFF90
:106DE400AE018029AF06C3743E99FE8020AF06AE83
:0D6DF40001801AC3743E9EFEC3743E99FFD9
:106E0100800EC3743E99FF8007C3743E9EFEAF019E
:106E110008EF2437FFE51B7007E51A700CE8800EB8
:106E2100A2E7E51A50030460F488F0A4E5F06001DC
:106E310004F923FA98FBC3E998C333F9906E43E54B
:106E41003873026E5B026E88026EBD026EEA026FDB
:106E510017026F44026F71026F9E05A7800BEB3022
:106E6100E7032A8002291E1FFBEEC45403F583EEBB
:106E71005408C42FF582EE5407243883F5F0E04519
:106E8100F0F0D8DA05A72205A7800BEB30E7032A3B
:106E91008002290E1FFBEEC45403F583EE5408C48F
:106EA1002FF582EE5407240B83F5F0E045F0F0D87E
:106EB100DA05A722804020100804020105A7800BF3
:106EC100EB30E7032A8002291E0FFBEEC45403F5C1
:106ED10083EE5408C42FF582EE540724EC83F5F0B9
:106EE100E045F0F0D8DA05A72205A7800BEB30E7E3
:056EF100032A800229C4
:106EF6000E0FFBEEC45403F583EE5408C42FF5823F
:106F0600EE540724BF83F5F0E045F0F0D8DA05A784
:106F16002205A7800BEB30E7032A8002291F1EFB00
:106F2600EEC45403F583EE5408C42FF582EE5407DD
:106F3600249283F5F0E045F0F0D8DA05A72205A7FC
:106F4600800BEB30E7032A8002291F0EFBEEC454A8
:106F560003F583EE5408C42FF582EE5407246583A7
:106F6600F5F0E045F0F0D8DA05A72205A7800BEB8F
:106F760030E7032A8002290F1EFBEEC45403F58373
:106F8600EE5408C42FF582EE5407243883F5F0E05A
:106F960045F0F0D8DA05A72205A7800BEB30E7030A
:106FA6002A8002290F0EFBEEC45403F583EE540823
:106FB600C42FF582EE5407240B83F5F0E045F0F07C
:106FC600D8DA05A7228040201008040201EC701FC1
:086FD600ED20E740D2E023CFDB
:106FDE0023CF30E7F980357B08801A7B1080167B33
:106FEE002080127B40800E20E4ED20E3EE20E2EFC5
:106FFE0020E1F07B80EE8BF0A4CF8BF0A4E5F02F98
:10700E00FFEC8BF0A4CD8BF0A4E5F02D2499838FAB
:10701E00F0A433E5F033FBE98BF0A4E5F0C88BF078
:10702E00A428F9E435F0F822FFFEFCFAF8F6F4F2A3
:10703E00F0EFEDEBEAE8E6E5E3E1E0DEDDDBDAD901
:10704E00D7D6D4D3D2D0CFCECCCBCAC9C7C6C5C45F
:10705E00C3C1C0BFBEBDBCBBBAB9B8B7B6B5B4B379
:10706E00B2B1B0AFAEADACABAAA9A8A8A7A6A5A465
:10707E00A3A3A2A1A09F9F9E9D9C9C9B9A99999829
:10708E009797969594949392929190908F8F8E8DD0
:10709E008D8C8C8B8A8A898988878786868585845C
:1070AE00848383828281818075A7009070DCE5469F
:1070BE00FA24FA50027A05EA2323F978107F049312
:1070CE00F60809E9DFF99070F4EA93F556227FC2CB
:1070DE00803E7F4680BA7E8C81747D1882E87A303D
:1070EE0085D074608BA08080402010081271000241
:1070FE007356D215D274D273C219C23A1256DC8E9E
:10710E0047757D0075460575520212914612022191
:10711E00E53524EB500E1291467F1990A11112768F
:10712E00F012DD46E55275F016A4F57012730C756B
:10713E007E151271D77F237E0990A0ED1277021271
:10714E00DD4610000810010D10021280E212727F4F
:10715E0075330180DA1272C475330180D2757E00E8
:10716E001271D77E0090A1001277357F237E059095
:10717E00A0F512770212722812DD46E55210000FAA
:10718E0010010510028780D5045403F55280CE12EB
:10719E0071D77F237E0B90A130127702E5466007F0
:1071AE001460041412411A12DD46E5461000081050
:1071BE00010B10021180D860D6154680D2B405029C
:1071CE0080CD054680C902711B75320012DF1C7F0F
:1071DE00017E1190A0E41277357E0012D5DDE57E9A
:1071EE00D26612D63475170812DA671241597571C4
:1071FE0000C20612D784741BFFF5177E0F90A136BE
:10720E00305D0390A13E127735129189125D0D12F9
:10721E0046BFC20612651C021E03E55260141460BE
:10722E001E1460297F647E2D791C1272721E1FD966
:10723E00F9227F6A7E1F79281272721FD9FA227F75
:10724E00487E2D791C1272720F1ED9F9227F567E3E
:10725E003379281F12DE610F0F12DE611F12DE61FD
:10726E001ED9F0221E12DE610E0E12DE611E02DE2D
:10727E0061E552605514606814606D800075709EF3
:10728E001272F98003757000E5732540F573E435CD
:10729E0074F574E43575F575227570161272968054
:1072AE000375702DE5762542F576E5773541F57750
:1072BE00E43578F57822E55260CB1460DC1460E199
:1072CE0080007570441272B2800375705AE5739522
:0972DE0040F573E5749400F574A9
:1072E700E5759400F575227570711272DB80037570
:1072F7007088E5769542F576E5779541F577E578F7
:107307009400F57822E54690732293F540FEAD4749
:10731700E4FFFC12546F8E418F4222020C1830603A
:10732700C07F40120E9E121E1912DD461275D1EB58
:107337007005909E3F800B1273DF90A45F500390FF
:10734700A4A57F3F7E0412770212DD4612DE2712C4
:10735700DE5775370990A09F121CFF907366730262
:1073670002930275260270FA0276020273560273BE
:107377007E0273970273287F2E12168680D17F367E
:107387007E0490A43312770212DD4612DE2780BFF7
:107397007F37120E9E121E1912DD461275B512485E
:1073A7004FD2AC1000A9306DFA12748F203BCF403A
:1073B700ED7568F97516001274DC40FB1276787F5C
:1073C700367E29E51612D3BD12DD4605161277A8BB
:1073D70078C6B6F7E20275AF7C0512484F12DC603B
:1073E700744112DC71745312DC2EEB12DC4F1277EE
:1073F700BA5003DCE5227515F975160010000EE585
:1074070015602512743140051274585002D3227F3B
:107417003F7E29E51612D3BD12DD467F1412DE3EEC
:107427000516E51664F870D4C322127D7075B9018C
:10743700E5BCB4811AE5BDF51570037516F778C676
:0B744700A616127EB9127EB1127EB1B3
:10745200C3027EB1D3227F0575F019D5E0FDD5F0C8
:10746200FA12484F12DC60744112DC71744212DC71
:107472002E7E0F78C6E60812DC2EDEF912DC5212DE
:1074820077BA400122DF012275F00080CEC23B12A2
:10749200484FD2AC12DBB9204C3CB440F712DBBEF1
:1074A200B4400312DBBEB4412DF53812DBBEB45337
:1074B2002512DBBEFA12DBBEE538701A12DBBEB44F
:1074C2000D1412DBBEB40A0EC3E5169A400302770E
:1074D2009FC2ACD23B22C2ACD3221277FE12484FDB
:1074E200D2AC1000F112DBB9204CEBB440F412DB49
:1074F200BEB4400312DBBEB441DCF53812DBBEB4CD
:1075020042D47E1078C612DBBEF608DEF9E538708A
:10751200C512DBBEB40DBF12DBBEB40AB9C2ACC326
:10752200220273567F0A120E9E121E1912DD461295
:1075320075B5124868D2AC1000E712DBBEB440F554
:10754200F53812DBBEB46EED12DBBEE538600A120E
:107552004868744F12DC3A80DC124868744012DCCE
:1075620071E51612DC3A12DC447568F975160012E0
:107572004868D2AC10003912DBBEB440F7F53812BD
:10758200DBBEB44EC07E1078C612DBBEF608DEF952
:10759200124868E5386007744F12DC3A80D11276DF
:1075A200780516745112DC3A78C6B6F7C21276150F
:0C75B200027356751500751603127D67F4
:1075BE0075B901E5BC30E70205160515E515242061
:1075CE0050EB227B007515F9127D7075B901E5BC83
:1075DE00B481010B0515E515240450EC7515011247
:1075EE007D6775B901E5BCB481010B0515E5152460
:1075FE002050EC227F1C120E9E121E5C400675154A
:10760E00F9127615027356E51560372404401A24D4
:10761E001E5019E515240740028027127D70127640
:10762E00510515E515240450F2751501127D677587
:10763E00B901E5BC30E7031276510515E515242096
:10764E0050EA22127666124EE605C6124EE605C6C0
:10765E00124EE605C6024EE674FF800574048001E4
:10766E00E4F5BCF5BDF5BEF5BF22E568606AF5151B
:10767E000515E5152404501D751501127D6775B9A4
:10768E0001E5BC30E70280190515E515242050EB05
:10769E00751500800C241C60F750E0E5152406508B
:1076AE0037E56875F004A485F0C7F5C675BC81E5AD
:1076BE0015F5BDF56878C6B6F70375BD00081276E8
:1076CE00DB1276D51276D586BC0886BD0886BE0836
:0976DE0086BF08124EE605C62223
:10C08F0012AECB12C18E12828112C113128289128B
:10C09F00C12002AECF12AECB12C18E1282817F5A57
:10C0AF00C23C12816312835F783F79437F607EEADF
:10C0BF0012C1821282897F6512816312835F783D7C
:10C0CF0079417F207E4E12C182303C2012C3441230
:10C0DF00C19F783F794312C0FE783D794112C0FE6F
:10C0EF0012C34478D7E65480F675370002935BC3CA
:10C0FF00E796FF1819E796FE0809C3E69FF7181988
:10C10F00E69EF7227F5B7E0690A5391277351F805A
:10C11F000A7F667E14745912D4D61F127FEC7E39B3
:10C12F00E402D4F57866E620E73418C3E694720883
:10C13F00E694045029C318E6941F08E69404401EA1
:10C14F007869E620E71818C3E6940E08E6940150C4
:10C15F000DC318E6947508E694004002D322C3225B
:10C16F00E67D0030E7011D08E62BFB18E63CFCE4FA
:0EC17F003DFD22C3EB9FF6F71819EC9EF6F774
:10C18D002212C133400CE47842F608F67840F608E6
:10C19D00F6227864C3E6946AF55708E6944CF55692
:10C1AD000808C3E69458F55B08E694AEF55A753960
:10C1BD0000AC56AD57EC12B278784C12B306AC5AAF
:10C1CD00AD5BEC12B278785012B3067F2B7E867D74
:10C1DD00777C1812B23D785012B2FA12B14912B2F0
:10C1ED003D785012B2FA12B14912B23D785012B2E6
:10C1FD00FA12B14912B23D7F367E847D257C6412E0
:10C20D00B23D785012B2FA12B14912B23D784C12C9
:10C21D00B2FA12B14912B23D7F3F7EA27D607C8B96
:10C22D0012B23D785012B2FA12B14912AF3712AFB5
:10C23D003712B3127F3F7E807D057CE6053912B142
:10C24D0049784812B3067F2C7E937D477C7F12B2CE
:10C25D003D785012B2FA12B14912B23D785012B275
:10C26D00FA12B14912B23D784C12B2FA12B149121A
:10C27D00B23D7F357EB47DF87CDF12B23D78501231
:10C28D00B2FA12B14912B23D785012B2FA12B14956
:10C29D0012B23D7F3F7EED7D227CCD12B23D784CBA
:10C2AD0012B2FA12B14912AF3B12AF37784412B342
:10C2BD00067F317E397D9D7CE712B23D784C12B2FE
:10C2CD00FA12B14912B23D784C12B2FA12B14912BA
:04C2DD00B23D7844B2
:10C2E10012B2FA12AF3B12B23D7F2C7E377D0C7C2D
:10C2F100A312B23D784C12B2FA12B14912B23D7892
:10C301004C12B2FA12B14912B23D784C12B2FA1281
:10C31100B14912AF3B12B3127F3F7E807D027C9FF9
:10C32100053912B149784412B306784812B2FA12AB
:10C33100B2AF8E428F43784412B2FA12B2AF8E403E
:10C341008F4122753900AC42AD43EC12B278784886
:10C3510012B306AC40AD41EC12B278784412B30688
:10C361007F2B7E537D507C0912B23D784812B2FA80
:10C3710012B14912B23D784812B2FA12B14912B261
:10C381003D784412B2FA12B14912B23D7F347EF2C5
:10C391007DCD7CA312B23D784812B2FA12B1491296
:10C3A100B23D784812B2FA12B14912B23D7F3F7ED6
:10C3B1000A7D2E7CAE12B23D784412B2FA12B14916
:10C3C10012AF3712AF37784C12B3067F2B7E4F7DF9
:10C3D100AF7CB212B23D784812B2FA12B14912B230
:10C3E1003D784812B2FA12B14912B23D784812B200
:10C3F100FA12B14912B23D7F357EB17D4B7C951267
:10C40100B23D784812B2FA12B14912B23D784412E3
:10C41100B2FA12B14912B23D7F3F7E497DCD7C45D2
:10C4210012B23D784812B2FA12B14912AF3B12AFC3
:10C4310037785012B306784C12B2FA12B2AF8D555A
:10C441008E568F57785012B2FA12B2AF8D598E5A5A
:04C451008F5B786421
:10C45500E557246AF608E556344CF608E5553404E4
:10C46500F608E55B2458F608E55A34AEF608E435D7
:03C4750059F62253
:1091A90012AECB12983A12AECF7F6690A51B1277FA
:1091B900331292177F5A78C41291F31291FB78C631
:1091C9001291F31291DE7F6578C81291F31291FB27
:1091D90078CA1291F37E2DE51B12D4F57E33E51A78
:1091E90012D4F57E39E51902D4F5860408860302FE
:1091F90053397E15E51C12D4F57E1BE51B12D4F5F7
:109209007E21E51A12D4F57E27E51902D4F57F5A95
:109219007E01E53A12D40B7E0B909C2EE53B93021E
:10922900D508E6FF08E6FE08E6FD339217E450018B
:10923900F4FC12B32375130A75390112B52178D7D5
:10924900E6C2E775F00A84F9303D02A9F012B323AA
:109259008913053912B4FA30170A053912B50D0503
:109269003912B50DA80302B30612AECB12983AC251
:109279003C7F5A7E0312851012921712DD461000A8
:109289000810011510022080EFE53A146004153A20
:109299008003753A3CD23C80DFE53AB43C05753A27
:1092A9000180F2053A80EE7E0312850B7E0B128552
:1092B9001012921712DD4610000810011510022035
:1092C90080EFE53BB40205753B158002153BD23CA6
:1092D90080DFE53BB41505753B0280F2053B80EE66
:1092E9007E0B12850B7F5A78C41291F31291FB12EF
:0792F900936412836F78C437
:109300001293BC78C61291F31291DE129396751CDB
:109310000012836F78C61293BC7F6578C81291F3F0
:109320001291FB12936412836F78C81293BC78CAAF
:109330001291F31291DE129396751C0012836F78CE
:10934000CA1293BC303C14E53B24F4500B78C9E6B8
:109350002410F618E63427F61293C212AECF127E0E
:10936000F102DD46C2247E15E51C128460F51CD294
:10937000247E1BE51B128460F51B1023E77E21E58C
:109380001A128460F51A1023E67E27E5191284600C
:10939000F5191023E822C2247E2DE51B128460F506
:1093A0001BD2247E33E51A128460F51A1023E77E5F
:1093B00039E519128460F5191023E622ECF608EB62
:1093C000F622129C4678C8E6FE0886073395E0FD33
:1093D000FC12B23D7FE87E037D007C0012B52112B5
:1093E000B23D78CAE6FE0886073395E0FDFC12B46C
:1093F000FA12B23D7F807E697D677CFF12B4FAEC81
:1094000012B27412B23D7F3F7E807D0D7C1D12B181
:109410004912B23D7F3D7E407D007C0012B23D7816
:10942000BC12B2FA12B14912B23D7F3E7E807D007D
:109430007C0012AF3B12B23D78BC12B2FA12B149B5
:0994400012B23D7F3F7E807D00E9
:109449007C0012AF3712B23D78B412B2FA12B149A8
:1094590012B1C1783C12B3067F407E807D007C004A
:1094690012B23D783C12B2FA12B14912B3A012B24B
:109479003D7F3F7EA87D007C0012B23D78B812B2D4
:10948900FA12B14912B14912B23D7F407E007D0006
:109499007C0012B23D783C12B2FA12B14912B3A063
:1094A90012B23D7F3F7EC07D007C0012B14912AFF0
:1094B9003B12B23D78B812B2FA12B14912B23D78F4
:1094C9003C12B2FA12AF3B785412B30612B38A783F
:1094D9005812B30612B23D12B14912B23D78C01208
:1094E900B2FA12B149784412B306785412B2FA1298
:1094F900B3A0783C12B30612B23D12B14912B23D83
:1095090078BC12B2FA12B149783C12B3067F3E7E9A
:10951900C07D007C0012B23D783C12B2FA12B1490A
:1095290012B23D7F3F7E007D007C0012AF3B12B23C
:109539003D783C12B2FA12B14912B23D7F3F7E80AA
:109549007D007C0012AF3B12B23D78B412B2FA1220
:10955900B149787012B30678C4E6FE0886073395D8
:10956900E0FDFC12B23D7FE87E037D007C0012B570
:109579002112B23D78C6E6FE0886073395E0FDFC68
:1095890012B4FA12B23D7FE07E5E7DF87CFF12B420
:10959900FAEC12B27412B23D7F3F7E7F7DE57CC941
:0595A90012B23D7870D4
:1095AE0012B2FA12B14912B1C1785012B3067F3F0E
:1095BE007EF07D007C0012B23D783C12B2FA12B100
:1095CE004912B23D7F3F7EC07D007C0012AF3B1240
:1095DE00B23D783C12B2FA12B14912B23D7F3F7ED3
:1095EE00807D007C0012AF3B783C12B30678BC1233
:1095FE00B2FA12B23D7F3F7E807D007C0012AF3703
:10960E0012B23D783C12B2FA12B23D78B412B2FAEE
:10961E0012B14912B149784012B306785412B2FA17
:10962E0012B3D8783C12B30612B23D12B149787417
:10963E0012B3067F417E107D007C0012B23D78C0D1
:10964E0012B2FA12B14912B23D7F407E807D007C8B
:10965E000012B23D784412B2FA12B14912B23D7FF5
:10966E00417E207D007C0012AF3712B23D7844124D
:10967E00B2FA12B14912B23D7F407E407D007C00AD
:10968E0012B23D787412B2FA12B14912B23D7F4055
:10969E007EA07D007C0012AF3B12AF3B12AF3712A3
:1096AE00B23D785012B2FA12B14912B23D78501250
:1096BE00B2FA12B14912B23D7F3D7E2A7DAA7CAB31
:1096CE0012B14912B23D7F3F7E007D007C0012AF89
:1096DE003712B23D783C12B2FA12B23D787012B225
:1096EE00FA12B14912B23D784012B2FA12B1C11259
:1096FE00B23D785012B2FA12B14912B23D78501200
:10970E00B2FA12B14912B14912B23D785412B2FAFC
:0C971E0012AF3712B23D7F4A7E517DD25F
:10972A007CCB12B14912B2AF78AC12B3067F407E3D
:10973A00007D007C0012B23D787412B2FA12B1496F
:10974A0012B23D7F3F7E807D007C0012AF3B12B299
:10975A003D784412B2FA12AF3B12B23D785012B2BF
:10976A00FA12B14912B23D785012B2FA12B1491244
:10977A00B23D785012B2FA12B14912B23D7F3E7E22
:10978A002A7DAA7CAB12B14912B23D785012B2FAC4
:10979A0012AF3712B23D785812B2FA12B1C112B2F0
:1097AA003D7F4A7E517DD27CCB12B14912B2AF12B3
:1097BA00B23DAF3AEF3395E0FEFDFC12B23D7F4079
:1097CA007E7E7D057C0012B52112B23D7F607E75DA
:1097DA007D587CFF12B4FA12B4FA78B012B3067844
:1097EA00AC751B641298118F1C78B0751B671298A0
:1097FA0011E51C75F00AA42FFF249C50027F007803
:10980A00D7E654802FF62275390012B2FA12B23D09
:10981A007F0A7E007D007C0012B5CDA81BE513F6F9
:10982A0008E512F608E511F6335004EFF404FF22B6
:10983A00C23D78647BAC12922BD23D78677BB01222
:10984A00922B129C467F007EE47D577C0012B23D2B
:10985A0078AC12B2FA12B4FA12B23D7F007E537D8E
:0E986A00077C0012B5CD12B25C85133B7F80E7
:109878007ECB7DA47C0012B23D78B012B2FA12B44D
:10988800FA12B23D7F407E7E7D057C0012B5CD1276
:10989800B25CE513F56F04F53A85126E85116D8596
:1098A800106C7F407E7E7D057C0012B23D786C1284
:1098B800B2FA12B52112B23D7F607E0C7DA27C0007
:1098C80012B23D78B012B2FA12B4FA12B50D786C31
:1098D80012B30678AC12B2FAEC12B27412B23D7F2F
:1098E800347E9C7D2B7C5F12B149785412B30612EA
:1098F800B38A785012B306786C12B2FAEC12B274CA
:1099080012B23D7F347E9C7D2B7C5F12B14912B22E
:109918003D785012B2FA12B149784012B3067F402E
:109928007E007D007C0012B23D785412B2FA12B16A
:109938004912B3A012B23D7F3D7EC07D007C00126B
:10994800B23D78BC12B2FA12B14912B23D7F3E7EE6
:10995800C07D007C0012AF3B12B23D78BC12B2FA57
:1099680012B14912B14912B23D7F3D7E407D007C63
:109978000012B23D78BC12B2FA12B14912B23D7F60
:109988003E7E807D007C0012AF3B12B23D78BC1257
:10999800B2FA12B14912B23D7F3F7E807D007C0051
:1099A80012AF3712B23D785412B2FA12B14912AF5F
:1099B8003712B23D7F407E807D007C0012B23D7838
:1099C8005412B2FA12B14912B3A012B23D7F3D7ED1
:1099D800707D007C0012B23D78BC12B2FA12B14917
:1099E80012B23D78BC12B2FA12B14912B14912AFA3
:1099F8003B12B23D78B412B2FA12B149785812B398
:109A080006785412B2FA12B3A0783C12B30678540E
:109A180012B2FA12B3D8785412B306783C12B2FADA
:109A280012B23D12B14912B23D78BC12B2FA12B16B
:109A380049783C12B3067F3E7EC07D007C0012B29E
:109A48003D783C12B2FA12B14912B23D7F3F7E0016
:109A58007D007C0012AF3B12B23D783C12B2FA1284
:109A6800B14912B23D7F3F7E807D007C0012AF3B42
:109A780012B23D78B412B2FA12B149787012B30634
:109A8800785012B2FA12B23D12B14912B23D78C002
:109A980012B2FA12B149784412B306785412B2FAE3
:109AA80012B23D12B149787412B306784012B2FA74
:109AB80012B23D12B149783C12B3067F407E807DD8
:109AC800007C0012B23D784412B2FA12B14912B2C7
:109AD8003D7F417E107D007C0012AF3B12B23D7885
:109AE8004412B2FA12B14912B23D787412B2FA12A3
:109AF800B23D7F407EA07D007C0012AF3712AF3BA5
:109B080012B23D783C12B2FA12B14912B23D7F3D11
:109B18007E2A7DAA7CAB12B14912B23D7F3F7E00FE
:109B28007D007C0012AF3B12B23D785412B2FA129B
:109B3800B23D787012B2FA12B14912B23D783C12B5
:109B4800B2FA12B14912B14912B23D785812B2FABA
:109B580012AF3B12B23D7F3F7E7F7DE57CC912B1DB
:019B680049B3
:109B690012B23D7F4B7E187D967C8012AF3B12B2BC
:109B7900AF12B23D7FE87E037D007C0012B5CD12A5
:109B8900B25C78C8A61208A61308A60608A6077824
:109B99007412B2FA12B23D7F3F7E807D007C0012C2
:109BA900AF3712B23D784412B2FA12AF3B12B23D4E
:109BB9007F3E7E2A7DAA7CAB12B14912B23D784024
:109BC90012B2FA12B14912B23D783C12B2FA12B18C
:109BD9004912B23D784012B2FA12AF3B12B23D7F40
:109BE9003F7E7F7DE57CC912B23D787012B2FA12D0
:109BF900B14912B14912B23D7F487EF47D247C00FF
:109C090012AF3B12B2AF12B23D7FE87E037D007CFA
:109C19000012B5CD12B25C78C4A61208A61308A624
:109C29000608A607223F3F4344454647484A4B4C4E
:109C39004D4E5051525354555657583F3FE4F539FC
:109C4900F5A7909C5A791078B4E493F6A308D9F94A
:109C59002232A5C24A4A19DC3A885CDB3BFFD6DCD2
:019C69003BBF
:10AECB00D2D58002C2D575A70490040078107F0BF1
:10AEDB0012AEF778267F0512AEF7783C7F2212AEC2
:10AEEB00F7786A7F0F12AEF775A7002230D506E60A
:10AEFB00F008DFFB22E0F608DFFB22D2D58002C28E
:10AF0B00D575A7049006FA78737F0612AEF775A76E
:10AF1B000022DA0CD902800BD906303701B3500569
:10AF2B0002B0AA923702B096D9F680F9D2368002D7
:10AF3B00C23612B0DB303606C86002B237C8923662
:10AF4B00DAD0D9E4B8000A12B122A236923702B095
:10AF5B007F60FBB51300400F12B122A23692F7A20D
:10AF6B00379236A2F79237C398F40424E740DF24D4
:10AF7B0019AD29AC28AB277A00C394084008CDCC77
:10AF8B00CBCAE4CD80F424086010F9C3ED13FDECBB
:10AF9B0013FCEB13FBEA13FAD9F1A236303701B3EA
:10AFAB0040308A17E5102BF518E5113CF519E51221
:10AFBB003DF51A501A13F51AE51913F519E518137F
:10AFCB00F518E51713F5170513E5137002051402B1
:03AFDB00B035E4AA
:10AFDE00C39AF517E5109BF518E5119CF519E512C6
:10AFEE009DF51A500DB237C378177F04E496F60814
:10AFFE00DFFA7A047019E513C39408F5135002159D
:10B00E0014E4C517C518C519F51ADAE802B0D6202A
:10B01E00E7BAE5137002151415137817C37F04E60B
:10B02E0033F608DFFA80E8E51A20E7137817C37FB6
:10B03E0004E633F608DFFAE513700215141513E56E
:10B04E00173378187F03E63400F6500E08DFF775D5
:10B05E001A800513E51370020514E51420E75470E9
:10B06E0027E513604E046020851A12851911851884
:10B07E00105326F0AC10AD11A237E51313FFE512F5
:10B08E0092E7FEA81302B25CE4F512F511F510F585
:10B09E00147513FF5326F043260580D8E5FFF512ED
:10B0AE00F511F510751400F513D2375326F043261B
:10B0BE000980C15326F0432603E4F512F511F5106D
:10B0CE00F514F513C23780AC5326F080EC79017A73
:10B0DE00018512F0E513A2F7339237751400F513BC
:10B0EE006002D2F785F012A813B8FF0809E512C264
:01B0FE00E76A
:10B0FF006001098C278D288EF0A2F7EF3304700AB8
:10B10F000AC2F705F00AD5F0011A146002D2F785CA
:10B11F00F02922C88813C512C529C512C511C52823
:10B12F00C511C510C527C51022DA03B8000302B038
:10B13F00AAD9028002D9F702B09612B0DB303701DC
:10B14F00B392377004D9E78005DADEB8000302B096
:10B15F00D6D9E2C3947E500215142513F51350026D
:10B16F0005147815760008B81BFA78277915E608C4
:10B17F00FAE8FC78108AF0E608A427F709E5F0371B
:10B18F00F7500989F00907E760FBA9F0B813E61932
:10B19F0019ECF8B82AD802B03502B0C1B8FFFA02DC
:10B1AF00B0AAD9FB02B096DAF6B800F002B0D61208
:10B1BF00B31212B0DB303701B392377007D9E3B84F
:10B1CF0000E280DBDAE1B8000280E1D9D5C8C3988C
:10B1DF0050021514247F50020514F513781A7600C7
:10B1EF007A1A7B80C3E5109527E5119528E512950E
:10B1FF00294016C3E5109527F510E5119528F5118F
:09B20F00E5129529F512E64BF653
:10B21800DA0302B035EB03FB30E703187600C3E529
:10B228001033F510E51133F511E51233F51240CA64
:10B2380030E7DD80B6E53905396010D0F0D0E0C0E0
:10B2480010C011C012C013C0E0C0F08F138E128D51
:10B25800118C1022E539146010D0F0D0E0D013D052
:10B2680012D011D010C0E0C0F01539227920800C1E
:10B278007910800479087D007E007F003392D550D4
:10B288000312B2ECEC33400FEF33FFEE33FEED3335
:10B29800FDEC33FCD9EE22EECCF5F0747E29A2D574
:10B2A80013FF92F7AEF022EF8EF0A2F7D2F73392A7
:10B2B800D5C3947F5006E4FFFEFDFC229420400491
:10B2C80074FF80F304CCFEE4FFFAE5F0CC6012C30F
:10B2D800CC13CCCD13CDCE13CECF13CF0450EEDA92
:10B2E800EC30D5D7C3E49FFFE49EFEE49DFDE49CCB
:03B2F800FC22E64F
:10B2FB00FC08E6FD08E6FE08E6FF22ECF608EDF694
:10B30B0008EEF608EFF622CFC513CFCEC512CECD81
:10B31B00C511CDCCC510CC22E4F513F512F511F502
:10B32B001022E493FCA3E493FDA3E493FEA3E49324
:10B33B00FFA322C0E012B23D12B14912B37112B396
:10B34B002DD0E0C0E012B23D12B36812B14912B277
:10B35B003D12B32D12AF3BD0E0D5E0E722AC48ADA8
:10B36B0049AE4AAF4B228C488D498E4A8F4B227483
:10B37B00FF7809FFFEFDFCE52654F048F526221266
:10B38B00B43104A2E1927F1420E01590B4B274049E
:10B39B0012B33E802912B43130E102B27F20E0EBD0
:10B3AB008C4C8D4D8E4E8F4F90B4C6740412B33EA1
:10B3BB0012B23DAC4CAD4DAE4EAF4F12B149307FDA
:10B3CB0004EF6480FFEE33EF337001FF2212B431D0
:10B3DB00C0E08C4C8D4D8E4E8F4F90B4EA7403129F
:10B3EB00B33E12B23DAC4CAD4DAE4EAF4F12B14968
:01B3FB00EC65
:10B3FC00C54CFCEDC54DFDEEC54EFEEFC54FFF90A7
:10B40C00B4DA740312B33ED08212B23DAC4CAD4DE3
:10B41C00AE4EAF4FE58230E00712B1C1B27F809DD6
:10B42C0012B1BE8098EE33EF3324605007D0E0D0D9
:10B43C00E002B37AEFA2E7547F927FFF12B23D7C19
:10B44C00837DF97E227F3E12B149EE33EF332481A6
:10B45C00501012B23D12B2AF12B274EFB2E7FF123B
:10B46C00AF3BEE33EF33602A2403F8C313FFEE92A5
:10B47C00E7FEE82481E4501A12B23D12B2AFEF0499
:10B48C00C2E0FCF58212B27CEFB2E7FF12AF3BE5F3
:10B49C008203FAEE33EF33600B148FF0A2F713FF35
:10B4AC00EE92E7FEEA2283FA703AE4E9AABCF8E0ED
:10B4BC00813EE6E99DBF0000803F1A3C2839666951
:10B4CC0099BBE335A33DE75D25BFDB0FC93FCCDB63
:10B4DC008D41EE3649C43F91C9453DF8B0C50000D9
:10B4EC00803F34F517C373FA2F45DDFD0AC6EF25EF
:10B4FC0013FFEE3512FEED3511FDEC3510FC02B2EA
:10B50C005CC3EF9513FFEE9512FEED9511FDEC95D6
:10B51C0010FC02B25CEFF88513F0A4FFE513C5F044
:0AB52C00CEF9A42EFEE435F0CDFAAE
:10B5360088F0E512A42EFEED35F0FDE433CC85133C
:10B54600F0A42CFCE5128AF0A42CFCE51189F0A4E9
:10B556002CFCE51088F0A42CFC89F0E512A42DFD46
:10B56600EC35F0FCE51188F0A42DFDEC35F0FC8AF5
:10B57600F0E513A42DFDEC35F0FC02B25CE4CCF84A
:10B58600E4CDF9E4CEFAE4CFFB75F020C3E513333E
:10B59600F513E51233F512E51133F511E51033F520
:10B5A60010EF33FFEE33FEED33FDEC33FCEF9BEE95
:10B5B6009AED99EC98400CFCEF9BFFEE9AFEED9904
:10B5C600FD0513D5F0C622C2D5EC30E705B2D5127B
:10B5D600B2ECE51030E70DB2D512B5F012B5831214
:10B5E600B2EC800312B58330D515C3E49513F51379
:10B5F600E49512F512E49511F511E49510F5102273
:10A6B000E57124885002D2191256DC8E4712D21B43
:10A6C000129189125A98305E0F125A3612887812F7
:10A6D000596712C02112425412393A1247FB103600
:10A6E00029201F1C301219E412A83612A84B12A9F7
:10A6F0004B12A96D30510302A9F712ACC8205109C1
:10A70000C251E4F552F545F5442275A7007583075B
:10A71000E559C454F0F582E0F538A3E0F518A3A399
:10A72000A3E0F51E74FF12A8361256DC8E1C8F1B98
:10A730007510DF751100E51164B4700612A801757B
:10A74000111012A7CE4028AE1CAF1B125764203246
:10A750001EAC03AB027A0C125371ED701275A70098
:10A76000758304851182ECF00583E510F00511D5A1
:10A7700010C412A80175C70375C6E075A70490053B
:10A78000007F0412A7BCDFFB75A700122B83125AAF
:10A7900036E4F5A7F8F559758307E8C4F582E06556
:10A7A000387011A3E06518700BA3A3A3E0651E70B9
:10A7B0000388592208C3E5589850DC22E0F5BCE034
:10A7C000F5BDE0F5BEE0F5BF124EE605C622E51088
:10A7D00075F004A4F5C685F0C775B901E5BC334032
:0BA7E0001F05C605C675B90185BE64E3
:10A7EB0085BF6505C675B90185BC6685BD6785BE28
:10A7FB006885BF69C322E51124FE502E75A7007F23
:10A80B0010AE111E7583048E82E0FD1582E0CDB56E
:10A81B0005005012F00582CDF00583E0FD1582E0B6
:10A82B00CDF00582CDF0DEDCDFD72275A754900486
:10A83B000005A79005007FB4F0F0DFFC75A70022A0
:10A84B0012BE75C2517B077AFFE4FFF5A790040097
:10A85B0012A931ED244C4035EC603075A7008D8288
:10A86B0005A712A8F77583058D82E02410401CF014
:10A87B0005A7E02CF0500505A7E004F0BA000CBBCF
:10A88B000009D251EF24DC50027F23DFC3EA6005BD
:10A89B0012A8AA8006EB600312A8E275A70022306B
:10A8AB00E0047553082230E1047553182230E2049A
:10A8BB007553282230E3047553382230E404755362
:10A8CB00482230E5047553582230E604755368224C
:10A8DB0030E7037553782230E0047553882230E15A
:10A8EB00047553982230E2037553AA22ED54F0C439
:10A8FB00232390A901735302FE225302FD2253021C
:06A90B00FB225302F722BB
:10A911005302EF225302DF225302BF2253027F224E
:10A921005303FE225303FD225303FB225303FB2255
:10A9310012BDAD12BC3BE4F5F7C2B2C2B2ADF7F540
:10A94100F7C2B2C2B2ACF7D2B22290050078B4E03D
:10A951006015FD54F0C4CD7C00540FFE1583E0FF5B
:10A9610012546FEFF005830582D8E42275830478D1
:10A97100FF088882E060FAF5D38812E512244C5072
:10A98100012285D3D288D4881279FF0512E512609D
:10A99100F00908E875F0B484A8F08882E060ECF56D
:10A9A100D3B9000280D5B9230050D0C395D292D13A
:10A9B1005002F40409FEE4FFFCAD0112547C740161
:10A9C100FA25D475F0B484A8F0AC06AB0712536332
:10A9D100EB30E7010CE5D22C30D1029C9C8882F04F
:10A9E1000AEAB501DCE512244C50012285D3D28557
:10A9F10012D4A812809390040012AAB68C068B057B
:10AA010012AAB6E4FFF512F5118C148B13C3ED9B5A
:0EAA1100F9EE9CFA4012E51199E5129A500AEE
:10AA1F008C148B138A1289118F528F82E0F9C3ED38
:10AA2F0099FDEE9400FEE582245A5002244C75F0F5
:10AA3F00B48485F082E0FA2DFDEE3400FEEB9AFB34
:10AA4F00EC9400FCE92BFBEC3400FC0FBFB4B0E539
:10AA5F005224D3400224B4F552C3E51333FBE5145B
:10AA6F0033FCE511FE2BFBE512FF3CFC1254D1E940
:10AA7F00F890AAC893F511FDEBF513FFECF514FE52
:10AA8F007C0012546F8F44E890ABC893FAAB13ACB1
:10AA9F001412539AAF03AE04AD117C0012546FEF32
:10AAAF007002F552F545227C007B007F5AE02BFBAC
:10AABF00EC3400FC0582DFF522B4B4B4B4B4B4B402
:10AACF00B4B4B4B4B4B4B4B4B4B4B4B3B3B3B3B33C
:10AADF00B3B3B3B3B3B3B3B3B2B2B2B2B2B2B2B23F
:10AAEF00B2B1B1B1B1B1B1B1B0B0B0B0B0B0B0AF4F
:10AAFF00AFAFAFAFAEAEAEAEAEAEADADADADADAC6A
:10AB0F00ACACACACABABABABAAAAAAAAA9A9A9A98E
:10AB1F00A9A8A8A8A8A7A7A7A7A6A6A6A5A5A5A5BB
:10AB2F00A4A4A4A4A3A3A3A2A2A2A2A1A1A1A0A0F2
:10AB3F00A0A09F9F9F9E9E9E9D9D9D9D9C9C9C9B2C
:10AB4F009B9B9A9A9A99999999989898979797966B
:10AB5F0096969595959494949393939292929191AE
:10AB6F0091919090908F8F8F8E8E8E8D8D8D8C8CEE
:10AB7F008C8B8B8B8A8A8A89898988888887878733
:10AB8F008686868585858484848383838282828179
:10AB9F0081818080807F7F7F7E7E7E7E7D7D7D7CBC
:10ABAF007C7C7B7B7B7A7A7A7979797878787777FE
:10ABBF007776767675757574740002030506080945
:10ABCF000B0C0E101113141617191A1C1D1F21220E
:10ABDF00242527282A2B2D2E303133343637393A76
:10ABEF003C3D3F404243454648494B4C4E4F5052E7
:10ABFF0053555658595A5C5D5F6061636466676868
:10AC0F006A6B6C6E6F707273747677787A7B7C7EFA
:10AC1F007F80818384858688898A8B8D8E8F9091A2
:10AC2F00929495969798999B9C9D9E9FA0A1A2A464
:10AC3F00A5A6A7A8A9AAABACADAEAFB0B1B2B3B43D
:10AC4F00B5B6B7B8B9BABBBCBDBEBFC0C0C1C2C331
:10AC5F00C4C5C6C7C7C8C9CACBCCCCCDCECFD0D040
:10AC6F00D1D2D3D4D4D5D6D7D7D8D9DADADBDCDC66
:10AC7F00DDDEDEDFE0E0E1E2E2E3E4E4E5E5E6E7A6
:10AC8F00E7E8E8E9EAEAEBEBECECEDEEEEEFEFF0FC
:10AC9F00F0F1F1F2F2F3F3F4F4F4F5F5F6F6F7F769
:10ACAF00F8F8F8F9F9FAFAFAFBFBFBFCFCFDFDFDED
:10ACBF00FEFEFEFEFFFFFFFFFFC251E4F544F81456
:10ACCF00FB900400A9007C0FC2D112ADE3E824056C
:10ACDF00F8B8B4F08B13E5122403FA244C5001FAA0
:10ACEF00BBFF012275112C8A1912AE1A8F16203D47
:10ACFF0012AA1975112312AE1A8F15751600303D51
:10AD0F00E2801175112312ADC2751500303D05E8B3
:01AD1F002F04
:10AD200013F51575111212ADC2751400303D05E80A
:10AD30002F13F514EA2404F552244C5002F552E482
:10AD4000F51AF51BF51CE516600AFB7A00AF137EB9
:10AD5000FF12AD88E515600AFB7A4FAF137EFF1234
:10AD6000AD88E516600DFB7A00E5146006FF7ECF26
:10AD700012AD88AE1CAF1B7C00AD1A12546F8F450C
:10AD8000EF2513F544D25122EFF5F0A4FCADF0EB22
:10AD9000F5F0A49CFCE5F09DFDEB8AF0A4FAABF085
:10ADA000EF8EF0A49AF8E5F09BF9E833F8E933F96F
:10ADB0007B00125515051AE51B2BF51BE4351CF518
:10ADC0001C22EA2511F9244C5001F9C2D112ADE13F
:10ADD000303D428F00C3EA9511F9500324B4F9D2F3
:10ADE000D17C09E4FDFEFF8982E060062FFFE43E8E
:10ADF000FE0D09B9B4027900DCEDED20D118F51E85
:10AE000024FE923D500F12547CEFB503005006858E
:10AE10001E1FFB881222F51D80E612ADC2203D43A5
:10AE2000740212AEB912ADC2203D38740412AEC124
:10AE300012ADC2203D2D740612AEB912ADC2203D36
:10AE400022740812AEC112ADC2203D17740A12AEB0
:10AE5000B912ADC2203D0C740C12AEC112ADC220AD
:10AE60003D0122C3E89F605088148F158A16400860
:10AE70001ABAFF0A7AB380060ABAB4027A0012AD8F
:10AE8000C2303D34C3E89FF9602EC3E5149515FB2D
:10AE90006930E7D4E930E703F404F9EB30E702F472
:10AEA00004C3995002AA16E5142515C82F28FFE4FB
:10AEB000FC33FE7D0412546F222AFA244C5001FA0E
:0BAEC00022C3CA9AFA500324B4FA22FD
:10BC0200758000C2B212DE3CD2B275F83022758065
:10BC120000C2B2F5F7C2B2C2B2D2B222758000C27D
:10BC2200B2F5F7C2B2C2B2856CF7C2B2C2B2856BCC
:10BC3200F7C2B2C2B2856AF722758000C2B275F746
:10BC420003C2B2C2B2856FF7C2B2C2B2856EF7C288
:10BC5200B2C2B2856DF72212BC92740612BC107485
:10BC62000212BC1E8FF7C2B2C2B2D2B222909F6F32
:10BC72007F631276F012DD46D214120E9412766EA3
:10BC8200124EE612BC92740612BC1074C712BC109B
:10BC920012BC9840FB22758000C2B275F705C2B291
:10BCA200C2B2C2B2C2B275F705C2B2C2B2C2B2C2A7
:10BCB200B2E5F7D2B2A2E022120E9485BF6C85BE25
:10BCC2006B756A00E56B7015E56A701112BC9274AF
:10BCD2000612BC1074D812BC1ED2B2D21F22E54B7F
:10BCE2000475F03C8485F04B12BF9D852E72E55F92
:10BCF200030354C0F8E55E543F28F57C3055012219
:10BD020012BD3712BC9840F7E54C60F312BC921298
:10BD1200BD4E12BD1C80F112BC92C21F740612BC31
:10BD220010740212BC1E787086F708B880FAD2B27C
:10BD320012BD6B808F787075A704758304E54CC4BF
:0CBD4200F5827F10E6F0DFFC054C801954
:10BD4E00787075A704758304154CE54C30E701E453
:10BD5E00C4F5827F10E0F6DFFC75A7002274102573
:10BD6E006A54F0F56AE4356BF56BE4356C540FF5F7
:10BD7E006C22E54B75F010A4256A54F0F56AE5F0D7
:10BD8E0080E4E56A24F054F0F56AE56B34FFF56B58
:10BD9E00E56C34FF80D7E56A24FF80ECC380EBE5C9
:10BDAE006D24F054F0F56DE56E34FFF56EE56F34ED
:10BDBE00FF540FF56F2212BE1C12BE44C22DC25488
:10BDCE00C255E57F7002D255147002D254E54A3046
:10BDDE00E00122B4061C20540D12BD9012BEEC12CE
:10BDEE00BF7C12BFB42212852F7E0412DE34754A38
:10BDFE00012220550D12BD6B12BF5B12BF9D12BEEC
:10BE0E00C52212852F7E0412DE34754A0522740374
:10BE1E0012BC1E7870E4F5F7C2B2C2B2A6F708B82B
:10BE2E0080F3D2B222740312BC1EE4F5F7C2B2C282
:10BE3E00B2E5F7D2B222E575F8541F30E40244E0C1
:10BE4E00F57585722EA2779226E57C543F30E50279
:10BE5E0044C0F55EE57C54C02323F55FE57FC2E761
:10BE6E0079BCF709A77E22856C6F856B6E856A6D2E
:01BE7E0022A1
:10BE7F00856F6C856E6B856D6A22E4FEFF740775A6
:10BE8F00A704F5838E8274FFF0DFFD75A70022747F
:10BE9F00067E007FB012BE8EE4F55AF55B2275A7C1
:10BEAF0004758306E55A600A75F00A84E5F070029E
:10BEBF00740AC4F58222307720E55A240240020525
:10BECF005A12BEADE55AF0E573F0E574F0E575F082
:10BEDF00E576F0E577F0E578F075A700223077F991
:10BEEF0012BEAD7F1074FFF0DFFDE55A24F550034D
:10BEFF0012BF17155AE55AB4FF02055AC3E55A95F2
:10BF0F005B50D6755B0080D112BE757F0A056D053B
:10BF1F006D12BC3BE4F5F7C2B2C2B2E5F7D2B23054
:10BF2F00E704DF02800512BDAD80E2056D12BC3B58
:10BF3F0012BEADE55A24F6F07F06E4F5F7C2B2C2A1
:10BF4F00B2E5F7F0DFF4D2B275A70022053FE53F67
:10BF5F00B43C17753F00053EE53EB43C0D753E0001
:10BF6F00053DE53DB41803753D00024ABB153FE59D
:10BF7F003FB4FF17753F3B153EE53EB4FF0D753ED1
:10BF8F003B153DE53DB4FF03753D17024ABB054226
:10BF9F00E542B43C0F7542000541E541B43C0575DF
:0CBFAF0041000540221542E542B4FF0F9E
:10BFBB0075423B1541E541B4FF0575413B154022E8
:10BFCB00AC40AB41A842EC75F03CA42BFBE435F044
:10BFDB00FC7A3C125363EB28FBE43CFC22AC3DABFC
:10BFEB003EA83F80E178AE8604AB3EE53FC313F835
:10BFFB00800C7800120E5DE5BE75F005A4FBE5BF65
:10C00B0075F03CA42BFBE435F0FC7A1E125363EB6A
:10C01B0028FBE43CFC2212BFFDAE04AD0312BFF0C3
:10C02B008C148B13120E67E5BFFF24F650027F01B1
:10C03B00E5BE75F096A4AAF0F9C3ED9513FBEE954A
:10C04B0014FC924E4B701120110E30480B75364B71
:10C05B003003037536FFD22E304E02DF1F7A0212E9
:10C06B00536375A7009004EEECF0A3EBF0C3E5BFB0
:10C07B009F04BF0102D2E79005CBF022ED29FDEE24
:04C08B003AFE80B544
:10DE210012DE2A12DE2A12DE2A7E0480067E02809B
:10DE3100027E017F0080087F6480027F017E00EF07
:10DE41004E6012E4FD0D1D0DEDC394AD40F7EF1FC3
:10DE510070ED1E80EA22753500C200C201C20222A5
:10DF0800F5D8D2DCE5F520E7FBE5DA540FFEAFD90A
:04DF180075D8002296
:10DB0F007F767E06909C7E127702740412DF087C6B
:10DB1F00007D5212546FEFF875F00A84C0F07F76D3
:10DB2F007E2312D4F57E29742E12D5087E2ED0E0D6
:10DB3F0012D4F57E35745612D5087F6B7E1190DBAB
:10DB4F007812D534E824E04001220423F824E7506A
:10DB5F0002781812DB68D8FB227F6CE82411FE795B
:10DB6F000512DE610E0FD9F922071DFFFFFFE080BE
:10DB7F00000020C0000038E0000008F0000038F876
:07DB8F00000020FFFFFFE092
:10DB960012DBBE30E6022409540F75F00AA4F5150F
:10DBA60012DBBE30E6022409540F25152212DBBE15
:10DBB600540F2275F000800875F044800375F00755
:10DBC600E4206D09D5E0FAD5F0F7D24C229247C28F
:10DBD600ACE54F623885504FA26E926D859950C262
:10DBE6006FD2ACC24CA2472212DBF8C4FA12DBF8A1
:10DBF6002A2212DBBE20E603540F225407240922F0
:10DC0600E612DC0D18E608FAC412DC13EA540F44D7
:10DC160030F924C6E950112407800D75F00A84C036
:10DC2600F012DC2CD0E0443030530975F00085E06A
:10DC3600E0D5F0FA3099FDC299F599623822E538B7
:10DC460080F2E53812DC0D800812DC2EE53812DC95
:10DC56002E740D12DC2E740A80CE744012DC2E74E3
:10DC66004080C5742C80C1742E80BD75380080B884
:10DF2E0085A0835383FE438380858384F0758400AC
:01DF3E0022C0
:10D9BD0074A212DF2E74A112DF2E74A612DF2E7444
:10D9CD00A412DF2E74C012DF2E742512DF2E12DA90
:10D9DD004D75C70375C6FC75B90112B606740812EC
:10D9ED00DF08EE75F020A4FEEF54F80303032E2498
:10D9FD0092C313FE24EA50027E16EE90DA3693257A
:10DA0D00BCFE24E6501F24E8401B748112DF2EEE6D
:10DA1D0012DF2E12DA5A744012DF2E742F12DF2EFF
:10DA2D0074AF02DF2E7E2680E1F7F7F8F8F9FAFBE6
:10DA3D00FCFDFEFF000000000101020202030303D2
:10DA4D00A8BCA9BDAABEABBFACC7ADC62288BC8958
:0ADA5D00BD8ABE8BBF8CC78DC622A8
:10DD4600C006C007C5F075A7019000007EB7E58C38
:10DD5600240340FA12DD681EBEAFF3C5F0D007D02B
:10DD6600062275A700EE12DF2E741012DF2E740441
:10DD760012DF2E85A08343838185838475A7517F17
:10DD860020E0F0E0F0E0F0E0F0DFF6E4F5A7F5845F
:01DD9600226A
:10DF1C0075A711900000E4C583F0C58330E2F8F5D5
:02DF2C00A7222A
:10DE6100EF20E723EE20E71F20E61C05A7C454039B
:10DE7100F583EE5408C42FF582EE5407240983F587
:10DE8100F0E045F0F005A7228040201008040201CF
:10DE9100EF20E723EE20E71F20E61C05A7C454036B
:10DEA100F583EE5408C42FF582EE5407240983F557
:10DEB100F0E055F0F005A7227FBFDFEFF7FBFDFE95
:10D4B500FDA42582F582E5F03583F583ED229060A4
:10D4C500AC7A0475F00512D4B57D05805E7A0580C9
:10D4D500027A04547FC0E0C083C082C39420500107
:10D4E500E490605C12D4C8802E9061BA7A058005FC
:10D4F5009062777A0675F00712D4B57D07802C7A8D
:10D505000580027A06C0E0C083C082C39420500122
:10D51500E490620712D4FAD082D083D0E022905FE3
:10D52500D075F00A12D4B57D0A7A07C2D18002D22D
:10D53500D1C0A7C082C083C007C006C0E030D109F2
:10D5450075A704E493FDE493FAEEFB75A704EBFEDF
:10D55500EAFC7901D9067908E493F5D4E5D423F5F5
:10D56500D420E01612DE910EDCEA0FDDE1D0E0D02A
:10D5750006D007D083D082D0A72212DE6180E89042
:10D585005F1075F00E12D4B57D0E7A0812D5309065
:10D595005FB875F00212D4B5E493FDE4A393FACE17
:10D5A5002408CE7C0812D5B17C06AD02ED23FD2002
:0ED5B500E00712DE910FDCF42212DE6180F737
:10D3A000F5D2C2D58036F5D2D2D58030F5D224F66A
:10D3B00050090E0E24A650030E0E0EE5D2F5D275BE
:10D3C000F0648485F0D3C2D57009D2D5742012D50B
:10D3D00008800312D4F5CE2406CEE5D375F00A8476
:10D3E00085F0D3700A30D507742012D50880031257
:10D3F000D4F5CE2406CEE5D312D4F5E5D222F5D26B
:10D4000075F0648485F0D3C2D58022F5D2C2D58070
:10D4100025F5D2D2D5801FF5D275F0648485F0D37E
:10D42000C2D57009D2D5742012D508800312D4EE6B
:10D43000CE2405CEE5D375F00A8485F0D3700A308A
:10D44000D507742012D508800312D4EECE2405CE61
:10D45000E5D312D4EEE5D222F5D2C2D58035F5D28D
:10D46000D2D5802F30E70DF404C0E0742D12D4D64D
:10D470000E0ED0E0F5D275F0648485F0D3C2D5707D
:10D4800009D2D5742012D4D6800312D4C3CE24047A
:10D49000CEE5D375F00A8485F0D3700A30D50774D1
:10D4A0002012D4D6800312D4C3CE2404CEE5D312E6
:05D4B000D4C3E5D22207
:1076E700909F6F1276F002DD467E00800E7405FED5
:1076F700F51EE4FFF51DF51F203C3375A700E49345
:10770700700122A3B40204051D8003B4010A051FFA
:10771700EF2409FFAE1E80E612D5087D06B44002AD
:107727007D03B421027D02EE2DFE80D27E0075A777
:1077370000E493700122A3B40204051D8003B40181
:107747000F051FEF2407FFAE1E80E612D4D2800874
:10775700B45B0050F612D4D60EB4210280D30EB417
:10776700400280CDB42C0280C80E0EB45F0280C1E7
:10777700B45B0040BC0E0E80B8E60812D508EE24B4
:1077870006FED513F422909CAC307409909CB0305F
:107797007303909CB502770275F019D5E0FDD5F01B
:1077A700FA12484F12DC60744F12DC71744B12DC12
:1077B7004FC322C2501277FE12484FD2AC12DBB928
:1077C700304C1212DBB9304C0C12DBB9304C06D2FC
:1077D70050C2ACD322B440E512DBBEB4400312DB87
:1077E700BEB44FED12DBBEB44BE712DBBE12DBBEFD
:1077F70012DBBEC2ACC32230530975F008D5E0FDD9
:10780700D5F0FA227F0575F019D5E0FDD5F0FA120B
:10781700484F12DC60745712DC71745012DC2E74FE
:097827008112DC2EE56312DC2E57
:10783000E56212DC2E78D0E612DC2E08B8D7F8E626
:10784000F8795F30E702792FE912DC2E12DC2E1274
:10785000DC2E12DC2E745812DC2E744312DC2EE463
:1078600012DC2EE8C2E775F00A84C425F012DC2E83
:107870007864E612DC2E08B869F8E612DC4F12775D
:10788000BA400122DF02800A20508B75F000808010
:10789000D250C2ACD3221277FEC25012484FD2ACA3
:1078A0002002EF12DBB9204CE7B440F412DBBEB487
:1078B000400312DBBEB457DAF53812DBBEB450D247
:1078C00012DBBE12DBBEF56312DBBEF56278D012AE
:1078D000DBBEF924A0500353015FE924E0400279A4
:1078E0005FA60108B8D8E8780612DBBED8FB12DB29
:1078F000BEFC53040FC4540F75F00AA42CFC249C46
:1079000050027C0078D78601E4B92F02D2E72CF62A
:10791000786412DBBEF608B86AF812DBBEE53860A0
:107920000302789212DBBE12DBBEC2ACC32290A36C
:10793000748003909FB57F2012773312DD4602DEFC
:1079400032753400C26B1279FD12DE32127DADE564
:1079500016600312795902025912800F121E461244
:10796000DD4610002010010280F8127E185013121C
:107970001E5112792E10000D10010280F8121DF315
:0579800080D7127B9D81
:1079850022C26BD22775480A122B77753400127EF6
:10799500E5C26A1233CF106A0512024A80ED12025F
:1079A5004A127D3F127E97127EF178D0E6642660FA
:1079B5004412800F121E4612DD46100038100102D7
:1079C50080F8127E18501BE965156018121E5112B9
:1079D500792E12DE2A10001D10010280F8121DF307
:1079E50080BCD26B127EC3751607855917122BF012
:1079F5007535008096020259127DAD127A1F127EEE
:107A0500F17F19127A3990A3A17E121277357E2360
:107A1500E51602D47490A4EE80EF7862E4127A3011
:107A250078D0745F127A3018E4F6227F08F608DF02
:107A3500FC227F7B7E007810742012D4D6CE2404DD
:107A4500FED8F5227F197E081277357E28909F97FC
:107A5500305303909F9C027735C26B127A1F127ABE
:107A650069020259C251127EF190A399127A491204
:107A75001E19127DAD7F20127A0812DD46E51670BB
:107A85000512DE27803675A6FF3051031277A8123E
:107A9500484FD2AC200025306DFA127899400C126F
:107AA5007E184011127B9DD25180BB105003127974
:107AB50033C25180D1D25112792E80CAC2AC22D2A2
:107AC5002775480A122B77753400C26B127EE5C202
:107AD5006A1233CF106A0512024A80EB12024A126B
:0D7AE5007D3F127E97127EF1127AF550DA85
:107AF200020259909FB0127A49121E2B12DD46C320
:107B020010001310010510020E80F412780B4001D0
:107B12002212793380DDD3C2AC22D227C26B7548E0
:107B22000A122B77753400127EE5C26A1233CF1027
:107B32006A0512024A80EDD26B127D3F127E9712C5
:107B42007D6775B901E5BCB2E7F5BC124EE6751664
:107B520007855917122BF080CB127DADE516601FF9
:107B620078D0E53D127B8EE53E127B8EE53F127B9F
:107B72008E765A08765F12C839127EC3027D7E7FE6
:107B82003E7E11909F8612770202DD4675F00A84CE
:107B92004430F608E5F04430F60822D26B127EC378
:107BA200127D7EE51775F01084240AF54824E8500A
:107BB2000375480A122B838558592275320012BE6A
:107BC2008975A704900700751500127D6775B901C4
:107BD200E5BC20E705E515F0801004600D648260C5
:107BE2000975BCFF75B90575B9020515E51524209F
:107BF20050D8E58224FE4003027C96A882187F00BA
:107C020075A7007583078882E0FE75F004A4127DD3
:107C120012A9BCAABDABBEACBF1582E0FD75F004D3
:107C2200A4127D12C3E995BC404C7052EA95BD4046
:0D7C320045704BEB95BE403E7044EC95BF95
:107C3F004037703DEE75F004A404127D12A9BCAA62
:107C4F00BDABBEACBFED75F004A404127D12C3E949
:107C5F0095BC4015701BEA95BD400E7014EB95BE98
:107C6F004007700DEC95BF5008EEF00582EDF01552
:107C7F0082E5826009C3EF95825003027C0A0FC32D
:107C8F00E89F4003027C0275A70490070075C703A5
:107C9F0075C6A8E0F5BCE0F5BDE0F5BEE0F5BF7533
:107CAF00B90575B90205C6E58224204006E5C6244C
:107CBF002050E00875C70375C68075B901E5BC1281
:107CCF007CFCF5BCE5BD127CFCF5BDE5BE127CFC71
:107CDF00F5BEE5BF127CFCF5BF75B90205C6E5C65A
:107CEF00245850D6E5320470FB75A70022B4FF016B
:107CFF0022F975A704900700E582686005E06970B6
:107D0F00F7E922F5C685F0C775B901E5BC645F7068
:107D1F000375BC27E5BD645F700375BD27E5BE64C1
:107D2F005F700375BE27E5BF645F700375BF2722C1
:107D3F0075C703E54875F004A42480F5C6E55975A9
:107D4F00F00484A8F00825C6F5C675B901A9BCAA28
:077D5F00BDABBEACBF8615F1
:107D660022E515242050037515DFE51575F004A4EA
:107D760054FCF5C685F0C722E51724204028E517F0
:107D860075F00484A8F00824A8F5C675C70375B96C
:107D960001A9BCAABDABBEACBFA61589BC8ABD8B6A
:107DA600BE8CBF124EE622E4F516F51579FF127D5C
:107DB6006775B901E5BCB4FF040516A9150515E5F7
:107DC60015242050E9891579FF75C70375C6A8756E
:107DD600B90109E5BC04601B09E5BD04601509E5A8
:107DE600BE04600F09E5BF04600905C6E5C6242088
:107DF60050DD09891722751600751501127D677504
:107E0600B901E5BC20E70205160515E51524205045
:107E1600EB227900E975F004A454FCF5C685F0C799
:107E260075B901E5BC20E73078D066702B08E5BD52
:107E360066702508E5BE66701F08E5BF6670190501
:107E4600C675B90108E5BC66700E08E5BD66700822
:107E560008E5BE667002D32209E9242050B6C32283
:107E6600127E86127E6EA8017F08E0F608DFFB22EE
:0B7E7600127E86127E7EA8017F08E6C7
:107E8100F008DFFB2278D0796275A704758307EBD0
:107E9100C454F0F58222127D6778D0127EB1E5BC20
:107EA100F9C23C20E702D23C127EB17862127EB167
:107EB10075B901A6BC08A6BD08A6BE08A6BF0805DF
:107EC100C622127D6778D0127ED3127ED3786212D9
:107ED1007ED386BC0886BD0886BE0886BF08124EC2
:107EE100E605C622125A3612DF1C12866E02DD46E4
:107EF10012DF1C7F007E0990A3861277027F0A7E23
:107F010012E5150412D3AC7F1412CA23121DF37F9C
:107F1100277E0875130778D0127780E6793E30E71F
:107F210002792F7E34E912D5087F3D7E0190A50AA2
:107F310012773520311B3030031291A9C23B1281D7
:107F4100A1127F57D23B1281A1127F691281E88071
:107F51007C12C08F80E6C23B7F44745320170274A9
:107F61004E7E0012D5088017D23B7F4F74572017E1
:107F71000274457E0012D5087E06E51E12D4F57EF8
:107F81000CE51D12D4F57E12E51C12D4F57E177492
:107F91008112D5087E1CE51B12D4F57E22E51A124A
:107FA100D4F57E28742E302602742712D5087E2D32
:107FB100E51912D4F57E33E51812D4F57E39302651
:0F7FC10007742C12D5047E3BE53702D4F5742DDE
:107FD000201702742B7F707E1512D508127FEC7E5D
:107FE0003A12D3557E0190A5350277027E1BE51C1F
:107FF00012D4F57E21E51B12D4F57E27E51A12D4A2
:10800000F57E2DE51912D4F57E33E51802D4F5126C
:10801000808D1280B812838F127EF11283E72017B1
:108020001E10021B1248F012C839128075121DFE74
:108030007F347E2F12778D127F2A12DD4680E21266
:108040001DF3203026203128C23B1281A11280CDA1
:1080500078661282A1D23B1281A11280E278691265
:1080600082A11281E812815C02834412927280F232
:1080700012C0A480EDE57D75F01084AAF075F00AB9
:10808000A42A547FFA78D7E654802AF6227F277EE6
:108090000879D08700C001D224B9D002C22412844A
:1080A0006ED001A70010230909EE2406FEB9D7E31C
:1080B0002219EE24FAFE80DB7E3479D7E7A2E7921C
:1080C0001712841B79D7E7A21792E7F722C224C2BE
:1080D0003B751E007F447E0012842B801E1023ED12
:1080E000802AD23BC2247F4F7E00128433D2247E6A
:1080F00006E51E128460F51E1023E7D2247E0CE5EF
:108100001D128460F51D303BD41023E1D2247E1271
:10811000E51C128460F51C1023E17E1CE51B128413
:0381200060F51BEC
:108123001023E67E22E51A128460F51A1023E87EF6
:108133002DE519128460F5191023E87E33E5181232
:108143008460F5181023E87E393026027E3BE5373C
:10815300128460F5371023E3227F707E1512842387
:10816300C2247E1BE51C128460F51CD2247E21E50B
:108173001B128460F51B1023E77E27E51A12846027
:10818300F51A1023E67E2DE519128460F5191023E4
:10819300E87E33E518128460F5181023E82278D7B7
:1081A300E6C2E775F00A847866F537303B057869EF
:1081B30085F03712821130262BE53775F003A404BE
:1081C3000475F00584FBE51975F00AA4251875F00C
:1081D30006A42BFBE435F0FC125585F537125585C3
:1081E300F5188B1922E563FC339217AB6250031227
:1081F30055F6305C0A7AD21253717840125513AE99
:1082030004AF037C277D1012547C8F1C8037E6FD5E
:1082130033921718860418860350031255FE7A0901
:10822300792778C01255108B1EADD3ACD2AB06792B
:10823300EA786012550E8B1DAF06AED27C177D70A7
:1082430012547C8F1CAF05AE047C037DE812547C72
:0F8253008F1BAF05AE047C007D6412547C8F1A24
:10826200ED75F00A84F51985F01822EC3392175057
:10827200031255F6751D30301786751D2D808178D5
:10828200427B607CEA800678407B207C4E12C16F84
:108292007927781012550E8B1CAF06AED280AB3008
:1082A200262AE51975F00AA4251875F00AA42537BF
:1082B200FBE435F0FC7A051253638C068B077C00D5
:1082C2007D0312546F8E048F031281DBE51E75F05D
:1082D2000AA4251D75F00AA4251C75F006A4251B09
:1082E200FBE435F0FC7A0A125363EB251AFBE43CFB
:1082F200FC7A0A125371EB2519FBE43CFCE43DFDC8
:108302007A0A125383EB2518FBE43CFCE43DFD3072
:1083120017031255FEA60518A60418A60378D7E679
:10832200A2E7923DC2E775F00A84FCABF0303B0E47
:10833200AB37EC75F00AA42BA23D92E7F622AC37DC
:1083420080F012835F305C0A7A4012537178D21245
:1083520055133017031255F68C638B622212836F0A
:108362007A0A125363EB2518FBE43CFC22E51C75E8
:08837200F00AA4251B75F00AB6
:10837A00A4251AFBE435F0FC7A0A125363EB25199B
:10838A00FBE43CFC221283C112DE2EC202C223127B
:10839A0083C110000810010510021B80F51031ED91
:1083AA0010300D102604D22680E3D230C23180DD8F
:1083BA00D231C23080D7227F3590A4F3127733901E
:1083CA00A51120300F90A52D20310990A502202655
:1083DA000390A4FA1F7E1712770202DD467F357ECC
:1083EA0001909F621277357F347E3A128510744E5F
:1083FA0012D50812DD4612DE2EC2027F347E3AD230
:10840A001775115975124E802675112E751227800F
:10841A001E75113E75122F801675112B75122D803F
:10842A000E75114E75125380067511457512571245
:10843A008510E511301702E51212D50812DD461033
:10844A00000810010510020B80F5D23C1017E3D288
:10845A001780DF02850B4430F812846AE8540F2231
:10846A00C2218002D221A22492229223128510E8EC
:10847A0030E709D23C7430302102745FF812D50813
:10848A0012DD4610003410010510025D80F5D23C61
:10849A00102266102367B43909745F2021DF743013
:1084AA0080DBB45F04742D80D4B42D04744180CD74
:1084BA00B45A04743080C60480C3D23C30240610F7
:0F84CA002237102338B44104742D80B1B42D042F
:1084D900745F80AAB45F04743980A3B43009745AF4
:1084E90020219B74398097148094B48908D223E899
:1084F90012D508800DF8C223800874898001E8022A
:1085090084879085258003908521C007EF2408FF83
:1085190012D534D00702DD460205F8F8020500003D
:10DCE60075A70090DD1875F02D84C2D5C2D16017D6
:10DCF600D2D1146007D2D514600DC2D1E5F093FCE1
:10DD0600742D95F093FB22E5F093FB742D95F0931B
:10DD1600FC220009121B242C353E474F58606870C0
:10DD26007880888F969DA4ABB2B8BEC4CACFD4D92A
:10DD3600DEE2E6EAEDF0F3F6F8FAFCFDFEFFFFFFA1
:10DDE000D23D8002C23DED8BF0A430E70205F0C3C6
:10DDF000E895F020D50425F025F0FEED8CF0A43058
:10DE0000E70205F0C3E995F030D10425F025F0FFD5
:10DE1000203D0B2487500122EF24CC40012202DE5A
:01DE200061A0
:10D78400203A7A7E1C7F5312DE617F5912DE611EBD
:10D794007F5712DE617F5512DE617E2312DE617FC8
:10D7A4005712DE611E7F5912DE617F5312DE611F44
:10D7B4007E2012DE617F5A12DE617E1E12DE617FE0
:10D7C4005212DE61120E67E5BD20E0143006117FAF
:10D7D400357E1C90D840E571700390D84A02D53448
:10D7E400E5716018E57012DCE6781F79567D091240
:10D7F400DDE4303A0312D8130DBD16F3227E1C7FEC
:10D804005390D82912D534200CD612CA7F80C0C0B8
:10D81400060E30D5021E1E12DE61D0061F30D10264
:10D824000F0F02DE61070700386C446C38000505F1
:10D834002070D8702005057088A8887008071038F3
:10D844007CFE383838000807102844C628283800D9
:10C85E0090A53F7F717E23127735120E67E5BC7E61
:10C86E003112D4C330121AC23C120E67E5BCFB75EE
:10C87E00F00AA4F904FAC23D12BE7512CAFC303D8C
:10C88E000122DAF712CA037C00EBF4042E4019AD34
:10C89E000312546FEFA2D1203C077E237F6502D195
:10C8AE0022AE16AF1702C9A4AD0112546FEF12D209
:10C8BE0010203C077E237F6502D146AE16AF1702CD
:10C8CE00C9C87F567E0512CA2F7F3D12CA427F6F9E
:10C8DE0012CA4212CA7F7E0A7F4112CAB27E227FDC
:10C8EE005912CAB22012012212BE75857A1D855EBA
:10C8FE001C857B1B855F1A7AC0C23D12CAF8203D8B
:10C90E005212CA037C007D1412546F74562F20D11C
:10C91E00029F9FFF24CB40028037EF248850028075
:10C92E0030EA1475F00384FE12DE61C3E51B957BBD
:10C93E00FEE51A955F92D55004EEF404FEEEC31395
:10C94E00FE24E0400C741F2E30D5029E9EFE12DE99
:10C95E0061DAA8227F5212C9747F5A12C9747517F0
:10C96E0053751600802B7E0012DE910EBE12F92238
:10C97E007F157E28742012D5087F1C7E2812DE912A
:04C98E000EBE40F9A0
:10C99200223012E712C97E75171575162DD23C0288
:10C9A200C877C23D6002D23D92D175F080305C04FE
:10C9B200F5F08001A4A2E792D5E5F075F03284F893
:10C9C200E5F075F00584C0E0E5F0A2D533C0E0E8FB
:10C9D200601E12D4F5EE2406FED0E0F8D0E012D4A8
:10C9E200F5EE2406FE742C12D5080E0EE802D4F5DC
:10C9F2007420303D07742B20D102742D12D508808B
:10CA0200D4C3ED957AFFEC955EFE92D15003125598
:10CA1200E6227F1512CA1B7F327E3E12DE61DEFBEA
:10CA2200227E0912DE610EBE36F9227E0112DE611D
:10CA32000E0EBE3FF8227E3312DE610EBE40F92298
:10CA42007E047D1112DE610E0E0EDDF81F1F7E3593
:10CA520090A548305C057E3190A54C02773574056F
:10CA6200305C097E32740112D4C374067E3612D44D
:10CA7200C37E3A740012D4C37E3D02D4C37F417E8A
:10CA82001F7D0F12DE610F0F0FDDF8227F687D031D
:10CA920080047F677D0512DE610FDDFA227F667DED
:10CAA2000780F37E1F7F5012DE611F1FBF3EF822F8
:07CAB2007D0A12DE610E0E89
:10CAB9000F0FDDF722203D07123C767003D23D228D
:10CAC900056D12BC3BE4F5F7C2B2C2B2ABF7F5F79C
:10CAD900C2B2C2B2E5F7FA30E411EB251DF51DE447
:10CAE900351CF51C0519EA30E3010ED2B280157820
:10CAF9000380027801203D07123C767003D23D2263
:10CB0900D8F3056DE56D2409F56D12BC3BE4F5F725
:10CB1900C2B2C2B2ADF7F5F7C2B2C2B285F71BF520
:10CB2900F7C2B2C2B2E5F7FCD2B2543F30E50244D3
:0FCB3900C0CC54C02323F51AE56D24F6F56D2208
:10D6AB007E017F0990D72912D5342051097E037F43
:10D6BB0000743F02D508E4FEFFC3E54512CF7AFDA7
:10D6CB00940AED403D9464ED4002746312D3A67E40
:10D6DB00017F09E552240575F02D84AAF075F0053C
:10D6EB00A4CA75F00B842A90D7149312DCE6BCB84D
:10D6FB00027BB87D04EE2DF8EF2DF90D12DDE0DD88
:10D70B00FB227E0312D4F580C6000C1622222D3983
:10D71B00444F4F5A66707C7C87939EA9A9000909D8
:10D72B00080041000000000088800000000041005C
:10D73B000800120E7BE5BCB4F8339004C3E0602CF8
:10D74B00FA24F340277F137E0012DE610F0F12DEE7
:10D75B00610E12DE911F1F12DE910EDAEC7F147E2A
:10D76B000012DE610E12DE910EBE12F5229005CC78
:09D77B00E0C3941240F60480C7DB
:10CF7A00305D0A75F08AA42480E5F034002220741A
:10CF8A00157F017E1190D00212D5347F0A7E0AE500
:10CF9A002E540702D3BD7F087E1190D01212D534C9
:10CFAA0020730C7F0A7E1712DE910E0E12DE917F1D
:10CFBA00007E0BE57112CF7A12D3AC7F0C7E11E59D
:10CFCA0071602F0EE57064B4602864B475F0328421
:10CFDA00C0F012D4EECE2405CED0E075F00584C0A0
:10CFEA00F012D4EECE2405CED0E023302D01040277
:10CFFA00D4EE90886A027702070FFFFFC473BDAFB1
:10D00A00A463B5FBCDE7FFFF030F0100FFFE03801A
:10D01A00306701227F357E00748812D508E5516099
:10D02A001712CF7A75F06484F87E06E5F012D40BF5
:10D03A00E860E07E0002D4F57E003074D6307316C4
:10D04A0079BCE7FC09E7FB12530B781D201704E6AD
:10D05A0070011802D2D6909CB0027702202C0122CD
:10D06A0090D07002D534050EFFF0E01CF004F81CD5
:10D07A00FFF0301201227F637E00909CC712D534E4
:10D08A007F1512CA1B7F1F12CA1B7F2912CA1B7F58
:10D09A00177E06E53F30E00B90A55C305C0390A557
:10D0AA007080132074077E01909CE7800990A55137
:10D0BA00305D0390A566127702307306E54E600272
:10D0CA00154E205718E54EB40113120E8AC3E55CBB
:0DD0DA009560F5BCE55D9561F5BD124EE673
:10D0E7007F217E01E53F30E021305705909E128079
:10D0F70016E54E7005909E1D800D909CF3127702E9
:0BD107007E30E54E02D41112770222A8
:10D2780012530B7F207E05751900781DC2D5E63044
:10D28800D51712D4EEEE2405FE18B818F17E1F74D7
:10D2980063305C02748202D5087005B8191880E200
:10D2A800D2D5CE24FACE7484301702742D12D50844
:10D2B800EE2406FE80C8742012D50480C8781C802D
:10D2C8000D7F007E23AC5EAB7A12530B781DC2D55E
:10D2D800E630D50C12D4F5EE2406FE18B818F12263
:10D2E8007005B8191680EDD2D53017E4CE24FACEE1
:10D2F800742D12D508EE2406FE80D5742012D508A8
:10D3080080D512530B781DC2D5E630D51612D4C37A
:10D31800EE2404FE18B818F10E745E305C0274270F
:10D3280002D4D27005B8191680E3D2D53017DACEF8
:10D3380024FCCE742D12D4D6EE2404FE80CB7420A7
:10D3480012D4D680CBC23D12D3600F0F0E0E746379
:10D35800305C02748202D50812530B781DC2D5E6E0
:10D3680030D50C12D523EE2408FE18B818F1227017
:10D3780005B8191680EDD2D5301716740BCE24F8DF
:10D38800CE12D523EE2408FE80D5740C12D5238046
:08D39800D5303DCB740A80E59D
:10D854007F797E24E55F30E70122AC5F1CAB7B124D
:10D864005339E51B700E742012D508EE2405FE1200
:10D87400D8A2800C12D8A2E51B12D4EEEE2405FE29
:10D88400E51A12D4EEEE2405FE742C12D5080E0E01
:10D89400E51912D4EEEE2405FE745E02D508742D4B
:10D8A400201702742B12D508EE2406FE22E55F3001
:10D8B400E70122AC5F1CAB7B125339E51B700E747D
:10D8C4002012D4D6EE2404FE12D8FB800C12D8FB0E
:10D8D400E51B12D4C3EE2404FEE51A12D4C3EE24CD
:10D8E40004FE742C12D4D60E0EE51912D4C3EE2401
:10D8F40004FE742A02D4D6742D201702742B12D479
:06D90400D6EE2404FE2211
:10D112007F097E2530040512D20C8028A275E5799C
:10D12200C23D6002D23D92D175F080305C04F5F0D0
:10D132008001A4A2E792D5E5F075F03284F8E5F01B
:10D1420075F00584C0E0E5F0A2D533C0E0E8602ABE
:10D1520012D523EE2408FED0E0F8D0E012D523EE5B
:10D162002408FE0F0FE52B5403701F746012D508BC
:10D172001F1FEE2404FEE802D523740C303D067412
:10D182000A20D1010412D52380C9205904742E80AB
:10D19200DC205804747F80D5748080D1300405125D
:10D1A200D20C8028A275E579C23D6002D23D92D1AF
:10D1B20075F080305C04F5F08001A4A2E792D5E519
:10D1C200F075F03284F8E5F075F00584C0E0E5F022
:10D1D200A2D533C0E07F3E7E1CE8602012D584D009
:10D1E200E0F8D0E07F3E7E2812D5847F447E327400
:10D1F2002E12D5087F3E7E37E802D584303DE0749A
:10D202000A20D1010412D58480D59005CAE075F0B8
:10D212000A84F8E4C5F0C2D522301105E54AB40209
:10D2220050C39006E9E0957AFB9006E8E0955EFC33
:06D2320050031255F6EC5A
:10D23800C31360047B63800FEB13FB249C40F5242D
:10D248004F4004C20480079005CAEBF0D204900650
:10D25800E6E09006E8F09006E7E09006E9F0E55E83
:10D268009006E6F0E57A9006E7F02212D25680DEC4
:10CB4800E54424F64001227800E552206607C395A3
:10CB580070500224B40475F00384F9E928FE24C453
:10CB68005001FE12CB8A12CB961E12DE61C3E998E1
:10CB7800FE5003243CFE12CB8A1E12DE6108B81F49
:10CB8800DA22EE2420FE24C250032402FE22E824E6
:10CB9800F1E8C2D55006D2D5E8F4241F23FF90CC83
:10CBA8001893CF0493FAE545F5F0A4ACF0FB1253C3
:10CBB8009AE544F5F0A49BFBE5F09CFCEB2420FBF4
:10CBC800EC3400FC12CBF9FAE5458FF0A430E7020B
:10CBD80005F0E5F020D502F4042A75F005201903C4
:10CBE80075F00384FF24DF50027F20C374329FFF57
:10CBF80022EC24F0500BEB2460EC340090CC6893CA
:10CC080022EB33FBEC33FCEB33EC3390CC38932240
:10CC1800FF00FF03FA0BF318EA2ADE40CF58BE7371
:10CC2800AB8D96A880C068D64FE835F51BFD00FF90
:10CC380000080B0E101214151718191B1C1D1E1FA7
:10CC480020212223242526262728292A2A2B2C2D71
:10CC58002D2E2F2F303131323333343435363637A9
:10CC6800373839393A3A3B3B3C3C3D3D3E3E3F3F05
:10CC78004042444648494B4D4E50525355565859D8
:10CC88005B5C5D5F60616364656668696A6B6D6E55
:10CC98006F7071727374767778797A7B7C7D7E7F1A
:10CCA800808182838485868788898A8B8B8C8D8E08
:10CCB8008F9091929394949596979899999A9B9C12
:10CCC8009D9E9E9FA0A1A2A2A3A4A5A6A6A7A8A92F
:10CCD800A9AAABACACADAEAFAFB0B1B1B2B3B4B45E
:10CCE800B5B6B6B7B8B9B9BABBBBBCBDBDBEBFBF98
:10CCF800C0C1C1C2C3C3C4C5C5C6C7C7C8C8C9CADD
:10CD0800CACBCCCCCDCECECFCFD0D1D1D2D2D3D42A
:10CD1800D4D5D5D6D7D7D8D8D9DADADBDBDCDDDD80
:10CD2800DEDEDFDFE0E1E1E2E2E3E3E4E5E5E6E6DB
:10CD3800E7E7E8E8E9EAEAEBEBECECEDEDEEEEEF3D
:10CD4800EFF0F1F1F2F2F3F3F4F4F5F5F6F6F7F7A4
:10CD5800F8F8F9F9FAFAFBFBFCFCFDFDFEFEFFFF13
:10CD6800E54524FD400122E552206607C395705031
:10CD78000224B40475F00384241FFE24C250032443
:01CD880002A8
:10CD8900FE12CDC3EEFD241EFE24C250032402FE72
:10CD990012CDC3E544240275F00520190375F0038B
:10CDA90084F4042432FF24EE500F12CDB8AE051ED0
:10CDB9001E7C0512DE610EDCFA227F1512DE610F80
:05CDC9000FBF2DF82250
:10D5C3007E00206615E5700475F0B484E5F075F00F
:10D5D3000384FE6004C3743C9EFE745312D5EE7440
:10D5E3005712D5EE744E12D5EE74457F2F12D4D652
:10D5F300BE00077E3C12D4D67E00EE240875F03CB4
:10D6030084AEF00F0F0F12DE610E12DE610F12DE19
:10D61300611E12DE61EE240775F03C84AEF0223009
:10D62300745C301259E54AB4040122B4060122E5C0
:10D633007112CBE28F057C037E1E30662AE57004EF
:10D6430075F00384241EFE24C6501C24FB500424BE
:10D65300038013C00612D66AD0E024C67C0160069C
:10D663000C1460020C14FE12D6760EEE24C1400296
:10D67300DCF5228D0712DE610FEF24CE50F722E591
:10D6830053206607C39570500224B40475F00384D5
:10D69300241FFE24C250032402FE12D6A10E7F23B0
:08D6A30012DE610FBF2DF92218
:10DD9700AF177E00E53C12D3A07E0C742E12D50877
:10DDA7007E12E53B12D3A07E1E742E12D5087E2468
:10DDB700E53A02D3A07E0E78ADE612D40B7E187436
:10DDC7002C12D5087E1B18E612D40B7E25742C1254
:09DDD700D5087E2818E602D40BE1
:10CDCE007F797E00E54012D40B7E0A743B12D504A7
:10CDDE007E0CE54102D40B7F797E16743B12D5048E
:10CDEE007E18E53F12D40B7F797E0078AEE612D422
:10CDFE000B7E0A743B12D5047E0CE53E02D40B303A
:10CE0E005EE52043E27F6D7E0078AEE612D40B7EA7
:10CE1E000A743B12D5047E0CE53E12D40B7F757E50
:10CE2E000075F00A84E5F012D5230F0F7E08743AD0
:10CE3E0012D5041F1F7E0DE53F75F00A84C0F01257
:10CE4E00D523EE2408FED0E002D523851C1E851BBB
:10CE5E001FAB1BAC1C305D0A7A1B12537178321259
:10CE6E005513C3EB33FBEC33FC923D125342303D72
:10CE7E00087409F51DF51CF51B7F75E51D60157E03
:10CE8E002412D5237E2CE51C12D5237E34E51B12ED
:10CE9E00D523803D7E22E51C601912D5237E2AE51E
:10CEAE001B12D5237F787E31742E12D5047F75E543
:10CEBE001A8019E51B12D5237F787E29742E12D580
:10CECE00047F757E2DE51A12D523E5197E3512D510
:10CEDE00237F777E3C125CCC851E1C851F1B227F18
:10CEEE00397E1F12DE610FBF40F9781F79567A0026
:10CEFE007D1A12DCE612DDE4EA2406FABAAEF37805
:01CF0E001B07
:10CF0F00C3E5119570500224B4FA604214603E14C8
:10CF1F00603A2450603A146036EA24A540278A1EEE
:10CF2F00751D007D1912CF3F0D30740312CF3F0DC9
:10CF3F00781F7956AA1DEA12DCE612DDE40AD3EA5D
:10CF4F00951E40F2228A1D751EB380D70808080867
:10CF5F007F367E1C90D840E571700390D84A12D569
:0BCF6F00347F3CAE0090852102D534D9
:10DA6700787512DAB77453201702744E207406E5DE
:10DA77002E54074430AF1712DAE17E3BE57DC454DC
:10DA87000F12D4F52074077E07742012D508787812
:10DA970012DAB7E5172409FF7457201702744520D7
:10DAA7007402742012DAE17E3BE57D540F02D4F54F
:10DAB700E6FD3392171886041886033017031255AC
:10DAC700FE7917787012550E8B13AF06AED27C0015
:10DAD7007D6412547C8F148D15227E0012D5087E2A
:10DAE70007E51312D3BD7E19748112D5087E20E590
:10DAF7001412D3A07E2B742E2073030E742C12D510
:08DB0700087E2FE51502D3A0F2
:10DC7600E54A602E7A2420E00E7A26141460087A8B
:10DC860028141460027A297F667E01EA12D50820DC
:10DC96005505205406800B745B8002745C7E00126E
:10DCA600D50820110778A9B60007802130261EC2A4
:10DCB60026909D8A7F681276F07F66A85AE54AB458
:10DCC600060108E875F06484E5F012CE4720080FD7
:10DCD600E537640260097F367E2E744112D4D6225F
:10D90A0020144F740512DF08EF33EE33F9EF0303E7
:10D91A00541FF5F090D95DE993A4C5F013C5F0132F
:10D92A00C5F013C5F013C5F0135403FCE5F013FB5F
:10D93A00E9242093C9244093C39BC4540FFBE99C58
:10D94A00C4FC540FF9EC54F02B2446F57BE934F669
:10D95A00F55F22FFFFFFFFFFE6C5AD9C8F857D7750
:10D96A00726E6C6A696A6A6C6F747A828D9DB4D9B8
:10D97A00FFFFFFFAE9DCD3CEC9C6C3C0BEBBB9B745
:10D98A00B5B4B2B0AFADABAAA8A6A4A2A09E9C990A
:10D99A0096918C00381CE735D137246F00C5B3C186
:10D9AA00E61F66B60E68C21867AADBF4EDB94675BB
:03D9BA0010A200B8
:10DEE800D2A27408D2A1D2A300C2A3C2A1D2A30015
:10DEF800C2A3D5E0EF7405D2A300C2A3D5E0F822EF
:10DEC100C2A3D2A2D2A1D2A300C2A375F0083392F9
:10DED100A1D2A300C2A3D5F0F5C2A175F003D2A3CC
:07DEE10000C2A3D5F0F822F6
:10C4780012DEC1D2A300C2A3C2A175F008E4D2A300
:10C4880000C2A3A2A233D5F0F5FE75F008E4D2A34A
:10C4980000C2A3A2A233D5F0F5FFD2A300C2A32203
:10C4A800E478806608B88BFB70012274D512C478D2
:10C4B8007881C3EE13FEEF13F692D118EE2460F6DE
:10C4C80074D612C4787888EF33CE33CE33CE33CED9
:10C4D80033A2D192E25407FCEEFB7A08125363ECC4
:10C4E800244FF608EBF674D912C478EF543F7882DB
:10C4F800F67886EF33CE33CE33CE33CE335403F6CD
:10C5080008EEF618161608E6C4FF54F0F618E6C446
:10C51800CF540F2FF674DA12C478EF232354FC7823
:10C5280083F67884EEF608EF54C0F67880E466085F
:10C53800B88AFBF62212C4807889C3EF96FF18EEFA
:08C5480096FEA2E792165010C6
:10C550001255E6740FF8F91253B0EF2CFFEE3DFEC2
:10C56000788BEEF608EFF622E6182016072CF7E691
:10C570003D19F722C39CF7E69D80F66A405E80561F
:10C58000E050F04B0044803DC0384031D02BA02516
:10C59000601F2018D014000F000AA00144015801A8
:10C5A000680178018801A001B401D001EC021002F9
:10C5B00038026802A002DA030C034D78BE802085A1
:10C5C0008E8A9D8F4D95BA9A97A0BEA631AC53B274
:10C5D0002AB801BD6AC1EDC4D1C78812C480788D64
:10C5E000EEF608EFF67887798C1253B0788379905D
:10C5F00012C5687885798C1253B07881799212C50A
:10C6000068788DE624E4FE08E63392D13392D5545F
:10C61000FCFFEEA2D133A2D533FE780F79921253EC
:10C62000B078947990C3EC97F61819ED97F6799451
:10C6300090C57B7F1F7D11EF93C3971F19EF9397D1
:10C640001F091DED600240EF0F90C59B798DEF93A0
:10C65000F7090FEF93F7788E79941253B090C5BB1A
:10C66000EF93C39BFB1FEF939C2420FC7897E62B52
:10C67000F618E63CF618E436F6740612DF08D237F0
:09C68000EE24F7400624025002EA
:10C68900C237EEFCEFFD740712DF08C3ED9FFFEC24
:10C699009EFE78B7E6FD337C0050011CEF2DFFEEBE
:10C6A9003CFE789CEF26F618EE36F622201412206E
:10C6B900370F789DE6B4050912C76D12C7A212C7D4
:10C6C900EB2220145E7897799A12C81C12556EC312
:10C6D900EE9420FE924550031255E67C007D05122A
:10C6E900547C3045031255E6E531B40C3612DA4D67
:10C6F900120E80E5BC2FF560E5BD3EF56120E7111E
:10C7090024F8500DFAC3E5609AF560E5619400F5E7
:10C7190061120E8AE5BC2560F57AE5BD3561F55EE5
:10C7290012DA5A7897799AC3E697FB1819E697FCB3
:10C739007A0212536330370B7A02125363ECFEEB21
:10C74900FF800312C76D12C7A220140312C7EB782A
:10C75900957998E6F776000809E6F776000809E67C
:10C76900F7760022799CE77700FB19E77700FC78D8
:0CC779009DE6B40506EB33FBEC33FCEC52
:10C78500A2E792D550031255F67A32125371ECFB9B
:10C79500EDFC30D5031255F6ECFEEBFF22EE240836
:10C7A500FE74042037167406307511789DE6B405BD
:10C7B50004740C8007F42406C323540FFD7C001277
:10C7C500534F789FE6FC08E6FBC374109DFA12539D
:10C7D50071EFF8EEF912556EE878A02FF6FF18EE16
:10C7E50039F62480FE22927540031255E678BBE6A1
:10C7F500F5F02438400375F0E1EF33EE3378A8F611
:10C80500A485F07930E7020579C276307508E579B7
:10C8150024F15002D27622E627FB1819E637FC18D8
:10C8250019E637FD2212BE1C7F087871793A12C8C5
:10C8350045024ABB855E63857A62787379647F06B3
:10C84500E6F70809DFFA227864797380F17873795D
:09C85500AF80EB78AF797380E548
:1052E900E4FEFFFC7D0A791DE7540F2FFFE43EFE23
:1052F900B9190280061912534F80ED301703125560
:10530900E622305C2BEC33921750031255F6EC244D
:10531900D950047C277B007AD2125371EB33CC33FA
:10532900CD33CC33ED33FBEC33FC3017031255F698
:10533900EC33921750031255F67919125585F7096E
:10534900B91DF8A70322EFF88DF0A4FFEDC5F0CE43
:10535900A42EFEEC88F0A42EFE22EB8AF0A4FBE535
:10536900F0CC8AF0A42CFC22EB8AF0A4FBE5F0CC6B
:105379008AF0A42CFCE435F0FD22EB8AF0A4FBE5CD
:10538900F0CC8AF0A42CFCE435F0CD8AF0A42DFDF4
:1053990022EB8AF0A430E70205F0E5F0CC8AF0A40C
:1053A9002CFBE435F0FC2286F0E7FDA4FAABF019FA
:0653B900E786F0A42BFBC7
:1053BF00E435F0FC18E68DF0A42BFBEC35F0FCE4A3
:1053CF0033FDE687F0A42CFCED35F0FD22EB89F0E0
:1053DF00A4CBAEF08AF0A42EFEE5F03400FDEC89EC
:1053EF00F0A42EFEE5F03DFDE433CC8AF0A42DFDB4
:1053FF00E5F03CCEFC22EB89F0A4CBAFF08AF0A411
:10540F002FFFE5F03400FEEC89F0A42FFFE5F03E0E
:10541F00FEE433CC8AF0A42EFEE5F03CFCED89F0DF
:10542F00A42EFEE5F03CFCE433CD8AF0A42CFCE581
:10543F00F03D8E058C068F04FF22C2D5EC30E705B8
:10544F00B2D51255EEEE30E70DB2D51255E6125425
:10545F007C1255EE800312547C30D5031255E62290
:10546F00C3EC13C0E0ED132FFFD0E03EFEBC000BEA
:10547F00BE0029EF8DF084FFADF022E4CCF975F07A
:04548F0008EF2FFFF4
:10549300EE33FEEC33FCEE9DEC994005FCEE9DFEF5
:1054A3000FD5F0E9E4CEFD22EDF9F5F0EE8420D23C
:1054B3001CFEADF075F008EF2FFFED33FD400799AB
:1054C3005006D5F0F222C399FD0FD5F0EA22EC3352
:1054D300EE3400FEEF3400FF7D007A007900780996
:1054E300C3ED9AFDEE9BFEEF9CFFB392D54009ED11
:1054F3002AFDEE3BFEEF3CFFA2D5E933F9ED33FD88
:10550300EE33FEEF33FFD8D92279007A00C380153A
:1055130079007A00C3EA13FFE913FEE8132BFBEECD
:105523003CFCEF3DFDE4F5D2F5D333FE7F19C3EE2A
:1055330098FEE5D299F5D2E5D39AF5D3B392D54047
:105543000DEE28FEE5D239F5D2E5D33AF5D3A2D54F
:02555300EB3338
:10555500FBEC33FCED33FDDF0122EE33FEE5D23308
:10556500F5D2E5D333F5D380C3EDC454F0FEECC4D6
:10557500FF540F2EFEEF54F0FFEBC4540F2FFF2204
:10558500EC75F00A84FCEB54F025F0C475F00A8440
:10559500C4CBC454F025F0C475F00A842BFBE5F0A8
:1055A50022AC10AB11125585A904AD03FA7C197B09
:1055B50099125363AE04AF03EA75F006A4F8AC1272
:1055C500AB131255852875F00A8485F014F8EF2B76
:1055D500FFEE3CFEEF28FFE43EFEE43DFDE439FC32
:1055E50022C3E49FFFE49EFE22E4C39DFDE49CFCF0
:1055F50022C3E49BFBE49CFC22C3E49BFBE49CFCF0
:10560500E49DFD2275D4107B807A0079807800EACC
:0A561500F5F0A4FCADF0EBF5F0A4F5
:10561F00FEAFF0EB8AF0A4C333C5F033C5F092D5DB
:10562F002DFDC5F03EFEE430D501043FFFB5150D4D
:10563F00EEB51409EDB51305ECB51201224006EADB
:10564F0098FAEB99FBD5D40ABB0001220ABA0001E4
:10565F000B22C3E913F9E813F8EA28FAEB39FB80B8
:10566F00A478087B807D807C00EDF5F0A4FAE5F04E
:10567F008EF0B5F007EA8FF0B5F001224003ED9BF5
:10568F00FDD827BDFF0122EDF5F0A4F9A8F0ED0438
:10569F00F5F0A4C399FAE5F09813CA1329F9E83A7B
:1056AF00F8C3E99FE89E50010D22C3EB13FBED2BCE
:1056BF00FD80B6C374689511FB74019510FC8004CE
:1056CF00AC10AB117A0B79B81253DC80177473F8E6
:1056DF00F9E627FB0809E637FC0809E637FD30E74E
:0556EF00031255FEEB63
:1056F40033FBEC33FCED3323FD242083F8ED241C31
:1057040083FFED241883FAED241483F9EF99F9E863
:105714009AFA1253DCEF9DFFE89EFE22FFFFFFB6CC
:10572400FED7FD63FB5DF8C4F59BF1E3ED9EE8CF86
:10573400E379DD9ED743D06BC919C153B91CB07945
:10574400A7709E06943F8A237FB674FF6A045ECBDB
:10575400535B47BB3BF1300423FB17DE0BB2FF80E6
:10576400C21DC232532CF8C3E5679576FBE56895F4
:1057740077FCE5699578FD30E705D2611255FE2482
:10578400F05003125838AA06A907125405EC2480D5
:10579400E43DFBF9F51AE43EFCFAF519E43F600236
:1057A400D2321253DC8B128C138D148E15C3E56424
:1057B4009573FBE5659574FCE5669575FD30E70525
:1057C400D2621255FEEBF9F51FECFAF51DED6002FD
:1057D400D232303201221253DCEB2512F512EC35B1
:1057E40013F513ED3514F514EE3515F51540E102F6
:1057F400560912576420323BEB242E40D3EA24018D
:10580400CB3400FC7A07793D1253DCC010C0118EF2
:10581400108D118C128B13E4FCFD7E077FD012B522
:0E58240083851203851302D011D010BB00053E
:10583200BA0002D21D22B261C374809BFB74F59C34
:10584200FC74209DFD22204D69204866303F637F15
:10585200697E0112CA2F7E1F12CA9F75A70090048B
:10586200EDE0A2E792171392E7FC1582E013FB30FA
:1058720017031255F6BC003AEB603720E73420E6F6
:105882003110E513201707C3741F9BFE80027E1F91
:1058920012CA940EDBFA22FB2017097E00C3742081
:1058A2009BFB8008EB241FFE74209BFB12CA8E0E0A
:1058B200DBFA2275A700758307E559C4440FF58208
:1058C200E0A2E792522212C8521258B5C2E775F00E
:1058D2000A84FEAFF075A7045382F1786412593E30
:1058E200AE07786712593E75A700E57DC4540FFED6
:1058F200E57D540FFF7873125932AE07787612594C
:105902003274AF1256DE1257F68B148A1312092024
:10591200ACCCAB017A0A125363E5139B9004ECF012
:10592200FBA3E5149CF0FCA2E7923DD23F02C858CB
:10593200860308860408860518188006E0FBE0FC4A
:0A594200E0FD7A0A12538320E70CFF
:10594C00EB2EF608E43CF608E43DF622C3EB9EF69B
:10595C0008EC9400F608ED9400F622204D0920483E
:10596C0006C23F302A0522C23380F6E54824F640B1
:10597C00F5E5580460F075A700758307E559C42454
:10598C0008F582E0FEA3E0FF1209207437125A2AB0
:10599C00500B30381BC23878C586468013743212CF
:1059AC005A2A400C203809D23878C5A646754600CC
:1059BC00740D125A2A404A1258C8303D3820112210
:1059CC00204D1F20481C204019BCFF16EB243250E0
:1059DC0011D240120E62E5BF75F019A4F536D22E25
:1059EC00D22F205238E55965586032204D2F20486F
:1059FC002CD2338028201109204D062048037536FF
:105A0C0000303319204D1220480F1291460559C30E
:105A1C00E55895595003855859C233C2402229FB89
:105A2C00E435CCFCC3EB9FEC9E22E558B4FF01227D
:105A3C0085581175A704758307E54824F650028034
:105A4C005C201259202905202A02805112C852E4E8
:105A5C00F516F517751000125AC2E510700312C82E
:0B5A6C004C125ADB302910E51B2517F7
:105A7700F517F51BE51C3516F516F51C125AE81235
:105A8700C84C0510C3E511951050D175A70002C881
:105A970058E55AF51124F6500375110A75A70475D0
:105AA7008306751000125AC2125ADB125AE8051003
:105AB700C3E511951050EE75A70022E510C4F582D5
:105AC700E0E0F564E0F565E0F566E0F567E0F568C8
:105AD700E0F5692275A701125ED4123ED775A704B7
:105AE70022E9F0E51CF0E51BF022E510C454F0F5BF
:105AF70082E0F512E5822406F582E0F511E0F51C57
:105B0700E0F51B22E512B426157F757E34740D125D
:105B1700D52320442575110012CEED025C397F6D27
:105B27007E3BE012D508E5137E3512D508E5127ED7
:105B37002F12D50820440312CEED12CE59025C393C
:105B4700202852E558B4FF012275A704758307E59D
:105B570059F51030330965586005204802051012C1
:105B67005AF1E0F513305E07204304E5376095E00E
:105B77007F797E3D12D4D6E5137E3912D4D6E5124D
:105B87007E3512D4D630480B7F7F7E3512DE610E0C
:105B9700BE40F980392012012275A7047583068556
:105BA7005B10125AF1305E0A204307E53770030293
:025BB7005D5B34
:105BB900E512700B7E3A7F79745D12D508800D75F8
:105BC900F06484E5F07E397F7A12D458E537B4025F
:105BD90005128FDE8045B403028040E51C7006E59E
:105BE9001B24FB5036E511F964B4602F20062CE51F
:105BF90037600D200C0AC3E99570F9500324B4F9F4
:105C0900E912DCE6781D79547D1D90D832E53F20F4
:105C1900E00390D83912DDE412D534751779751679
:105C29001930280375161DE51264266003125C7C81
:105C390075A7009006E3E511F0A3120E7BE5BC758C
:105C4900F01970040475F014A4951BFBE5F0951C7C
:105C5900FC922450031255F6ECF0A3EBF0C24FC2AC
:105C690063EC700EEB24E64002D24FEB24C84002ED
:105C7900D26322E51C24ED402BAE1CAF1B125E9EA5
:105C89007C007D3212547CC005EFAF17AE1612D4DA
:105C990011CE2405CE742C12D5080E0ED0E0231295
:105CA900D40B801B125E95125CD6CE2405CE742CC3
:105CB90012D508CE2402CEE875F0058412D4EECEB2
:105CC9002404CE7422305D02748302D504EE243D8F
:0D5CD90050047EC37F4B7C017DF412547C8F
:105CE600C004C005EF6007AF17AE1612D411D00777
:105CF600D0067C007D3212547CA805EFAF17AE1695
:105D0600CE240ACE02D4EE125E95EE2450305D0308
:105D1600EE24A150047EC37F4B7C017DF412547C9B
:105D2600C004C005EF6007AF177E2F12D45ED00700
:105D3600D0067C007D3212547CC005EFAF177E374B
:105D460012D4C37E3B742C12D4D67E3DD0E075F0BF
:105D5600058402D4C37F6D7E2F746312D508E512C5
:105D660075F06484E5F07E3512D3A012CEED02CE36
:105D76005930480320740122E4FCF5A79006E3E0BD
:105D8600F9A3E0FE24FE40EFA3E0FF7D78E537604F
:105D960008304FE3200C2A800B120E67E5BD20E089
:105DA60010304F0DD206E57124FE5015125E8B8021
:105DB600107D3CE546600A7D141460057D0A14706A
:105DC600B6891112534F7D6F12546FBE00A9EF248E
:105DD600E240A4AD07E51112DCE6202404B2D5B2F8
:105DE600D1781F795612DDE4A806A907E511242DFE
:105DF60075F0B484E5F012DCE67407304F02740ED9
:105E0600FDFA12DDE4B2D5B2D112DDE4B2D5B2D1DB
:075E1600DDF0AD0212DDE436
:105E1D00850616850717B2D5B2D112DDE485061EAB
:105E2D0085071F7A03304F027A06E511241675F0A7
:105E3D00B484E5F012DCE6A816A917AD0212DDE474
:105E4D00DDFBE51124EA400224B412DCE6A81EA90C
:105E5D001FAD0212DDE4DDFBE5377021304F1E90E2
:105E6D00A614305D0390A6107F3C7E331277351259
:105E7D000E67E5BD20E00612CAA512D7D322C3E9ED
:105E8D009570500224B4F922E51B2402FFE4351C61
:105E9D00FE305D1ABEC305BF4D028012AC06AB07C6
:105EAD007A1B1253717832125513AE04AF03227858
:105EBD007379641256E01257F6751CC3751B4B208F
:105ECD0032048B1C8A1B22125EBC30320122AC19AB
:105EDD00AE1AA91DAF1FB90005BC00028010C3E9A1
:105EED0013F9EF13FFC3EC13FCEE13FE80E8BF298B
:105EFD00005006BE2900500122C3EF13FFC3EE135D
:105F0D00FE80EB3E7FE3E3E3E3E3E3E3E3E3E37F01
:105F1D003E0C1C3C7C7C1C1C1C1C1C1C1C7F7F3EDA
:105F2D007FE3E3E3070E1C3870E0E3FFFF3E7FE302
:105F3D00E3030F0E0F03E3E3E37F3E070F1F3F77EE
:105F4D00E7E7FFFF0707070707FFFFE0E0E0FEFFBA
:105F5D00030303E3E37F3E1E3F73E0E0E0FEFFE358
:105F6D00E3E3E37F3EFFFFE3E30303070E1C383853
:105F7D003838383E7FE3E3E37F3E7FE3E3E3E37FBF
:105F8D003E3E7FE3E3E3E37F3F030303E77E3C0015
:105F9D000000181818FFFF18181800000000000066
:105FAD00000000FFFF0000000000003FF00000387F
:105FBD001C38F00180C1F020F0FC0038F03FE0000B
:105FCD000000007CC6C6C6C6C6C6C6C67C183878D4
:105FDD001818181818187E7CC6C60C183060C0C664
:105FED00FE7CC6C6061C0606C6C67C0C1C3C6CCCCC
:105FFD00FE0C0C0C0CFEC0C0C0FC0606C6C67C3CDC
:10600D0066C0C0C0FCC6C6C67CFEC6C6060C18302F
:10601D003030307CC6C6C67CC6C6C6C67C7CC6C6FD
:10602D00C67E060606CC78000018187E7E1818006D
:10603D0000000000007E7E00000000000000000057
:10604D000000000000C6E2E2D2D2CACAC6C6C20033
:10605D000000000000000000008080A0C0A0003003
:10606D004020C08080C0A0A0000060A0600000A003
:10607D0040A05098D090882050A850888850A850A3
:10608D002060806000000040E040000000000080C3
:10609D000000E000000000000040002040800040B3
:1060AD00A0A0A04040C04040E0C02020C0E0E020C3
:1060BD004020E02060A0E020E0C02020C06080E013
:1060CD00A0E0E020404040E0A0E0A0E0E0A0E02023
:1060DD00C0004000400000800080002060E0602093
:1060ED0000E000E00080C0E0C080E0E0E0E0E00023
:1060FD000000000040A0E0A0A0C0A0C0A0C040A033
:10610D0080A040C0A0A0A0C0E080C080E0E080C022
:10611D0080806080A0A060A0A0E0A0A0E0404040F2
:10612D00E0202020A040A0A0C0A0A080808080E022
:10613D00A0E0A0A0A0A0E0E0E0A040A0A0A040C0F2
:10614D00A0C0808040A0A0C060C0A0C0A0A0608002
:10615D004020C0E040404040A0A0A0A060A0A0A072
:10616D00A040A0A0A0E0A0A0A040A0A0A0A0404062
:10617D0040E0204080E02020A870202070A8202042
:0D618D0008F030D0100000F0A8A8000000BD
:10619A00E0000000902048708898984000E0E0E015
:1061AA0000A0E0E0E04060301030604040E0404055
:1061BA0060909090909060206020202020706090E5
:1061CA0010204080F06090102010906010305090A5
:1061DA00F01010F080E010109060609080E09090D5
:1061EA0060F0102020404040609090609090606085
:1061FA00909070109060C0E0F0F8F0E0C0000000ED
:10620A000000000000000000000000506050007014
:10621A007050000078807008F000F8888888F800CC
:10622A00C0C8102040981800C0B098B0C0006020C4
:10623A0040000000000090D8FCD8900000246CFCBC
:10624A006C24000020A870A82000002020F820203C
:10625A000000000000000080000000F000000000C4
:10626A0000000000606000081020408000708888EC
:10627A00888888702060202020207070880810206C
:10628A0040F8F810201008887010305090F810105C
:10629A00F880F008088870304080F0888870F80824
:1062AA00102040404070888870888870708888788C
:1062BA0008106000606000606000000080000080DC
:1062CA0000002040F84020000000F800F80000001C
:1062DA002010F8102000708808102000200000000C
:1062EA000000000070888888F88888F08888F0881C
:1062FA0088F070888080808870E09088888890E034
:10630A00F88080F08080F8F88080F0808080708843
:10631A0080B8888878888888F888888870202020BB
:10632A00202070381010101090608890A0C0A090A3
:10633A0088808080808080F888D8A8A88888888803
:10634A0088C8A898888870888888888870F088881B
:10635A00F080808070888888A89068F08888F0A08B
:10636A00908870888070088870F82020202020206B
:10637A00888888888888708888888888502088884B
:10638A0088A8A8A85088885020508888888888506B
:10639A00202020F80810204080F800CCAC9CACCC1F
:1063AA000000CCD4E4D4CC0004781828C800FC40FF
:1063BA00A04018202018000000000000F80000008B
:1063CA0000A040A05000788888986870884030887B
:1063DA0070200000F0A8A8A8A878484848487888FB
:1063EA0070888080887020A88898A8C8888880507B
:1063FA0048FC485080304C5C6060603C00E0F0082B
:10640A000808F88044485C484480F880808080808E
:10641A008078484848484888B8A8A8E8A8A8B8880A
:10642A0088888888F808500070888888708080F08A
:10643A0088888888F8888888888888F090909090DA
:10644A0090F0A8A8A8A8A8A8F8888888F808080832
:10645A0050008888888878A8A8A8A8A8F808000002
:10646A000000000000000000000000008888888802
:10647A00E8A8E8A8A8A870A8A8A80000000000003A
:10648A000000000000000000000000000000000002
:10649A000000000000000000006000606000600072
:1064AA0060006060205020000000005090B890D03A
:1064BA0090886050500070705000882020887000CA
:1064CA000080C0A090F8003048B4B448300030488A
:1064DA00B4B44830FC0098D02058C800F8E8D880F6
:0A64EA00D8E8F8404050F850404058
:0300000002005E9D
:03000B0002B61327
:0C000E00206E06859950D26E32D26F32FF
:0E00230010990AC298206DE385994FD26D3274
:10003800E4F537F534F52F12DE57C229C22AC26813
:09004800C227C214C215022D9C4E
:03005B00022B2A4B
:10B606008530F0C5F065308530F060F722C0D0C0D7
:10B61600E0C0F0C0A775A700C083C08275D00875CA
:10B626008A00300503758A7A758CEA0532E5327030
:10B636000215320530E530640A6026201520E53112
:10B64600B40C0BE530B4010612BA8E12D90AE531F4
:10B65600B4180BE530B4060612BA8E12D90A02B82F
:10B666002DC2AFD2C075C07AD2AFF5300531E53103
:10B6760064197040F531201529C225C22C7D0A7443
:10B686000412DF08EF33EE339005CCF0EE24F540DC
:10B69600112402400B24014005DDE4022B2AD225A9
:10B6A600D22CE5A6600215A678B5E660011678B636
:10B6B600E6600116302E0BE5367007C22FC22E1239
:10B6C600B9BBE5367004C24B8002153678A9E66030
:10B6D600011678D8E66001160535E5357002153590
:10B6E600E590307B0B30E008D278C27BC200801A2E
:10B6F600307C0B30E108D279C27CC201800C307DEF
:10B706000930E206D27AC27DC202E59044F8F470AE
:10B7160003753500304A09E53324FA5003753305BD
:10B72600E5336005153302B7D2E590F4540770038C
:0DB7360002B7D2A2E09200A2E19201A2E2CD
:10B74300920230100320143D75330820001B201093
:10B753000C2011098013E59030E10E8006E53724B3
:10B76300FC40F3E543541FF53320100375A6FF2077
:10B773002E5D301004E536705620100C201109E5BB
:10B783003524F55003753304D21BD2A5D2A612B9C2
:10B79300BB75B44075B24078D8E6700205342027F3
:10B7A3002E20682B202928202A25A2107211501F31
:10B7B300E52054076019E53424375004C24A800F4A
:10B7C3002401400B200026200119D27D7534C820A6
:10B7D3001558E531702412DEE874E812DEC1802AC0
:10B7E30002B900E53724FC40E6D27C80DF3011DF6C
:10B7F300E53724FC40D9D27B80D275F00384E5F091
:10B8030070DE12C53D74E812DEC1E531B4060512DF
:10B81300C6B58016B40C0512C6CB800EB412051241
:10B82300C6B58006B4180312C6CBE59030E10530E7
:10B83300E202800620100820110520103C807D20A4
:10B8430027F82068F52029F2202AEFE53424304038
:10B85300E9240750E5600B205E088590F020F20292
:10B86300740190B87593D2A5201002C2A512B9A68F
:10B87300806FC8A08269554646202F12E536603C8A
:10B8830024AA500AE53675F01984E5F06040D2A683
:10B89300201002C2A6D2A5202F0C7418304B0274BC
:0EB8A3006412B9A6803BE53675F00C30480300
:10B8B10075F00684A2E0744640E9743780E5E52B13
:10B8C1005403600C20100E301106E54A6402600535
:10B8D10012B9C1800312B918101B08A25892A5A26F
:10B8E1005992A675A700D082D083D0A7D0F0D0E01E
:10B8F100D0D0201009C5A67003022B2AC5A632C2DA
:10B9010018B40202D21812C5DB30180874E412DE32
:10B91100C102B80D02B80878A7E5B4600924E04077
:10B9210005760002B9C1E534702920412220751F36
:10B93100300D1CE57924CE40167AFFE5B110E70100
:10B941000A2325B3F5B3EA35B4F5B4C313F5B2E66A
:10B9510060021622C2412075028075E579FF6058A8
:10B9610020120424FD5051206502C21CD265FF241F
:10B97100B050027F4FEF90BA3E9375C70375C6FC76
:10B9810075B90185BFF0A4E5F0F624F44002760C08
:10B99100301C2DE5BEC39FF5F0A4E5F024E0400383
:10B9A10075F020E5F0C21C79AA770375B300F5B4F0
:10B9B100C31375B100F5B222C26578A77680D24172
:10B9C10079AA7703D21CE4F5B3F5B4F5B1F5B22247
:10B9D100C26579A1E57924CE500DE720E7E276280A
:05B9E100301CDD743292
:10B9E60080BE7680E720E7D3E5799740CE79AAE74F
:10B9F600FAE5792323B4C500400274C42437300E17
:10BA060031F42437300D15F7BA0302FA0AC39AF552
:10BA1600B175B300EAF5B4C313F5B222101C07D210
:10BA26001C76C802B9A8763274FF200E02749B02F7
:10BA3600B9A8C313247E80CCFFF3E8DDD3C9C0B810
:10BA4600B0A9A29A948F8A85817D7975716E6B688B
:10BA560065625F5C595653504E4C4A4846444240D4
:10BA66003E3C3A383634333231302F2E2D2C2B2AA9
:10BA76002928272625252424232322222121202084
:10BA86001F1F1E1E1D1D1C1CD2B5C28EAE8DAA8D7B
:10BA9600AF8BAB8BE4F58DF58BD28E30140122780B
:10BAA600B6BE0007EF24E24002800806E624EC500A
:10BAB600027614206705E624F64005E4FEFAFFFB4D
:10BAC6007C007D0A12534F7C007D5E12546F8F51AD
:10BAD600EE60037551FFEAFC7A33125363EBF5F01F
:10BAE600A4E5F0CB8CF0A425E0C5F035E0CB92D5EB
:10BAF60025F050060BBB0002D2D530E7060BBB0083
:10BB060002D2D5ECF5F0A42BFBE5F03400FC30D5E1
:10BB1600010C78A6E6C39BFF18E608F6EB18F618A4
:0EBB2600E69CFE18E608F6EC18F63014012234
:10BB34007A0050040A1255E67C007D6E12546F8F11
:10BB4400F078A2E6A4FBACF0125585EBBA0002F43F
:10BB540004FAE4F8FFEA30E70118E5796006207595
:10BB6400031FF4042AF579EF38D27520E70860033F
:10BB74007579FF02C80EC2750470F5E579F40460A6
:10BB8400EFF57980EE120E5D78BBA6BC120E7BE554
:10BB9400BE78A2F624F65007E4F5BEF6124EE6127D
:10BBA4000D46E5BEF54824F65008E4F5BEF5481206
:10BBB4004EE6E5BFF54324F3503924F34035120E25
:10BBC4007178A1A6BCE5BF789DF61424FB500874D7
:10BBD40003F6F5BF124EE678B7A6BE120E67E5BDB2
:10BBE400A2E39266A2E49267035403C253B401022F
:0EBBF400D25322740DF5BFF543124EE680C009
:10005E0078FFE4F6D8FDF4F5A6D2B4D2C075C07A16
:10006E0075D75075AE1375AF017581D87590F8754B
:10007E00EFBC75FDFFD2A412DE2EC2A47450122B5B
:10008E0042758951D28C75A882D2BC12BC0212DE86
:10009E00E812C4B312BB8912D9BD122A087F407E62
:1000AE0001909C73127702124D4A12DE2E12DB0F54
:1000BE0012DD4612DE577C1412DE38300003022B9E
:1000CE002ADCF512489F753A001248EDE53A701693
:1000DE0012DF1C7F437E0690A3F612770212DD46D6
:1000EE003000FD022B2A75A6FF12489F12BB891203
:1000FE002A0812DD4612DE2A12DE5778B5761E1257
:10010E00D9BD12C4A8C215C214122A08909CBA7F77
:10011E00781276F0205E0A7F767E12909CC712D5FA
:10012E00347F4012DDBC7F497E0978AEE612D3A043
:10013E007E15743A12D5087E1AE53E12D3A07E269D
:10014E00743A12D5087E2BE53F20E00805A6E5A6F9
:10015E00700215A6E53F12D3A07F5312CA237F5714
:10016E007E0B12D2CD12D3557F602073030202088C
:10017E007E0BAC5DAB5C12D2D112D3557E311277B1
:10018E008D7F697E1212D8583025087E1290DB784A
:10019E0012D534E5A60303543FFDFE0D7F7312DE28
:1001AE00610F12DE611EDDF478B5E57124F64002B2
:0801BE00761E307419E660564C
:1001C6007F727E16744012D4D67E17E612D45E7EF7
:1001D6001F745312D4D612DD4610003710013710A3
:1001E600023712483FD2AC75369612DBBEB4E00534
:1001F600124935800AE53670F112488D12DE270263
:10020600010D2074097E2BE52E540712D4F57E17B6
:1002160002018C022B2A022D628072E53524C85019
:1002260049E59020E244D0E0D0E012027102735614
:10023600E53524D25034E59020E22FD0E0D0E0120C
:10024600DF1C8038E53524D25020E59020E21BD013
:10025600E0D0E012DF1C306B0B7F091276E7124FFD
:100266001E127BBD1202710206BE2212DF1C90A472
:10027600AF7F001276F012DD4602DE2712DF1C90F9
:10028600A4AF7F001276F012DD4612DE2AC215C236
:1002960014C227C26812DE57753701909DA7121C3B
:1002A600FF9002AB730200F70217C2020B56021F41
:1002B60012021F0E0206BE0206FB0273560202C699
:1002C60012DE5775370790A146121CFF9002D673AF
:1002D60002029302096B0209A50209D90202FA0277
:1002E60005AD0202C60202C60203180202FF024B55
:1002F600B30203261248F0805A7F517E00747212B0
:10030600D504121E5C40B9124E3512D9BD12BB89F6
:1003160080AE7F49A25E120D31925E120D5080A012
:100326007F64120E9E121E5C401DE5352480F47516
:0C033600F0198460157F727E1F12D4F550
:1003420012DD461001E810000280E30202C612BC70
:100352006F0202C6124EE612DE5775370290A31FD5
:10036200121CFF900369730202C6020EA8020F0D4F
:10037200020F61020FB6020FFA02100902035902BC
:10038200051302038980D0D21412DF1C7F147E056C
:1003920090A369127702121E1912DD46124868757F
:1003A200A6FFD2AC1000DE12DBBE204CF2B405EF89
:1003B200E4F511F514F5151204411204D51248683A
:1003C20075A6FFD2AC1000BD12DBBE204CF2B415F4
:1003D200051204C880E7B406E712047FE51424FC82
:1003E20050D5E4F56FF56EF56D12048B1204D5123B
:1003F200486875A6FFD2AC10004212DBBE204CF258
:10040200B415051204C880E7B406E71204B5E56F17
:1004120024F050D5124868743B12DC3A7A47909C1B
:100422006A1224C9742A12DC2E909C731224C97495
:100432002A12DC2EDAF912DC5712DE38020359AC2A
:1004420014AB157A0412536375A704900400E4F008
:10045200ECF0EBF08514C78515C67F08120467DF40
:10046200FB75A7002275B901E5BCF0E5BDF0E5BE5C
:10047200F0E5BFF005C6E5C6700205C722E5152402
:1004820008F515E43514F5142275A704900400E567
:100492006F4410F0E56EF0E56DF0740312BC3B7F23
:0404A20020E4F5F766
:1004A600C2B2C2B2E5F7F0DFF4D2B275A700227489
:1004B60020256D54E0F56DE4356EF56EE4356FF587
:1004C6006F2205117F287E00E51112D41780069051
:1004D6000402E070177F287E15900400E012D417FE
:1004E6007E2A900401E012D41712DD461248687481
:1004F6003A12DC7175A7009004007F23E0A312DC9A
:100506000DDFF912DC483099FD2202035912DF1C77
:100516007F0F90A6A31276F0121E1912DD46C214A2
:10052600C21512DE277510651000DFE53170F9E59A
:10053600106465700D855E14857A15E4F512F51361
:10054600800C78A8E51326F513E43512F5127F1E04
:100556007E19E51012D3BDC3E57A9515F517E55E4C
:100566009514F5167F287E0BAC16AB1712D2D11256
:10057600D35512DD4612DE38D510ADAB17E516FCA5
:1005860030E7031255F67A0A79001253DCA912A84D
:1005960013125515EBF510243840037510C8120ECA
:1005A6005D8510BC02035612DF1C909CFF7F017E06
:1005B60009127702909D087F0A7E091277027F133F
:1005C60012CA1B751700120E6CE5BC12068DE5BD2E
:1005D60012068DE5BE12068DE5BF12068D909D5959
:1005E6007F5F7E06127702121E9E12DD4675170089
:0605F60012066D10000862
:1005FC0010011510024880F20517E51724F7500377
:10060C0075170075100080E2E51764087015120E5E
:10061C006C75BC0175BD2375BE4575BF67124EE682
:10062C000205ADE51012069F12DD4612064D0510AF
:10063C00531007E51724FE400353100380AC02024D
:10064C00C6A9BCAABDABBEACBFE5171304F8E64007
:10065C00085407C42510C4800454702510F6027D7C
:10066C00A17800E875F009A42417FF7E3B7D20E8F3
:10067C00651770027D89ED12D50808B809E502DD11
:10068C0046F8C4120693E812069F7E030517E51779
:10069C0002D4F5540775F009A4909D112582F582BA
:1006AC0050020583E51775F009A42417FF7E0C0290
:1006BC007702C26812DE57753705909EE9121CFF4F
:1006CC009006D073020293027941027986027B1C58
:1006DC000206BE0206F4027A5E027AC402178B028C
:1006EC0006BE021771020C627F2E12168680C31290
:1006FC00DE57753706909FC6121CFF90070B7302CE
:10070C0002930217C802182A0218A30219700219C0
:10071C00A2021A19020750020749021A62021B07A9
:10072C0002072F7F64120E67E5BDA2E7120D31128E
:10073C000E67E5BD92E7F5BD124EE680B27F491219
:10074C00168680AB12090C122B6912DF1C121DF3DA
:10075C00E55804607790A0961207F912871E12DDF7
:10076C004610000810011310021C80F50559C3E552
:10077C0058955950D575590080D01559E55930E721
:10078C00C985585980C4E559B40F02802FB51F0292
:10079C00802A75F007A42408F51775162774B82558
:1007AC0059F987001207E712DD46100028100128BE
:1007BC0010020280F574B82559F9A700E53524FA22
:1007CC00508878C7A64812090312DF1C12DD4612A6
:1007DC00DE2A0206FB1880CC0880C9E875F005A457
:1007EC0085F01CF51BC000125C7CD000221287AF78
:1007FC00B4FF0122751000751FFF1287C6E5106447
:10080C000F6017120830401274B82510F8E675F016
:10081C0005A485F01CF51B125D0D0510C3E558955C
:10082C001050D7221211AEF8602E6404602AE8141E
:10083C00B51025F51F120E7BE5BC70060475F0147F
:10084C00800375F019A485F01CF51B125D0D7E223A
:10085C0090A644127735D322C322E558B4FF012267
:10086C00751000E510640F602EE51075F007A424D8
:10087C0009FF74B82510F8E61208ED75F00A84C06B
:10088C00F07E2012D45E7E28742C12D4D6D0E07E5A
:01089C002A31
:10089D0012D4C31208AD0510C3E558951050C322EC
:1008AD001211AEF8603964046035E8146510702FCC
:1008BD00120E7BE5BC1208EDF8C313923D7E1C129F
:1008CD00D4747E28742C12D4D6E4303D067405B849
:1008DD000001147E2A12D4C37E18742312D4D6229A
:1008ED00305D1275F036A42432FBE435F0FC125560
:1008FD0085125585EB221209151276D5DFFB2212D2
:10090D000915127EB1DFFB2275C70375C6F078B8E5
:10091D007F042275C70375C6F375B901E5BFB548E8
:10092D0031E55924F1402BE55975F00484A9F024E3
:10093D00F0F5C675B901C5F0A9BC600CA9BD146070
:10094D0007A9BE146002A9BFE975F005A4F985F0E9
:10095D00CC22120E7BA9BD75CC0022124EE612DE02
:10096D005775370390A1B3121CFF90097B730202D8
:10097D00C6020C7B02131F020C90020C9B0216E6A2
:10098D000213A6020D5C0213DA02142002173802BC
:10099D00138E021465124EE612DE5775370490A2BF
:1009AD0074121CFF9009B5730202C6020CAA020C48
:1009BD00B50209A5020CCB020CD60210230209A523
:1009CD00020CE5020CC0020CFF124EE612DE57754A
:1009DD00370B90A2C5121CFF9009E9730202C602E3
:0B09ED0010D10210D1020A6F020AAD07
:1009F800020A10020A330217CE02117602123E02D0
:100A080011E70212CF020D19120E67E5BF1470C16B
:100A18007F2E120E9E1F120E67E5BDA2E6120D3143
:100A2800120E67E5BD92E6F5BD80A37F37120E9ED4
:100A3800120E62A8BFE8120A6712DD4610000810FD
:100A4800010D10021280EE18B802EA780A80E60852
:100A5800B80BE2780380DE120E6288BF0209D67FE7
:100A6800367E2CE802D3A67F1C120E9E120E67A8B3
:100A7800BE120AA112DD4610000810010D10021462
:100A880080EF18B800EB780B80E708E824F450E111
:100A9800780180DD88BE0209D67F1B7E35E875F0B7
:100AA80005A402D3A07F25120E9E120E67A8BF12BE
:100AB8000ADF12DD4610000810010D10021480EF45
:100AC80018B800EB780980E708E824F650E17801C7
:100AD80080DD88BF0209D67F247E3BE802D4F51268
:100AE8000E5DE5BF75F03CA4ACF0FDE5BE75F00504
:100AF800A42DFDE5F03CFC120E67E5BF14603675C9
:100B0800F005A485BEF0A42DFFE5F03CFE7C007D39
:100B18003C12547CC005EF75F01884E5F07F2D7EFB
:100B28002412D3A07E30743A12D5087E35D0E01254
:070B3800D3A002DD467F2D72
:100B3F007E0590A666127702120E67E5BDA2E67FCC
:100B4F002D12161502DD46D25712DF1C121DF3129D
:100B5F000B640202937F177E02909E071277027F2B
:100B6F004C7E02909E1D127702AC5DAB5C7F577E70
:100B7F000412D34D120E8A85BC6285BD63E56124D4
:100B8F00F84044909E287F371276F0AE61AF607CBC
:100B9F00017D5E12547CC3741F9FFAAC63AB62EC91
:100BAF0033921750031255F6125363AB047C003087
:100BBF0017031255F674F52BFB74033CFC125339D3
:100BCF007F377E1512D2C5909E357F697E0F1277C3
:100BDF0002E560240FFBE43561FCA25C923BD25C22
:100BEF007E1E12D2D1A23B925C7E30742012D508A9
:100BFF007E36742012D508E5602562FBE56135630A
:100C0F00FC7F227E0412D34DE56245637016742E6D
:100C1F007E3A12D50812DD4610000D100115100294
:100C2F0026020B8C742080E81562E562B4FF0C1568
:100C3F006380080562E56270020563E53524F550AF
:100C4F0003753301020B8C120E8A8562BC8563BD5E
:100C5F00024EE67F637E00747212D504121E5C4052
:100C6F00087F631276E7124EED0206BE120E71E593
:100C7F00BCA2E77F0A120D34E5BC92E7F5BC02096E
:030C8F00687F1C5F
:100C9200A20D120D31920D80097F25A20E120D3187
:100CA200920E120D5002096B7F0AA20F120D3192A1
:100CB2000F802A7F13A208120D319208801F7F52E3
:100CC200A20C120D31920C80147F25A20B120D3151
:100CD200920B80097F2DA209120D319209120D503B
:100CE2000209A57F49120E67E5BDA2E3120D31127A
:100CF2000E67E5BD92E39266F5BD0209A27F5B1223
:100D02000E67E5BDA2E5120D31120E67E5BD92E553
:100D12009243F5BD0209A27F6D120E67E5BDA2E006
:100D2200120D31120E67E5BD92E0F5BD0209D61231
:100D32000D468F1F9217120E9EAF1F1F7E3912840F
:100D42000BA21722120E7685BC2B85BD2122120E14
:100D520076852BBC8521BD024EE6203714120E711A
:100D620085BE12120D89120E718512BE124EE680D8
:100D7200057F3F120D7B02096B7E0390A23F127723
:100D82000212DD4602DE2775A6FF12DF1C12B6062E
:100D9200740712DF088FF0740612DF08EF2512C302
:100DA20095F0A2E7923D4010FD24CD50027D32AC79
:100DB20005C3743F9DFD800FF404FD24C850027DDD
:100DC20037AC0574402DFD7F4012CA1B7E1212DE25
:0F0DD200610EBE1EF91F303D020F0FEF6D70ED69
:100DE100E536700A753606EC2513F5148C13120ED0
:100DF1000712DD4610000710010830020722151204
:100E01008002051280827F377E28742E12D5087FDA
:100E1100347E21740A303D010412D523E514FC24EB
:100E21009C50027C637F347E2DEC12CE477F437E43
:100E31001E12D2CD7E00E51212D4647F057E02908F
:100E4100A2481277027F6D7E0190A2531277357FFF
:100E5100747E0490A264127735021DF375C6F48086
:100E61003575C6F5803075C6F6802B75C6F78026B8
:100E710075C6F8802175C6F9801C75C6FA8017758C
:100E8100C6FB801275C6FC800D75C6FE800875C64E
:100E9100FF800375C6FD75C70375B9012274721F02
:100EA10012D5040F02DD467F0A120E9E7E2A1248D9
:100EB100F0120E7BA8BF120EDC10001210010510FB
:100EC100021580F508E824E750EC781880E818E866
:100ED10030E7E3780080DF88BF805F7F097E05907F
:100EE100A527B80C0390A5211277027E27E53D289E
:100EF100240C75F01884E5F012D3A07E33743B12F4
:100F0100D5087E35E53E12D3A002DD467F13120ED1
:100F11009E120D46120F3E10000810010510021717
:100F210080F2105C07205D0BD25C80E8105DE5D299
:0D0F31005D80E1D25C80DD852BBC020356A3
:100F3E00205C10205D1890A57A7F127E2312770216
:100F4E0002DD4690A58E205DF090A58180EB90A5E8
:100F5E008780E67F1C120E9E120E76A8BF120F9887
:100F6E0010000810011110021A80F2E824F250034A
:100F7E001880EA780D80E6E824E740030880DE78E2
:100F8E001980DAE8F5BFF54380A37F1B7E26E412B5
:100F9E00D4F5E82323B464087E26740112D4F5E454
:100FAE007E2E12D3A002DD467F25120E9E120E85D6
:100FBE00A8BCE8120FF112DD4610000810010D104A
:100FCE00021F80EEE824E050E9188006E824CF40A6
:100FDE00E108120E8588BC124EE6D21512D9BD80DC
:100FEE00D180157F247E3724E202D4117F2EA20AEF
:100FFE00120D31920A120D500203597F37120E67ED
:10100E00E5BDA2E4120D31120E67E5BD92E49267C2
:10101E00F5BD0203567F367E00747212D5040F7E24
:10102E0016743F12D4D6120E71A8BD12109C12DD8A
:10103E004610000810010510021080EFE8248750BA
:10104E0004240A800224E8F880E17F377E1674209B
:10105E0012D4D67E2C743F12D4D612109C12DD46BA
:10106E0010000810011410022080EF18B80904783F
:10107E007880E7B878E478E780E008B87904780AF1
:10108E0080D8B8E8D5787980D188BD0209A2E82445
:10109E0087923DE8500224917F367E30C313923BF7
:1010AE0012D4117E3CE4303B02740512D4EE7E1A4B
:1010BE0090A46D303D0390A4711277027F3C7E3A6E
:1010CE0002DE617F127E00747212D5040F7E2074D0
:1010DE003F12D4D6120E5D85BE1085BF1112115867
:1010EE0010000810011110021B80F21511E511B449
:1010FE00FFEB75111780E60511E51124E850DE753A
:10110E00110080D91211587F137E20742012D4D66C
:10111E007E31743F12D4D612DD4610000810011134
:10112E0010021B80DF1510E510B4FFD875100B8070
:10113E00D30510E51024F450CB75100080C6120EA6
:10114E005D8511BF8510BE0209D67F127E24E51182
:10115E0012D3A07E30743A12D5087E35E51075F0A4
:10116E0005A412D3A002DD467F49120E9E1211AEC7
:10117E00F81211B410000810010D10021280F218AE
:10118E00B8FF02780480EA08B80502780080E212FF
:10119E000E5D88BD124EE6B800030209D902123E5A
:1011AE00120E5DE5BD227F487E0590A48712770260
:1011BE00E8601CB4040A7E0590A47C127702800CB1
:1011CE0090A4931277027E38E812D4F502DD469091
:1011DE00A48E7E2912770280F31211AE601D640474
:0211EE00601986
:1011F0007F5B120E9E120D46121219120E7610000F
:101200000B10010810020C80EF0209D9105FE9D21F
:101210005F80E5852BBC0209D61211AE601F640405
:10122000601B7F5A7E0590A4871277027E2390A4CC
:1012300097305F0390A49E12770212DD46221211AE
:10124000AE70030209D97F527E11120E9E120E7BE0
:10125000A8BC12127E120E7B1000081001081002AA
:101260000880EF1880EC0880E9120E7B88BC124ED3
:10127000E6120E85E875F005A4F5BD0209D6121137
:10128000AE604BE875F03270040475F028A4ADF040
:10129000FC305D11ACF0FB7A8A125371EB30E7053C
:1012A0000CBC00010DAE05AF047C007D6412547CC3
:1012B000C005EF7F517E1A12D3BD7E2C742C12D53F
:1012C00008D0E07E2F12D3A01241B712DD46227F54
:1012D00064120E9E120E7BA8BD121300100008109F
:1012E000010F10021680F218E824CD50EC783280FD
:1012F000E808E824CD50E2780080DE88BD0209D6F7
:101300007F63E823C2E012CF7A75F06484C0F07E78
:101310002612D4F57E2C742C12D508D0E080A47F40
:1013200013120E9E120E71E5BCA2E7923DC2E7F8C1
:10133000E812135E12DD4610000810010D100212B3
:0313400080EE1824
:10134300B800EA783280E608B833E2780180DEE854
:10135300A23D92E7F5BC79A1F78079547F305C0117
:10136300237F127E2375F00A84C0F012D4117E2DE0
:10137300742C12D508D0E07E2F12D4EE0F7E359058
:10138300A594305C0390A5F00277357F64120E9E1E
:10139300120E7BE5BE7F637E2C128460F5BE79A2BC
:1013A300F780317F37120E9E120E76A8BC530003CE
:1013B3007F367E32E812D4F512DD461000081001A4
:1013C3000710020780E718180880E2E5BC54FC48C0
:1013D300F5BCF52B0209687F49120E9E120E85A8F3
:1013E300BE12141112DD4610000810011110021A6A
:1013F30080EFE8240AF8242450E778DB80E3E8242C
:10140300F6F8247F40DB788180D788BE80C6E8F475
:1014130024DC75F00A847F487E3B02D4F57F5212A8
:101423000E9E120E85A8BF12145812DD4610000836
:1014330010011110021A80EFE82408F8245750E72E
:1014430078A880E3E824F8F824A040DB786080D70C
:1014530088BF0213D7E8F424A923C47F517E3B023B
:10146300D4F5122C74754A00D210C211D214D2755D
:1014730075791475340012DF1C7F007E0290A2225E
:101483001277029041E07F087E2612D534E52B5473
:10149300030F7E3912D4F5121E0E12D19E128ED175
:1014A30012DD4610000810011A10022480C52075B1
:1014B30004057980BE1579E579B4FF05C2757579A0
:1014C3000180B02075EB1579E57970A7D27580A3FB
:1014D300C210C21402096B120E76E5BE7F097E3A72
:1014E30002D4F5120E7BA8BF120EDC120D46120FAA
:1014F3003EA8BF120F98120E85E5BC120FF17F2D87
:10150300A20A1216157F36A267121615120E5DE592
:10151300BC7F487E3202D417120D467F1BA20D12E8
:1015230016157F24A20E121615120E71E5BC1213A6
:101533005E7F09E5BCA2E7121615A8BF121724E5C2
:101543002B54037F367E3212D4F5120E7BE5BE7F19
:10155300637E2C12D4F5120E85A8BE121411A8BFF7
:10156300121458120E67A8BC021769120D467F09A0
:10157300A20F1216157F12A208121615120E67E596
:10158300BDA2E37F48121615E5BDA2E57F5A1216E8
:10159300157F51A20C1216157F24A20B1216157F6C
:1015A3002DA209121615120E71A8BD02109C120E5F
:1015B3005D85BE1085BF11121158120E67A8BE12A9
:1015C3000AA1A8BF120ADF120AE7120E76E5BE7F50
:1015D3003F7E3A12D4F5120E62A8BF120A67120EAA
:1015E3005DA8BD1211B4120E7BA8BC12127E120E9E
:0415F3007612121941
:1015F700120E7BA8BD121300120E67E5BDA2E07F95
:101607006C800B7F098040120D467F48A25E744EA6
:10161700400274597E3A02D508127DAD7F73127A63
:101627000B127DFC7F6C127A1A7F2D801A120E67BF
:10163700E5BDA2E77F63121615120E76E5BE7F0998
:101647007E3A12D4F57F4812166EB40104BF090121
:10165700E4F51075F005A47E1E909F972582F5820C
:1016670050020583027702120E67E5BD035403C2D9
:1016770034C25330E103D2342230E002D253221273
:101687000E9E1F12164E12DD46E5101000121001B5
:101697000610020280ED22045403B4030AE4800713
:1016A700145403B403011423C5BD54F925BDF5BD76
:1016B700124EE680CE1275D1EBF516F5147F6C123B
:1016C7007A1A1275B57F647E23E51612D474C3E5C2
:1016D700169514F5167F73127A0B7F2D02164E7F1F
:1016E7002E120E9E120E71A8BFE824FA400330375F
:1016F70002780312172412DD4610000810010D109E
:10170700021280E518B800E1780580DD08B806D92F
:10171700780180D5799DE8F7F5BF0209687F2D7EAE
:101727002C7420B80502742E12D5087E32E802D434
:0C173700F57F5B120E9E120E67A8BCE846
:1017430012176912DD4610000810010D10021280F5
:10175300EE18B800EA780380E608B804E27801805E
:10176300DE88BC0209687F5A7E2CE802D4F5D26871
:1017730075480A1248F0D214122B77127EE5123301
:10178300CFC26B12024A80F3D214751501127D6722
:1017930075B901E5BC20E71C127E9775A6FF127E82
:1017A300F1121E1912DD4612780B10000F500512AC
:1017B300793380E70515E515242050D10206BE12C2
:1017C30017D40202931217D40206FB1217D402098C
:1017D300D91217E0120E768548BE024EE6122B6927
:1017E300122B83125A3612DF1C90A03FD249128764
:1017F3004B128704121DC912DD4610001410010597
:1018030010021B80F50548E548640A7002F548801C
:10181300CF1548E54864FF700375480980C28548C1
:1018230049122B83E558221248F0122B6985484947
:10183300C250E558B40F02D250125A36803AD2271A
:1018430075480A122B77125A3612DF1C12866E90D5
:10185300A43E20290390A449121E8BC26A1233CFDF
:10186300106A0280E1C227127D3F854948121C3667
:10187300122B83D229125A3612DF1C909F521287E1
:101883004920500E121E7512DD461000101001AED5
:1018930080F8121E1912DD4610000280FB0206FBBF
:1018A300122B69E55830E7137F1B90A4287E05129D
:1018B300770212DD4612DE2A0206FB122B83125A2E
:0A18C3003685594912DF1C121E037E
:1018CD0090A44912874912870E12DD4610000810A8
:1018DD00010A10020C80F512193B80DB12194880A9
:1018ED00D612DF1C121E0390A04E12874912870ECE
:1018FD0012871212DD4610000810010A10020C802A
:10190D00F512195480DB12196280D6121BFC122BB2
:10191D0083125A3612DF1C90A38F128749121E4173
:10192D0012DD4610000510028880F80206FB0559ED
:10193D00C3E55895595003755900221559E5596459
:10194D00FF7003855859220549D3E5491495584030
:10195D0003754900221549E54964FF70058558490D
:10196D00054922122B69E55830E7057F240218AD91
:10197D00122B83125A3612DF1C90A059128749126E
:10198D001E8012DD4610000A10010280F8121CA5FF
:10199D0080DE0206FB122B69E55830E7057F2D022C
:1019AD0018ADC26B7559FF125A3612DF1C121DF39A
:1019BD00E55930E703121E0E90A06B12874912876E
:1019CD001E12DD46E55820E7061000081001111023
:1019DD00021B80F00559C3955950CF7559FF80CA28
:1019ED001559E55964FE70C285585980BDE55920D9
:1019FD00E711D26B75A700758307C4F582E0B2E7D6
:101A0D00F080A7306B03121C530206FB122B69E505
:101A1D005830E7057F360218AD122B83125A361255
:101A2D00DF1C90A076128749121E5C4009121C9A89
:091A3D00121CCF121A460206FB2E
:101A4600120E7BE5BD75F00584F5BCF5BDF5BEF55A
:101A5600BF120915124EE605C6DFF922122B69E5FB
:101A66005820E7087F5190A0800218B012DF1C9022
:101A7600A454128749121E1912DD4612484FD2ACE1
:101A860010001FE55830E7F8306DF5121B9C7E20DC
:101A96007F00501390A4A512773512DD4612DE2A78
:101AA60080CAC2AC0206FB1B8B13909F6F12773560
:101AB60012DD46C26B7B007514B8121C8F127E664F
:101AC600127E185025A814E824384004A6010514EF
:101AD6000BC3E5139B50E678B8121CD1306B03128A
:101AE6007BBD122B83125A368082127DADE51660BD
:101AF600E6D26B127EC3C003127D7ED003A9158089
:101B0600C4122B69E55830E7057F5A0218AD122B2F
:101B160083125A3612DF1C90A08B128749121E368A
:101B260012DD4610003510010280F8754605121BBD
:101B36006450157F007E357407954612D47412DD05
:101B46004612DE2AD546E7D390A45F500390A4A59B
:101B560012874912DD4612DE2A80B30206FB1248BE
:101B66004F12DC60745212DC71745412DC2EE5588C
:101B76000475590012DC4F1277BA4016127D3F12D7
:101B86007E9712780B400B0559C3E558955950ECD2
:101B9600C322C2ACD32212484FD2AC12DBB9204CBE
:0D1BA600F1B440F712DBBEB4400312DBBE09
:101BB300B452E2F53812DBBEB454DA12DBBEFA607B
:101BC300D424EF40D012DBBEE53870C912DBBE125D
:101BD300DBBE12779F7B007E031278965010205055
:101BE300B412DBBE204C03B440F7DEED80A7127EB7
:101BF300760B12779FDAE0C322121CE0E55924C862
:101C0300F88602E54924C8F9986013146010500F50
:101C130018E608F618E86970F7A702121CCF22E548
:101C230059640F60F91908E618F608E86970F7A710
:101C33000280E8121CE078C8C250E6B4FF028007B5
:101C430008B8D8F6D25022B8D702D250A615807C55
:101C530078B8121CE2E4F9F5A7758307E9C4F582A5
:101C6300E030E70AE924B8F82438400276FF09C3D4
:101C7300E5589950E7121C9A78B879C8E6B4FF0280
:101C83008002F70908E8243850F2804079B877FFDA
:101C930009E9243850F82279C877FF09E924285044
:101CA300F822121CE0C23D78D7B6FF04A900D23D4A
:101CB30018B8C7F5203D0279D81978C8B6FF0122B4
:051CC300C3E899500781
:101CC800C6C7C6081980F478C8121CF1127ED31250
:101CD8007ED3127ED3027ED378C8121CF1127EB155
:101CE800127EB1127EB1027EB175C703E54875F068
:101CF80004A42480F5C62212DF1CC23C1276F4E547
:101D080037605314604D14604514603D14603514F9
:101D1800602D14602514600E14600B14600D14609F
:101D28001414600C803012160E802B1216BC8026FC
:101D38001215B1802112160A801C1216348017124F
:101D48001620801212156E800D12151B80081214B1
:101D5800E680031214DA12DD4612DE2E121DF3128B
:101D6800B9C7A81F08E814C23BB51D02D23B75F0DD
:101D780007203C0375F009A4FF7E00303C0C74205A
:101D8800303B02743E12D4D6800A740B303B027486
:101D98000A12D4EED8CF12DD46E51D100008100156
:101DA8001010021880B9651F7003751DFF051D808E
:101DB800AE7005851F1D80A7151D80A375F003A4AF
:101DC800227F7B7E0090A3A7127735E54824F64052
:101DD800087E0A90A40B12773522127A377E057492
:101DE8005B12D4D27E1D745C02D4D2121DE27E3402
:101DF80090A3B8027735127A378003121DE27E313C
:0E1E080090A3BC027735121DE27E3190A4B08B
:101E1600027735127A377E008005127A377E2D904A
:101E2600A4B0027735121E367E31909FAB0277350D
:101E3600121E197E1A909FB0027735121E1980C0A5
:101E4600121E197E18909F5C027735121E197E1A93
:101E560090A4B5027735121E197E1A90A4BA12778D
:101E66003512DD46D3100006C310010280F6221299
:101E76001E197E1A90A049027735121E197E1890F7
:101E8600A0640277357F007E2012773502DD461288
:101E96007A3790A4C0027733127A3790A4D10277AA
:101EA6003312BE89120E94E5BDF55EF56CE5BCF500
:101EB6005FF56B756A007561FF75A70490070012E0
:101EC600BE33B4FC23E582C313F561E56CF0E56B24
:101ED600F0E582600F12BDAAE56C655E70E1E56B08
:101EE600655F70DB75A700223024EA0460E7240FE3
:101EF60040D380E1E560758307C333F582E0A3F53F
:101F06006CE0F56B756A0022D2248002C224D214DA
:101F1600C21F121EA7756000E561B4FF1612DF1C12
:101F2600909E387F0A7E0512773512DD4612DE272F
:101F3600020293C210C21112DF1C121DF3301F0AD7
:101F46007F07909E4612773380647F007E01C3E54B
:101F56006012D4747E0E742812D4D2856048740739
:101F6600F51FFF7E00743E12D4D6E548121EFC1201
:021F7600C82A77
:101F78001224D80548C3E5619548FD401CE51F2497
:101F880007F51F24C850E17F387E01ED0412D47490
:101F98007E0E742912D4D2800DE51F2407FF7E011E
:101FA80090A4AF127735201F0312251B12DD4610AF
:101FB800001910012C10020280F5120236301F3D64
:101FC800020282101F02D21F021F39E56160F4E588
:101FD8006065617005201FF080E9201FE6056080BC
:101FE800E7E56160DEE56065617005201FD5800961
:101FF800201FD5E560700280CA156080CB121EA72D
:10200800121EFA12C82A12260F756A1012BE1C1266
:1020180026C6909E50D23C1276F4121D6490202958
:1020280073021F3902330F022049022035121E5C49
:1020380040CB121EFA12BE33C2E2FF12BC59021F75
:102048001212DF1C7F6490A6891276F07F7990A621
:10205800961276F012DD4675160010000A10010976
:1020680010020280F505160516C253121EFA12C890
:102078002A75370A909E6C121CFF902086730220E6
:10208800050220AD02227C0222810220710220B4C6
:102098000220B90220710220F70220FB0220FF0271
:1020A800210602210A7F0A12168680BD124868801E
:1020B8000312485D780A1221D9740912DC2C122205
:1020C8001812DC4812225312BE1C12BE4412BD6BF9
:1020D80012BF5B122362D5150C75150A12226612FF
:0C20E800248912DC48100204E57F70DB44
:1020F400022005780A800678048002780112486874
:102104008009780A8002780112485D1221D9740985
:1021140012DC21122218E54812DC0DE516540344A2
:102124003012DC2E742A12DC2E12DC2E12DC481241
:10213400225312BE1C12BE4412BD6B12BF5B12238B
:1021440062D51548854815122266E51C12DC0DE59A
:102154001B12DC0DE51B2548F51BE4351CF51CE4BE
:10216400A27792E7A27492E0A27392E112DC0DAD21
:1021740075AC74AB73E57DC412219AAD78AC77ABC2
:1021840076E57D12219A1224A712DC48100204E598
:102194007F709F022005540F2375F00584F8C3EB6C
:1021A40033FBEC33FCED33FDC3EB33FBEC33FCEDE1
:1021B40033FD20E713EB28FBE43CFCE43D12DC0D8B
:1021C400EC12DC0DEB02DC0DC3EB98FBEC9400FC91
:1021D400ED940080E88848121E20E4F54AF549751C
:1021E4006A2075150112BE1C12BD6BD5150E8548EB
:1021F40015E5492401F549E4354AF54AE57F70E5DA
:10220400744012DC71747812DC2E746312DC2E7448
:0F2214002102DC21122464E56012DC0D121EFA97
:1022230012C82AE53A12DC21E53B12DC21E53C1217
:10223300DC21E53D12DC21E53E12DC21E53F12DC29
:1022430021740112DC0DE54A12DC0DE54902DC0DB7
:10225300121EFA756A20E4F51CF51BF514F51375C7
:10226300150122753800E51412DC0DE51312DC0D9F
:102273000513E513700205142212486880031248FF
:1022830052121E201223BC12DE32756A207515010C
:1022930075A6FF754A0112BDC412BD6B12BF5B1256
:1022A3002362D5150975151E12238612DE3C1224EE
:1022B30089E57912DC0DE412DC0DE5711223471276
:1022C300DC0DE57012DC0DE57B24ACFFE55F340922
:1022D30012DC13EF12DC0DE51520E033857D56E4A7
:1022E30012DC0DE52EC412DC1312DC5712DE3C1097
:1022F300021A30559B744012DC2E744512DC2E7486
:102303004F12DC2E744612DC2E12DC57022005E538
:1023130056122321C4FAE57D1223212A80C2FBC46D
:1023230012232E2323CB12232E2B22540FFC24F60D
:1023330050027C0090233DEC932200000101010236
:1023430002030303FA2440400A24804003EA3322B1
:10235300D2E72274FF2220E703C3132224C022E51D
:102363003F701F7F7B7E0078AEE612D45EEE2404BE
:01237300FE6B
:10237400743A12D4D6EE2404FEE53E12D45812DD8B
:102384004622C015C016D21212A6E1C212D016D02F
:102394001578AEE612DC21E53E12DC21E53F12DCC5
:1023A40021E54512DC0DE55212DC0D740A12DC0D38
:1023B40074C012DC0D02DC57744012DC2E7454120B
:1023C400DC71744E12DC2E743012DC2EE5165403CC
:1023D400443012DC2E122464742112DC21E53D12F7
:1023E400DC21E56012DC0D121EFA12C82A78ABE675
:1023F4000812DC21E60812DC21E60812DC21E612D0
:10240400DC21E53E12DC211229EFE51212DC21E584
:102414001112DC21740112DC0D90A4E21224C9759E
:102424006A1012BE1C057F057F787F12DC06787B5C
:1024340012DC06787D12DC06787712DC06E4FEFFF7
:10244400780712DC0612DC06E57412DC0DE5751261
:10245400DC0DE412DC0DE412DC0D12DC0602DC57A8
:1024640075C70375C6FF75B901C217751D0085BC14
:102474001C85BD1B85BE1A85BF191252E9EE12DCFC
:102484000DEF02DC0DE57512DC0DE57412DC0DE5D3
:102494007312DC0DE57812DC0DE57712DC0DE576C0
:1024A40012DC0DE51664016011E55E12DC0DE57ABF
:1024B40012DC0DE516640260012278BCE612DC0D24
:0A24C40008E602DC0D75A700E493A2
:1024CE00700122A312DC2E1A80F4AF1F7E0478ADA9
:1024DE00E612D4587E0C742C12D4D67E0E18E61248
:1024EE00D4587E1A78AEE612D4587E22743B12D49B
:1024FE00D67E24E53E12D4587E2FE54012D45E7E61
:10250E0037743B12D4D60E0EE54102D45875320004
:10251E00121EFA12C82A857946787A796412C8434F
:10252E0074641256DE8E4712260F756A20D23D1243
:10253E00BE1C12BE44122646303D09307406C23D02
:10254E008E1E8F1FE57F602BE54C24FFF54CE54D6D
:10255E0034FFF54D454C600512BD8080D2751D3C93
:10256E0012BE1C12BE4412BD6B122646E57F6003DE
:10257E00D51DED1226A79026BF12D534203D0DAEE7
:10258E001EAF1F1226A79026B812D534E546FD7051
:10259E000B90A618305D1190A614800C047010904C
:1025AE00A614305D0390A6107F381241B2804BE422
:1025BE00FFFC7E05305D047E027FB312546FAC06C5
:1025CE00AB071253397F38C23DE51C6007D23D7E02
:1025DE002C12D4C3E51B203D026007D23D7E301283
:1025EE00D4C3E51A203D026007D23D7E3412D4C317
:1025FE00E5197E3812D4C31241B7E53224C850FA19
:10260E0022E54075F03CA42541FFF54CE435F0FE83
:10261E00F54D7C007D1012547C0F8F4BAF4CAE4DA0
:10262E007C007D3C12534F7C00AD4B12547CEE4F20
:10263E0070010F8F4C8E4D2278647973C2D11226A1
:10264E005DFF78677976D2D112265DFE02DE61C318
:10265E00E796FB0809E796FC0809E796FDA2E792C4
:10266E001750031255FE75135A30D10E751320B242
:10267E0017AA47125383AB04AC05E546600B046002
:10268E000BAA4612539AEB03FBEB03FBEB543FFBF7
:10269E00E5132B2017029B9B22EE141430E701E466
:1026AE00FEEF141430E701E4FF2205057088A888B8
:1026BE007005052020F8202075320012DF1C7E1ECA
:1026CE007F1C12DE61DFFB12DE617E1E7F1C12DEBE
:1026DE0061DEFB7E1D7F1D12DE61DEFB7F007E2133
:1026EE0078ADE612D4587E29742E12D4D67E2D18CB
:1026FE00E612D4587E35742E12D4D67E3918E612D0
:10270E00D4587F077E21745412D4D67E25744F126E
:10271E00D4D67E2D78AEE612D4587E35743A12D4C5
:10272E00D67E39E53E12D45878AE1229EF7F0E7E52
:08273E0021744C12D4D67E2553
:10274600744112D4D67E2DE51212D4587E35743AD1
:1027560012D4D67E39E51112D4587F157E257444DD
:1027660012D4D67E2DE54012D45E7E35743A12D44C
:10277600D67E39E54112D4587F217E0190A5E31219
:1027860077357E0EAC77AB7612D30A7E2B85795FD2
:1027960085787B12D8B17F287E0190A5E712773520
:1027A600751D2B751E10E5741229A37E25742F1234
:1027B600D4D6751D2D751E2BE5751229A37F367E81
:1027C6000290A5D3127735E5721228501228E81226
:1027D6001EFA756A209004E6E56CF09004E7E56B56
:1027E600F0AE4DAF4C7C007D4012547CBF00010F13
:1027F6000FAC07AD07E4FED23D12BE1C12BE44125A
:102806002891E57F602CE54C24FFF54CE54D34FF1F
:10281600F54D454C600512BD8080DE751D3C0E12DF
:10282600BE1C12BE44122896E57F600612BD6BD50B
:102836001DED1228667F7812CA2D7F767E007430D1
:1028460012D4D6E53224C850FA227E2112CF7A124B
:10285600D4747E2F90A5EB305D0390A5F0027735FA
:102866009004E6E0FD9004E7E0FCC3E56A9420FBF3
:10287600E56B9CFCE56C9DFD50032410FD12556E26
:0D2886009004E8EEF09004E9EFF022DD038D
:10289300AD040E7F78E55E20E72AE57A8549F0A44A
:1028A300A9F0E57A854AF0A429F9E435F0FAE55E62
:1028B3008549F0A429E435F02AFAE55E854AF0A4B7
:1028C3002ACF9FFF12DE61103D18C3EF9B50131BED
:1028D300EF6B600E8F018B0712DE611FEF6970F8DB
:1028E300AF01AB072290A598305C0390A5B1754A60
:1028F30040754900AF76E577FE20E76B7005EF245E
:10290300105064EF24A8EE34FD401190A59D305C77
:102913000390A5B5754A1975499A8075EF2450EE51
:1029230034FB401190A5A2305C0390A5BA754A0C04
:102933007549CD805CEF24A0EE34F6401190A5A537
:10294300305C0390A5BF754A067549668043EF2442
:10295300F0EE34F1401390A5A8305C0390A5C47544
:102963004A04754944802A8028EF2490EE34E840D5
:102973001190A5AB305C0390A5C9754A0275498FC8
:10298300800F90A5AE305C0390A5CE754A017549C2
:102993009A7F401277337F4612CA2D7F5F02CA2D7A
:1029A300AE1E75F064305C0375F03284C0F0F870CD
:1029B30004EE2404FEE51D12D4D6EE2404FEE860E2
:0129C300070C
:1029C40012D4C3EE2404FED0E075F00A305C037523
:1029D400F00584A8F012D4C3EE2404FE742C12D49F
:1029E400D60E0EE8305C012302D4C3E53E2541F542
:1029F4001124C45003F511D3E63540F51224E850F0
:102A040002F5122212B9C1C21012DF1C7F057E0921
:102A1400909C6A1277027F137E08902A3C12D53468
:102A24007F2B7E01902AA412D53420370A7F277E7B
:102A340027902B1612D53422113007FE1FE001E136
:102A440001F80F00061B00F80C00180E007C1000A3
:102A54007006003C2000E006003E4001E004001E39
:102A64008003C004001F0003C004000F000780009F
:102A7400000F800780000017800F00000027C00FA0
:102A840000000043C00F00100083E00F002003018A
:102A9400F00700C00F01F80383007F87FE01FC00EC
:102AA4000E3E1800000300000000180000030000A0
:102AB40000003800000000000000300000000000AA
:102AC4000000FC761F0E1C6030ECFCBC3F172DF0A0
:102AD400F978613866264F619A706070C60E1EE3FD
:102AE40030E06060C60C1CC360C0E0618C0C18C789
:102AF400C0C0C0E18C1C39C611C0C4C19C993196B8
:102B04003180C8C1FF1E31E7E180F0C0EE1C31C343
:102B1400818006163091882892884924904927900C
:102B24009248A0E3C8BCC2AFD2C075C0107581D8AA
:102B340074FE122B42E4F5F9F5FBC2B480F7D2A679
:102B4400C2A512B9A612DE2E02B9C775C703E5489D
:102B540075F004A42480F5C6C23C75B901E5BC0433
:102B64007002D23C22120E76E5BEF54824F65003DC
:102B7400754800753400753704C228D229D22A75E5
:102B8400C703E54824E75003754800E54875F00499
:102B9400A42480F5C6751607751700C23C122BC411
:102BA400122BC4122BC4122BC485175815587559EF
:102BB40000E548B40A09E5586005F46002055922A5
:102BC400203C1D75B90105C6AABCABBDACBEADBFEA
:102BD400EA122BE5EB122BE5EC122BE5ED122BE5BB
:102BE40022203C07F515B4FF03D23C22C0C7C0C65F
:062BF400127D6775A704C5
:102BFA00851683E517C4F8F58275B90105C6E5BCE3
:102C0A00F0C582F82406F92403C582E5BDF0E5BEC5
:102C1A00F0E5BFF075B90105C6E5BCF0E5BDF0E524
:102C2A00BFF08516838982E4F075B90105C685BCB3
:102C3A001385BD14E4F0F08882E5BEF0E5BFF075B7
:102C4A00B901E5BCF0E5BDF0E5BEF0E5BFF075837E
:102C5A0006E51723541E24B0F582E513F0E514F0B7
:102C6A0075A700D0C6D0C705172212BB8978BEA6A1
:102C7A004808E4F6F55908761808F6D23608760AAE
:102C8A0008F6060876BEC254C25512BE9E122B77AB
:102C9A00C229C22AC207C227C268120E67E5BDA2AC
:102CAA00E59243C24AE4F52EF534F536F52F78B6A7
:102CBA00F678B5F678A9F6789EF678B8A65E08A6EC
:102CCA007A12D273C26BC233C238C240C223C22242
:102CDA00122CF475460278C5A646C23AD221C21908
:102CEA00C226E4F542F541F54022E45407205E0984
:102CFA00B4040040027403801B120E6CC313A9BCF7
:102D0A00600C14A9BD600714A9BE6002A9BFE940FE
:102D1A0001C45407F53722122B69125A3612090CCC
:102D2A0012DF1C121E41E55804700A7F327E05909C
:102D3A00A42812770290A68012874B1208667F7227
:102D4A0090A6751276F012DD461000051002048076
:102D5A00F8D322C3220200F7120E67E5BD20E70569
:102D6A00122D2140F0754E50122C7412852C754488
:102D7A00031248ED12AF06D54403022B2A201EF196
:102D8A00789F7680754A0012BCBAD210C211C2135B
:102D9A00C21212483F75A60C12D9BD12C4A8E5A6E4
:102DAA0024FA400612488D75A60C20250CE590548D
:102DBA00057009E53524E25003022E54E532241841
:102DCA00400D75F00C84E5F070D41233D280CFD266
:102DDA001ED2AC306DC87532F012DBC3B4E0BF123C
:102DEA004935E53124F39205201203123264122E7A
:102DFA001AC014128E17D014200A03122F3D123350
:102E0A00D212A6B01233D212852F1233D2022D9CBF
:102E1A0030122EE54024F0401C7A0AC3E53F954B58
:102E2A006013401E24E2400D305405C254757F01E0
:102E3A0012BCE0DAE679BCE7D2E7F57F09877EC201
:102E4A007722F40424E250ED80DE12DF1C7F2A7E12
:0C2E5A000E90A4E612770275A6FFC210CD
:102E66001012137F367E08909F8D12770212DD4670
:102E760012DE270200F7D22112491112BCEA7F1E88
:102E86007E0B90A40112770212DD46122EA77F3E1A
:102E96007E0790A12312770212DD4612DE21022B55
:102EA6002AD215D21412BE75120D4675B90575B91A
:102EB6000212BE7FD25512BDA47F0012BC5912BEAB
:102EC6007FE56A600512BD6B80F7857A62120E9403
:102ED60085BEBC85BFBD856BBE856CBF75B90575E6
:102EE600B90285BD6C85BC6B756A2012BE75123041
:102EF600DE12BE7F756A0012BE1CE57064FE703479
:102F06007570FC854077854178851F797818797AC0
:102F160012C84312BD1912DE3C12BE7F756A10122A
:102F2600BE1C7F087810797212C84585627C855E62
:102F36007D12BD19C2152212486812308A745212C7
:102F4600DC2E744D12DC2E744312DC2E12309912D4
:102F5600DC697441207402745612DC2E122FE612BC
:102F6600303012DC69E53C12DC21E53B12DC21E560
:102F76003A12DC2112306612DC69744512DC2E121C
:102F860030CF12308A744712DC2E744712DC2E744E
:102F96004112DC2E123099122FE612DC69E43074ED
:102FA600010412DC2C12DC699004C3E012DC21124D
:102FB600DC699004E4E075F00A84AFF012DC2112BB
:102FC600DC6DEF12DC2CAC5EAB7A1230ABAC5DABD9
:102FD6005C1230AB12DC6912DC691230CF02483F5A
:092FE6007875C23D122FF17878D4
:102FEF00D23D12DC69128211303D05E51E12DC2C38
:102FFF00E51D12DC2C123073E51812DC2CE57D2058
:10300F003D01C4540F12DC2C12DC69303D097445AC
:10301F0030170274578007744E301702745302DC56
:10302F002E207408123066123066802775A7049020
:10303F0004BFE0FCE0FB7A1B125371783212551378
:10304F001253391230709004C1E0FCE0FB12533977
:10305F0012307075A7002212DC69E4F51AF5198099
:10306F000D12DC69E51C12DC2CE51B12DC2CE51AB9
:10307F0012DC2C12DC6DE51902DC2C742412DC2E10
:10308F00744712DC71745002DC2E12DC69E53D12BC
:10309F00DC21E53E12DC21E53F02DC2112826D12BC
:1030AF00DC69E51D12DC2E781CE612DC2C18B81733
:1030BF00F812DC6DE412DC2C12DC69744D02DC2E8C
:1030CF00C038742A12DC2ED03812DC4802DE3C786D
:1030DF00107F0EE4F608DFFCF564F565F567F5681B
:1030EF007515FC751AC0751DC075664075694075FC
:1030FF004A0112BDC430550302319412BD6BE57104
:10310F00B510004002F510E4F511E512207502E547
:10311F0013C395795006207545857913D3E57A95B4
:10312F0014E5156480FFE55E64809F400C857A147A
:0E313F00855E15857B16855F173074B3C2D18F
:10314D007864797312317278677976123172D2D1CF
:10315D0078187973123172781B79761231728091E9
:10316D0085791280B9D3E7960809E7960809E664D0
:10317D0080FFE764809F20D101B3400AE7F618195C
:10318D00E7F61819E7F622E51AB4C00E7873791828
:10319D0012C8437873796412C84378187964C2D120
:1031AD0012320574181256DE8E47AE1EAF1F781BF5
:1031BD007967D2D1123205C3E51F9FE51E9E5004DB
:1031CD008E1E8F1F7EFF7FFFAC1EAD1F12547C7AAB
:1031DD0004EF8AF0A4E5F0CE8AF0A42EFEE435F0DB
:1031ED00BEFF011E60051460057EFF8E1F22EE7E60
:1031FD000020E7F77EFE80F3C3E697FB0809E6970C
:10320D00FC0809E697FD1818191930E7031255FE49
:10321D00C3EB33FBEC33FCED33FDEB33EC33FBED68
:10322D0033FC30D105AA4712539A0BBB00010C7524
:05323D001E03751FFFD8
:10324200EC24FC40048C1E8B1FE627FB0809E637A2
:10325200FC0809E637A2E713F618EC13F618EB138D
:10326200F62210131978B5E624FA401AE57124F60D
:103272004008E57924F6400280360606803212DEE6
:1032820038E59030E2DF753612D22EE4F534F55A85
:1032920012BED01232B5C219C257122CF412914684
:1032A200129173D212853F4B754C00205E02D228D8
:1032B200022CECD214123304E6F008DFFB857A62AA
:1032C2001232FA7570FE783A797112C84312BD193A
:1032D2001232FA85627A855E7B120E8A85BC7E8501
:1032E200BD7F7570C012BD19123304E0F608DFFB12
:1032F20075A700D254C2142274FF7870F608B88001
:10330200FB2275A7049004F078707F1022121EFA37
:10331200122C7412DF1C12DD46C258C259754A01C2
:10332200753901756A2012BDC41256DC8E47C2106F
:10333200D211D214D21212BED0129146129173122D
:10334200D9BD75A6FF753609753200E59020E206F3
:10335200E5352405400CE5905405701FE53524E25F
:103362005019C211C21212DF1C12DD46E4F535F506
:083372002F7E0612DE34C202B8
:10337A00022005C221E54AB40202D22112BDC412BA
:10338A00A6B030260F125A9812852F753606E536E2
:10339A0070FCC22612852C1233D2E54A20E021B4F1
:1033AA000209753900E53670F9808CE53960FAFD55
:1033BA0024E24002053912BDC42026C9DDF880E99D
:1033CA0075390080E475370410003A1001161002AE
:1033DA0016E52F5407600312B9BB20783D20790AFD
:1033EA00207A1F220235C802351CE53760091460AD
:1033FA00091460090236740235E7023645C27902B9
:10340A00369102354FE53724FC500FE537640760E3
:10341A000302370C0236D00234E62011FAE5902076
:10342A00E2028056753400201203D2132278A9E6EC
:10343A007017C226767DE5377005106B02D26BD203
:10344A0077753614D22E02BEC5E537604314604044
:10345A00B40227200B24E6249B401F2414501C127C
:10346A00914690A3D37F207E0812770212DD46751B
:10347A003608D22E78A9E624ECF622241940FB2439
:10348A001450F712914612917390A3DC7F2980D7CA
:10349A002028E7E54824F640E1E5580460DC7F5D32
:1034AA007E10E6249B40D324145015C2330559C319
:1034BA00E55895595005855859D22690A3C180A937
:0434CA00241940B6CB
:1034CE00241450B2E55960021559102606E55960CC
:1034DE0002155990A3CA808D10780122753900E526
:1034EE003424384007754A0175340022700AE54AC3
:1034FE0030E0F2754A0280F0146008754A061291A7
:10350E00738006754A0412914675390180DA3029A6
:10351E0009C229D22A7559008005302A1BD22912D8
:10352E0086FA1286C8E53524AF400475340022753C
:10353E003700C229C22A80F3206841302703D26A9D
:10354E0022D2221238A812DD46107A0122E5342446
:10355E00384007122CF475340022700FAA37122C43
:10356E00F46A70F27401122CF580EB04122CF5241F
:10357E00FC50E3E537B40706D22880DA8036C2283D
:10358E00E53724FC2324BEF879C4E7F9A74809A738
:10359E005979C4E8F78648088607E537B4050575F6
:1035AE004818D236122B838F59E53764067002D233
:1035BE000702356412388402382EE537601B14601A
:1035CE007614600F146009E53724F9400902378636
:1035DE000236740236BF023753D223124096107948
:1035EE000122E534243840077546017534002278EF
:1035FE00D87020304A0BC24AE624F85004B24380F9
:03360E000AD24A93
:103611007614E54624FE40DDE54660D9154680D89E
:10362100B600D5B40500500C04F54624FA50C9750E
:10363100460580C424F95005127B5B80BB100FB88E
:10364100D20F80B4D223E53464C8600312409610CF
:10365100790122E534243750097011105B32D25BB5
:10366100802E100802D2081240968024100C21D21C
:103671000C801DD22312409610790122D24BE534E1
:1036810024374010C258C259201105D22E75360771
:103691007534002224FD401524037006D258C25906
:1036A10080EEC258D2591460E7D25880E3120E71ED
:1036B100E5BCB2E7F5BC79A1F7124EE680D278B845
:1036C100A65E08A67A2011C8753605D22E80C130B3
:1036D100122B128734055BE55B75F00B84E5F0F581
:1036E1005BE55A24F64009E55A955B5003755B008A
:1036F10012873812DD46E5346003D534D2753400C3
:1037010022D229D22A75480A0237F4C2401007F1A1
:103711003029030237F41286F612870A102A1BC2D7
:10372100330559C3E558955920E7025008755900EA
:10373100E548B41816E558B4FF0375590012871E01
:1037410012DD46E5346003D534C122D22A1286FA4D
:1037510080EE301223128734155BE55B30E70C7580
:023761005B0A01
:10376300E55A24F64003855A5B12873812DD46E595
:10377300346003D534DA75340022D229D22A75484D
:1037830017804CC2401007F22029441286F6128794
:103793000A102A22C2331559E55930E71C855859B6
:1037A300E558B4FF03755900E548B41802800AD2FE
:1037B3002A1286FA800E855859E558B4FF037559C5
:1037C3000012871E12DD46E5346003D534B522208E
:1037D300106220115F7F180548E54864187008F5EA
:1037E3004830270375480A122B4F303C2DDFE88001
:1037F3002620105A2011577F181548E54830E70551
:10380300754817800A640970063027037548171234
:103813002B4F303C05DFE275480A122B83125A36D0
:10382300E532244C50051286C8800312866E753427
:103833000002DD4612386B7F15E5486B70048A4839
:1038430080020548122B4F303CD0DFED80CC12387C
:103853006B7F15E5486A70048B4880021548122B6C
:103863004F303CB6DFED80B27A007B09E537B40414
:1038730001227A0A7B17B40601227418FAFBF54871
:103883002275A704758307E559C4F582E0E0F57353
:10389300E0F574E0F575E0F576E0F577E0F5787539
:1038A300A700025A36E59020E23EE534243750382B
:0638B3001238EC1238C9C6
:1038B900205E4F7F2C909D23123933909D2C806A76
:1038C900E534243775F009A42435FF205E0624BEAB
:1038D90050027F3EEF249B50027F627E3274891230
:1038E900D5082275A7049000317E087F3AE4F0DFFD
:1038F900FDE5822446F582E43583F583DEED75A77F
:1039090000227F2C120E6CE5BD12391CE5BE12395E
:103919001CE5BFF8C4123922E8540775F009A490D0
:103929009D112582F58250020583EF2409FF027655
:01393900F09D
:108529000285E312DF1CE53724FC40F4B4FE142075
:10853900110EE590F45407600122E532247450EFDE
:10854900028E2312DF1C12D6AB12D73D12CF88122E
:10855900D2C912D1127E197F3612D06612DC761278
:10856900D07CC206E53760051460338053C23A12E5
:1085790086871241591242EE1245D41264F41265EB
:108589001C123E04E54864186009E54824F65003C6
:108599001246BF128DB912CE0D1241F48014D23A8F
:1085A9001286AD1239421241C312C993128DB91202
:1085B900CDCE125D7712D784125848125B478012CC
:1085C90012869312C8D012D85412C962128DB912E8
:1085D900CDE530101112D01A800C12DF1CE53724BA
:1085E900F9401E1286703022091238A8E53470024B
:1085F900C222302309124096E5347002C22302DDFB
:1086090046121DF375170012DA677F1212CA1B3062
:10861900124A75100075A704758306125AF1E51000
:1086290075F009A42415FFF5177E00E512602F7572
:10863900F06484E5F00F12D4581F7E0EE51112CFB5
:10864900D0751623125CAD0510C3E55A9510400686
:10865900E51024F550BF3012031287388088745D05
:1086690012D50880D5C249302905121DC9800312C7
:108679001DF3909F5212874B202A7602871E3012D3
:1086890023305E2030501D028A2F301217305E06CB
:03869900200B11A2
:10869C0002909012CA147F1712DDBC75172002DAF3
:1086AC006712D62212D5C330121120510512D68270
:1086BC00800612CD6812CB481251AB22E4FEFFE5C6
:1086CC004824F6400D90A40B1277357E16E548022F
:1086DC00D4C3B40E0690A41102773590A418127767
:1086EC00357E12E54824F702D45E7D20800C7D3F58
:1086FC00302A077D633029027D3C7F0080247D2059
:10870C0080127D3E800E7D3CE54975F007A4240661
:10871C00800A7D3FE55975F007A42409FF640270B7
:10872C0001FF7E1CED02D4D67D2080027D3FE55BEF
:10873C0075F009A42416FF7E09ED02D4D6C24912A5
:10874C0087AFB4FF01227510001287C67920E03084
:10875C00E702792F3049171211AEFAB40408E5106C
:10876C00700C79658008EA14651070027923E97E33
:10877C001812D4D67E20E51230E708909F8D127720
:10878C00358016E51112883C125D0D201005201164
:10879C000280063012031287EE0510C3E5589510BF
:1087AC0050A7227E207F001277351286C87E007F6C
:1087BC000690886E12D534E5582275A70475830788
:1087CC00125AF1E51075F007A42409FFF5177E0085
:0B87DC00E51212D4D67805EE2404FE4E
:1087E700E012D4D6D8F6221288F612890CFD7C0046
:1087F700AE1CAF1B12546FBE003A8F00C3E57A95CB
:1088070013FFE55E9514FE402B7C007D2812547CF7
:10881700C3EF98401F75F0058404FB24F950027BD1
:10882700067E2CAF170F12DE610F12DE610F12DE0C
:10883700610EDBEF2264B4602464B475F03284C047
:10884700F012D4C3CE2404CED0E075F00584C0F076
:1088570012D4C3CE2404CED0E02302D4C390886AB6
:108867000277352D2D2D000140FFFFFFE0FFFFFFB1
:10887700FFC25030123F20283CE558F460372048AB
:1088870003200931D250E559F51030330665586099
:108897000205101288C012891C75A7049006DCE532
:1088A70012F0E511F0E517F0E510F075A704900652
:1088B700E0ECF0EBF075A7002275A70475830712AB
:1088C7005AF17813E0F608B819FA9006D07811E64D
:1088D700F008B819FAE51CF516F0E51BF515F012C6
:1088E70088F69006DAE514F0E513F075A70022750F
:1088F700A704758306E51023541E24B0F582E0F51E
:1089070013E0F51422120E71E5BD2487E5BD923BF5
:0289170050020C
:1089190024912212890C75F005A485F012F511E451
:10892900F519FEF51CF51D12BE75C23DC2567F3CF8
:1089390012CABE303D05751900807DDFF3E5596522
:1089490058700A301007EE24D35002D2568C1B8D72
:108959001AE519FD24E250DEAE1CAF1D7C0012544D
:108969006FEFF51924F650CEAC1BAD1A12CA0320CD
:10897900D1108E048F05E51975F0A7A4AEF0FF128A
:10898900546FAC12AB117AA012539AEB33FBEC3350
:10899900FC20D11AEF9BEE9C5014C3E51213FCE5A1
:1089A9001113FBC3EF9BEE9C4004AC06AB072048B8
:1089B90007203B048C128B119006E2E519F0128A0C
:1089C90004AC16AB157AC8125371A912A811125525
:1089D90015ED7005EC249E50057C807B0822C3E5CB
:1089E9007A305602E55C9513FFE55E305602E55D87
:1089F9009514FEC3EF9BFBEE9CFC22AE16AF157CD3
:108A090000E519FD24F6501A12546F7C007D0612F8
:108A1900534F7C007D0512546F8F10EEF51724E932
:098A290050037517FF2212CA1454
:108A3200128A4C128A8F12D278128AB520480912F1
:108A42008BA3128BD3028C3680747F177E20204832
:108A52000E748A204D101258B5500E742F80077470
:108A62006A305F02746712D50875A7049006D07841
:108A720011E0F608B819FA7F177E00781275190509
:108A8200E60812D508EE2406FED519F42275A704CD
:108A92009006D8E0F516E0F515E0F514E0F513E0E0
:108AA200F512E0F511E0F517E0F510E0FCE0FB75DA
:108AB200A700227F187E26AC14AB1302D30A9006BD
:108AC200E4E0F51CA3E0F51B7F2A304E13120E677B
:108AD200E5BF90A475B4010390A66F1276F08042B0
:108AE2000F7E00745312D4D69005CBE0F830E70520
:108AF200E53F30E0091F7E00E8540F12D4EE9004E7
:108B0200EEE0FEF51EA3E0FFF51F128B4BE51E24DF
:108B1200E9500C7E06742B12D5087E0C12D5081271
:108B22008B7BC20375172A751627125C7C202415CD
:108B3200205F15D2037F2A7E1E908B69304E0390F0
:108B42008B7202D534205FEB227C007D3C12547C78
:108B5200A805EF7F2A7E0812D4117E12743B12D52B
:108B6200047E14E802D40B0707384C9EBAF264382C
:0F8B72000707387CE6C2E67C38AC1CAB1B7A48A0
:108B8100305D027A27125371A91EA81F125515EDE7
:108B91004C60027BFF7F207E28EB12D4177E3902C6
:108BA10091237F2B90A41E127733E517F46022AE38
:108BB10017AF107C007D3C12547CA805EF7F2A7E04
:108BC1000C12D4117E16743B12D5047E18E812D40F
:108BD1000B22AE12AF117C007D0A12547CA805EF66
:108BE1007F207E3012D4117E3A742C12D5087E3C3F
:108BF100E812D4EE0F7E29744502D4D6748580071D
:108C0100748720560274867E2912D508301707749E
:108C11002D7E3A12D508227C007D0A12547CA805CB
:108C2100EF7F2A7E3012D4117E3A742C12D5087E41
:108C31003CE802D4EE128D67E54824F65005128C0B
:108C41001880B9E559046558600D128C18128BFD16
:108C5100E559655860AA22A217923D8E1E8F18858C
:108C610015179006D0E0F51185581015101245B46E
:108C7100C3E51195105002F404F924A65005C374FC
:108C8100B399F9E975F00584F924EE500279119050
:108C91008DA7E993F5F0120920E5CC7004E930E7DE
:108CA10002747F23A4A9F0E51B2517FDE51C3516E9
:108CB100FEC3ED99F515EE9400F51675A7007583C1
:108CC10006E55823541E24B0F582E0A3F513E0F520
:108CD10014128D67203D2C201729120E71E5BD2439
:108CE10087E5BD5002249175F007A4FB9518E5F0C6
:108CF100951E400FEB9FE5F09E4008EF9518EE950D
:108D01001E500EA23D9217AE1EAF18128C18028B88
:108D1100FD306B10128D04E53F20E00774867E2242
:108D210012D5082275A7009006E0E516F0A3E51517
:108D3100F0128C18128C0174857E2312D508855887
:108D4100101288C0128A4C128A8F8C168B15128AC7
:108D5100B51289CA1288B212D2789006E2E0F519EA
:108D6100128A04028BA3C3E57A305602E55C95139F
:108D7100FFE55E305602E55D9514FE921750031231
:108D810055E6AC16AB157AC8125371A906A807129D
:108D910055157E037FE7ED700CEB2418EC34FC4095
:108DA10004AE04AF032200172E43576C8092A4B681
:108DB100C5D3DFE6EDF3F8FD305E4F30504C75A7BB
:108DC100009006E0E0A3FCE0FBECA2E79217402054
:108DD10024FE50047F3B8022AE04AF037C007D144F
:108DE10012547C74542F2017029F9FFF7462800CD1
:108DF1001255F6EC24FE50E07F6D743D7E0012D4D6
:108E0100D67E017D197C03128E0C227F3D12DE611C
:108E1100EF2DFFDCF822E537B40206E534243750A4
:108E2100292212DF1C12D6AB12CF88128FA312C8CF
:108E31005E12CDF5128FFB125B477F207E2B12D085
:108E41006612D73D12DC761238A812D19E128ED14D
:108E510012514502DD4620041EE579FD24A0500291
:108E61007D5FED24CD401E744520750C2DFFF5125C
:108E7100128EA61FBF44F922C39DFFF512128EA6C2
:108E81000FBF46F92220750EED2413FFF512128E45
:108E9100A60FBF78F922C374779DFFF512128EA633
:108EA1001FBF12F922EF24BA40082433FCC37432E5
:108EB1009C1404FC24D750047C238009EC2375F016
:108EC10005842413FC7E0512DE610EECB506F82242
:108ED100E59020E206E53424374003128E577F45A2
:108EE1007E047D1212DE610EDDFA7F437E00746422
:108EF10012D4D67F4F7D12128F8C7F3B7D12128F41
:108F01008C7F597D16128F8C7F317D16128F8C7F4D
:0F8F1100637D1A128F8C7F277D1A128F8C7F6DD4
:108F20007D1E128F8C7F1D7D1E128F8C7E057F19FA
:108F300012DE610FBF72F97804E57924CD50027812
:108F400009E8305C0123F87F1B128F7B7F6B128F47
:108F50007B18305C01187F25128F7B7F61128F7B1D
:108F600018305C01187F2F128F7B7F57128F7B1870
:108F7000305C01187F39128F7B7F4D7E00E875F0E1
:108F80000A847004E802D4C3E802D45EEF6512607C
:108F90000C7E04EE20E00712DE610EDDF62212DE0A
:108FA0009180F790A5357F287E2C1277357E3B1275
:108FB000D321AC5EAB7A7F307E19C23D12D3609074
:108FC000A4227F5D7E2D12773578B9C3E57A961895
:108FD000FBE55E96FC7F507E19D23D02D360E51121
:108FE00064B4700122E51112DCE67831790F7D0B53
:108FF00012DDE41F1E90908B02D534E5716012E5FE
:109000007012DCE67831790F7D0412DDE00DBD0AC7
:10901000F97F011290637F1D1290637E2312906D81
:109020007E3F12906D7E247F171290777E397F02EB
:109030001290777E247F071290817E397F1C1290D8
:10904000817E317F0212DE617F1C12DE617F0F7E26
:109050002412DE617E3E12DE617F0C7E2E90D829C6
:1090600002D5347E2A12DE610EBE39F9227F081243
:10907000DE610FBF17F9227D0612DE610E0FDDF9EA
:10908000227D0612DE610E1FDDF9220303E0A0E05F
:1090900012CA147F18909D621277337F217E01746B
:1090A0004112D4D67F2A7E01745312D4D69005BEC5
:1090B000E0F51AA3E0F519A3E0F51EA3E0F51D8580
:1090C0001A1C85191B751720129140E519251DF5ED
:1090D0001BF51DE51A351EF51CF51E751729129195
:1090E000409005BA129130AC1AAB19751720129046
:1090F000FE9005BC129130AC1EAB1D751729EC70AB
:1091000006EB24CD4001227A48305D027A271253C3
:1091100071125515ED4C600122AF177E07EB12D38B
:10912000BD7E1A0F90A5F8305D0390A5FB02773540
:10913000E0FEA3E0FD12BFCBC3EB9DF8EC9EF9224D
:10914000751627025CAD12BFCB75A7049005B478E5
:10915000737F06E6F008DFFBECF0EBF0E0E0E0FC0C
:10916000E0FDE0FEE0FFEF2DFFEE3C9005C0F0EFEC
:0B917000F0801275A7049005BAE0FB28
:10917B00E0CBF0EBF0E0E0E4F0F075A7002275A790
:10918B00049005B478647F06E0F608DFFB75A70052
:0E919B00125EBC9005BEE51CF0A3E51BF022A1
:10393A00D23C799E77008002C23C12BE75E4F51033
:10394A00F511F512F513F514F515F516F517C23D2F
:10395A00123C8A203D1F123C8A203D19E51F30E5A2
:10396A001130E40E1239B1303C08799EE724F55043
:10397A000122D510DBAE14AF157C00AD12125449EA
:10398A008F55AE16AF177C00AD1312546F125670D6
:10399A007E00E55530E7011E2DFFE43E30E7027F49
:1039AA0000740A2FF55622C235E51CAF1DBFFF056C
:1039BA000FD235F404FABF003F532CF8E518AF19BB
:1039CA00BFFF050FD262F404BF002D20E72A205B57
:1039DA000123FF24AA4021E51AAE1BBEFF050ED221
:1039EA0061F404BE00128547F0A4E5F020E709203F
:1039FA005B0123FE24AA5001227C807B8030516621
:103A0A00302163C006C0078AF0E545A4AEF0FFE5A1
:103A1A0056205B011375F009A4ACF0FD12546F74C3
:103A2A00FFBE0001EFFA24C050027A3FD007D00649
:103A3A00E55212DCE6303504B2D5B2D1EA8CF0A4F4
:103A4A0030E70205F0748025F020D10495F095F056
:0A3A5A00FCEA8BF0A430E70205F04F
:103A6400748025F030D50495F095F0FBC3EC2F203D
:103A74006203C39F9FFFEB2E306103C39E9EFE2013
:103A84003C64200C05123B1E4064123B00405F1254
:103A9400DE61E51EFD24FB50550E12DE61ED24F6B9
:103AA400504C1E1F12DE61ED24F150421E0F12DE37
:103AB40061ED24EC50380F12DE61ED24E7502F1F26
:103AC4001F0E0E12DE61ED24E250231E0F0F12DED4
:103AD40061ED24DD50180E12DE61ED24D8500F1E66
:103AE4001E1F1F02DE61123B004003799E0722E97C
:103AF400242AFFE82461FE123B1E401DEF2460408F
:103B040018243F5013EE2460400F243F500AEF2442
:103B1400D6FFEE249FFEC322D322532CF8432C0459
:103B2400EE10E706D2E7F404D261FE24D340EAEFB4
:103B340010E706D2E7F404C262FF24D340DBEFB5FA
:103B440006005003CED26070057480FE8062FF24AC
:0D3B5400FD5060903C0A938EF0A4AAF0335F
:103B6100CA33CA33CA33CA33CA33FA903C34938F47
:103B7100F0A433C5F033CA903C5593FB123BD29568
:103B810070500224B412DCE6EA8BF0A430E702059F
:103B9100F0C3748095F020D50425F025F0FEEA8C61
:103BA100F0A430E70205F0C3748095F030D104250C
:103BB100F025F0FFC3227A01EE6F70097B16BF0278
:103BC100BB7A0380B7BF01047B0080B07B0D0A8004
:103BD100ABE52C540723C3903BDC73800E800E8031
:103BE10024801E8010800A80108012EB22742D9B8D
:103BF10022742D2B22745A9B22745A2B2274879B78
:103C01002274872B2274B39B22FFFFCCAA9280716E
:103C1100665D554E4944403C383533302E2C2A28B8
:103C2100272524232221201F1E1D1C1B1A1A1918A7
:103C31001817178181818282838384858687898A87
:103C41008B8D8F90929496989B9D9FA2A4A7A9ACCF
:103C5100AFB1B4B400010203040405060708090A60
:103C61000A0B0C0D0D0E0F0F10111112131314145A
:103C7100151516161612BDAD12BC3BE4F5F7C2B20E
:103C8100C2B2E5F7D2B264C022203D07123C767081
:103C910003D23D22056D056D12BC3B7D008DF7C23F
:103CA100B2C2B285F71F8DF7C2B2C3E5F79573F5BE
:103CB100188DF7C2B2C2B2E5F79574F5198DF7C246
:103CC100B2C2B2E5F78DF7C2B2C3E5F79576F51A40
:023CD1008DF76D
:103CD300C2B2C2B2E5F79577F51B8DF7C2B2C2B295
:103CE300E5F78DF7C2B2C2B2E5F7F51E8DF7C2B2A2
:103CF300C3E5F7957AF51C8DF7C2B2C2B2E5F78D2D
:103D0300F7C2B2C2B2E5F7D2B2543F30E50244C0C3
:103D1300955EF51D156D156DE51024784001227E25
:103D230000AF55EF30E7011E0512E51FA2E592D55E
:103D3300400EE515951EF515E5149400F514800B5A
:103D4300E515251EF515E43514F5147800E51E6018
:103D53000620D50318F404C39FF5F0E89E30E7016D
:103D6300220513E5F0A42517F517E5F03516F5162A
:103D730022303D03D23D22123C7660F8123C76603D
:103D8300F3E546600A123C7660EA123C7660E5058C
:103D93006D056D056D12BC3B7D008DF7C2B2C3E5A9
:103DA300F79573F5188DF7C2B2C2B2E5F79574F5BE
:103DB300198DF7C2B2C2B2E5F78DF7C2B2C3E5F708
:103DC3009576F51A8DF7C2B2C2B2E5F79577F51B72
:103DD300D2B2156D156D156D2230742412BE75C2E5
:103DE3003D75101E123D74203D167902123E484067
:0A3DF3000CA806A907123AF34003DA
:103DFD0012DE61D510E422200F4030123D2006CF97
:103E0D00304806200C03204FC6E546790260147930
:103E1D000614600F791614600A79361460057976E8
:103E2D0014701712BE75C23D7896123D74203D0A6E
:103E3D00123E48400312DE61D8F022532CF8AB1825
:103E4D00E519FC339262123E9ABC002BEB89F053BC
:103E5D00F00784FF24DF401FAB1AE51BFC33926192
:103E6D00123E9AAA4712539ABC000CEB89F053F0FC
:103E7D000784FE24DF5002D32274562F2062029F46
:103E8D009FFF741F2E3061029E9EFEC322500312AF
:103E9D0055F6E920E40122C3EC13FCEB13FBE920FA
:103EAD00E50122C3EC13FCEB13FBE920E60122C371
:103EBD00EC13FCEB13FB2274542F2062029F9FFF27
:103ECD00741D2E3061029E9EFE2279B4203249204F
:103EDD001D46EFB506009260AC06AB074004AC077B
:103EED00AB06903F26EC2304938BF0A4A9F0EC23B2
:033EFD00938BF0B4
:103F0000A429F9903F8693C9904086E52C540793E5
:103F100013E95001F490408EF9E52C54079329756C
:103F2000F0B484A9F022FFFFFFFF7FFF55553FFF4C
:103F300033332AAA24921FFF1C711999174515556E
:103F400013B1124911110FFF0F0F0E380D790CCC60
:103F50000C300BA20B210AAA0A3D09D8097B0924BF
:103F600008D30888084207FF07C107870750071CC6
:103F700006EB06BC06900666063E061805F405D15B
:103F800005B005900572000000000001010101016B
:103F90000101010102020202020202020203030302
:103FA00003030303030304040404040404040405D6
:103FB00005050505050505050606060606060606A9
:103FC000060607070707070707070708080808087E
:103FD0000808080808090909090909090909090A55
:103FE0000A0A0A0A0A0A0A0A0A0B0B0B0B0B0B0B2A
:103FF0000B0B0B0C0C0C0C0C0C0C0C0C0C0C0D0D02
:104000000D0D0D0D0D0D0D0D0D0E0E0E0E0E0E0ED9
:104010000E0E0E0E0F0F0F0F0F0F0F0F0F0F0F0FB4
:10402000101010101010101010101010101111118D
:10403000111111111111111111111212121212126A
:104040001212121212121213131313131313131347
:104050001313131313131414141414141414141426
:104060001414141414151515151515151515151505
:1040700015151515151616161616161616161616E5
:1040800016161616161600FFFF00FF0000FF002E82
:10409000B5875B2D5A88E537607414603EB40258CA
:1040A0007F347E12E5342437400810644B90A3F22D
:1040B000801AF89041E012D534E824FD501179A11E
:1040C000E77E0590A22D20E70390A2360F803A24C8
:1040D000040F7E2312D4F5D26480627F357E02E520
:1040E000342437401410641090A11A30081B127742
:1040F000027E1A90A3F1801122700590A12E8009F2
:10410000909D8F200C03909D9B12770280C97F3574
:10411000E5342433402A2404501B7D0F600C7D1E9F
:104120001460077D3C1460027D78ED305D02C3139E
:104130007E2B12D3BD7E0090A12F12770202DD46A6
:104140007E0524FE5005909F7A8009909D72200F75
:1041500003909D7E12770280E4E546604A14603C3D
:1041600014602E14602014601290A62C205D4190E3
:1041700041D97F367E3412D534803C90A62C305DF8
:104180000390A628802A90A628305D0390A624805C
:104190001F90A624305D0390A620801490A62030A6
:1041A0005D0390A61C800990A618305D0390A614AC
:0241B0007F3658
:1041B2007E331277357E3C7422305D02748302D5E1
:1041C20008305D0890A604305BE4800690A60C20BF
:1041D2005BDC90A60880D70508B28D8DB5BA0910B0
:1041E20006000A10F248922492249224F2480A10FD
:1041F2000600305E5220434F20284CE55864FF6091
:1042020046E54824F640407F3FE55804F9C23D1296
:10421200424A1211AE601AB404047401D23D75F020
:1042220003A4243CB5070A7E3A303D027E36124290
:104232004C0F0F0FD9D7E55975F003A4243EFF1296
:10424200424A0F0F12424A227E3D12DE610EBE40EA
:10425200F922C248C249305E56202853E55864FF0D
:10426200604DE54824F640471211AE6042D249B48F
:104272000402803B1465597036D248304E31E559FC
:104282006558602B3074281242B7120E67E5BFB42E
:10429200011DE5BD20E618202416205F129006E4D9
:1042A200E0700CA3E024CE400624255002055922DA
:1042B200305FFC80E820113375A7009006E4E070BF
:1042C20028A3E0302402F404305F02F4042404F949
:1042D20024F74015E924FC4003D26C2270012230FD
:1042E2006C097536A7D22ED22FC26C22305E0830EE
:1042F2007405E558B4FF0122C244C24D780075A787
:0B4302000475830712463688188A1ED7
:10430D008E168F17C23EC23BE54824F6500302437A
:10431D00C7D23EE55860F7E8655970F22048EF12B4
:10432D00447C30D13BAE16AF17A818E54670551238
:10433D000920E5CC49604DD244E5CC7033E924CD5C
:10434D00402EE975F038A4ACF0FB12558512558559
:10435D00EBFDF5111243DD304D2CC206C23B8043FF
:10436D00E546705C120920E5CC7005E924CD50506E
:10437D00124F7C75A704758307A8181246368A1E3E
:10438D008E168F178037120E67E5BDA2E0B3923BF4
:10439D005011307428123AF34026A907A806D20608
:1043AD0012CAA51243F91243F0124439890788063F
:1043BD001E1F90463112D534800630D103124411A0
:1043CD00A81808C3E55898400302430075A70022BA
:1043DD0074562F2062029F9FF9741F2E3061029E2A
:1043ED009EF822E51865586001227D057A00EA12D3
:1043FD00DCE612DDE40A0AED24F240020A0AEA24A0
:10440D004C50EB22AE16AF17123EC41E303E021EAC
:10441D001EE51E12D4D6EE2404FEE51212D4D630BB
:08442D003E09EE2404FEE51334
:1044350012D4D622E5186558603CC001C000C012F0
:10444500C0138518101245B4D013D012D000D00176
:10445500E510303B07C39570500224B412DCE6200A
:104465003B07AE16AF171243DDE5112402FD7A06B0
:1044750012DDE41DDAFA221211AEB40457E87054C5
:10448500120E85E5BD604D78C6A61308A61208A6CE
:104495002C12C85275A704758307751001125AC2EC
:1044A50012C84C1510125AC21256DC8E628F631256
:1044B50057648B1C8A1B12C85820320E1245642083
:1044C5003B08D24D1266FF1244DA78C68613088679
:1044D5001208862C22120E85AABD7C027BB31253CC
:1044E5009A8C128B13AA1DA91F1253DCA91CA81B99
:1044F5001255158C1D8B1FAC12AB13AA19A91A12D4
:1045050053DCA91CA81B1255158C198B1AE56E25B1
:104515001AF9E56D3519F8C3E56E951AFBE56D9544
:1045250019FAC3E554951FFDE56F951DFCE5542566
:104535001FFFE56F351DFEE52C23652C30E206ECEB
:10454500CEFCEDCFFD75A7049005C2E8F0E9F0ECCF
:07455500F0EDF0EAF0EBF0DD
:10455C00EEF0EFF075A70022D23BC3E5649573C56E
:10456C00659574F564E5669575600404600822E54C
:10457C006424E0500822E5642420400122C3E5674E
:10458C009576F567E5689577F566E5699578600940
:10459C0004600122E566F48002E5668562F0A4748D
:1045AC00E025F04002C23B2212C85275A704758365
:1045BC0007125AC212C84C0510125AC2C02C125AF9
:1045CC00DBD02C891002C85830125120064E7800CE
:1045DC0075A70475830612463630D139123EC4E5F0
:1045EC004624FE500A0E0F90462C12D5348026EA33
:1045FC007007745D12D4D2801C75F06484ADF070B9
:10460C000FED75F00A847008E5F00E12D4C3800526
:10461C001EED12D45808C3E55A9850B475A7002261
:10462C00030340A040030340E040D2D1E8C4F5822C
:10463C00E0FA797312468F30D146AF06532CF8ED61
:10464C00BFFF07F40460390FD262BF00331247C3B7
:10465C00402E797612468F30D126E5822403F582DE
:10466C00E0F512E0F513EEA2E713FEED13BEFF0723
:0A467C00F404600C0ED261BE0006CB
:104686001247E0400122C2D122C3E09709FDE0971C
:1046960009FEE097600904700AEE30E7068007EE2F
:1046A60030E703C2D122E546600E14600BF9EDCE69
:1046B600A2E713CE13D9F8FD227C007B44E54660C1
:1046C600207C007BCC1460197C017B981460127CE2
:1046D600037B3014600B7C067B601460047C0C7BCF
:1046E600C08C148B157AE9125371A8471255138C96
:1046F600168B1775C70075C6047510DF75B901E509
:10470600BC20E76FF51385BD1205C605C675B90150
:10471600532CF8C3E5BE9573FBE5BF9574FC05C63F
:1047260075B901E5BC9575FD5005D2621255FEC3FB
:10473600E5159BE5149CE49D40338C198B18C3E565
:10474600BD9576FBE5BE9577FCE5BF9578FD5005F2
:10475600D2611255FEC3E5179BE5169CE49D400DFC
:104766008C1B8B1A12478AE5322428401305C6E5AE
:10477600C68006E5C62404F5C6700205C7D5100135
:0F47860022024702AE19AD181246ACED1247C31E
:10479500AE1BAD1A1246ACEE13ED131247E0123EF6
:1047A500C4E54624FB50080E0F90463102D5341E51
:1047B500E51312D4D6EE2404FEE51202D4D675F024
:1047C500067FFDA946B9000575F0027FFF84C5F097
:1047D5002F500205F0C5F0FF24DE228547F0A430F6
:1047E500E70205F0E5F0A946B9000280050475F079
:1047F5000384FE24E022E537B4020122E537700286
:10480500D23964027002C239E53724FC799EE7602B
:1048150005640B600C22D27E20081E401C107F1000
:1048250022D27F2008134011107E01227537012204
:104835007537002039037537022275F9FF75FB00BE
:10484500800E75F9FF75FBFF801C2053F512487D1E
:10485500759E85759D2D801412487D759E84759D68
:104865002D800912487D759E83759D09C2AC75988A
:1048750052C26DC26EC26F2212166EC253E4F5F9B2
:10488500F5FB30340215FB22D2A47F3212DE3EC284
:10489500A412D9BD12DD4612DE27C214C215124874
:1048A5003F74C012DC7174A312DC2E748F12DC2EDF
:1048B5001248D374C012DC7175A7049048DD7F10CF
:1048C500E49312DC2EDFF91248D375A70022E538F0
:0548D50012DC2E74CA84
:1048DA0002DC2EA29494859C8080808080818380D3
:1048EA00819E8075A60A12489FD269D2ACE5A62499
:1048FA00FA500C306DF712DBC3B4E0F1124935C23D
:10490A00ACC26975A6FF22D21EC274C273E4FDF559
:10491A0071F570C22D12483FD2AC12DBC3C5F070DC
:10492A0005DDF7C2AC22C5F0B4E0EFF538E4F532A4
:10493A0012DBBEA2E19273A2E2927475A7049004FC
:10494A00B4F012DBBEC2D1124B1C20690330740BC7
:10495A008D758E748F73E514C4F57D124B9C124BC2
:10496A001C20690330740C8D788E778F76E51425B8
:10497A007DF57D124B9CD2D1124B1CEEF0F55DEF0A
:10498A00F0F55C207303E4FEFF79BCA70609A707CC
:10499A0012DBBE7D0A124B898F71EE60037571FFBF
:1049AA007D14124B89C22DED24F150010F240A50B7
:1049BA0002D22DBFB4027F008F7012DBBEF0540703
:1049CA00C52E54F8252EF52EE571700EE4F571F515
:1049DA0070C22D9004BFF0F0F0F012DBBEE5386033
:1049EA0009D21EC27412AF0A8005C21E12AF061285
:1049FA00DBBEB4E1FA75A7049004C412DBBEF01260
:104A0A00DBBEF0F53A12DBBEF0F53B12DBBEF0F589
:0B4A1A003C12DBBEF0F53D12DBBEF0ED
:104A2500F53E12DBBEF0F53F12DBBE12DBBEB4E293
:104A3500FA12DBBEF07E0C12DBBEFF12DBBE12DB10
:104A4500BE12DBBE12DBBE20E1027F00EFF012DBFF
:104A5500BEDEE412DBBEB4E3FA12DBBEFF12DBBE40
:104A6500CF60027F7F9004E4EFF0E4F012DBEE907C
:104A750004D8124B8912DBBEB4EAFAC2AC75A7049E
:104A85009004DAE561F0E560F0E55EF0E57AF0E5E1
:104A950079F0E52EF0E55FF0E57BF0E551F0207467
:104AA50012E4F571F5709004B4F09004BDF0F0F0E7
:104AB500F0F0F075A70078ABA63A08A63B08A63C2F
:104AC500120E7BE5BF253D240C75F0188478AEA643
:104AD500F0186005640260182216E670121816E6D2
:104AE5007004760C181678ACE6904B0F9308F622F6
:104AF5000618E608904B0F930466700D76011806AC
:104B0500E6640D70047601180622001F1D1F1E1F86
:104B15001E1F1F1E1F1E1F12DBBEFC12DBBEFD1259
:104B2500DBBEFE12DBBEFFECA2E692E7921713FC9A
:084B3500ED92E713FDEE92E79B
:104B3D0013FEEF92E7301701F4F513ECA2E713FC27
:104B4D00ED92E713FDEE92E7301701F4F512ECA2AA
:104B5D00E713301701F4F510ED92E7301701F4F576
:104B6D00111255A620D10E8C1C8D1D8E1E8F1F125D
:104B7D00B3121255A630170312B2EC2212DBBEC3CC
:104B8D0013FEF012DBBE92E7FFF07C0002547CAC0A
:104B9D001CAD1DAE1EAF1F30170312B2ECECF0EDC5
:104BAD00F0EEF0EFF022124BBC0202C612BC7AC23C
:104BBD00101248F07F5A7E0590A40112770212DD83
:104BCD0046D214D215C255122CEC789F76800876F9
:104BDD000012BCBA1232FA7570FE853A71853B72BD
:104BED00853C73853D74853E75853F7612BD1912E2
:104BFD0032FA7570C0757B03757A54E4F57FF57ED6
:104C0D0012BD19751421751348755F01757B0075FB
:104C1D00750475745275780175776CE4F57DF551F1
:104C2D00757F0190DF5C85836E85826DC23D124C70
:104C3D009A851C1D75A6FF305505C221022EA7129F
:104C4D004C9AE572A2E59275A2E79277D274D2736F
:104C5D00E51275F008A4AEF0FF2075031255E612AB
:104C6D00C7A212C7EB124D1DE51C251D13F571854D
:054C7D001C1D12BC9299
:104C820012BCEA757F02E56A70B57F5A7E2FE54154
:104C920012D3BD12DD4680A7856E83856D82C25513
:104CA2007873124CFE7876124CFEE493F570B4B42D
:104CB20002D255A3E493F51CA3E493F512A3203D7D
:104CC2000FA97BE493F57BC399502A20E702055F85
:104CD200A385836E85826D103D16D23DE582240543
:104CE200F582E43583F583E493F52654F0F57222D8
:104CF200E526C480F630E7D8155F80D48601E493B8
:104D0200F6A308C399500A20E70606B60002080671
:104D12002230E70616B6FF0218162230750DE5138B
:104D22002579F513E43514F514800DC3E51395794F
:104D3200F513E5149400F514AE14AF137C007D0A4C
:104D420012547C8E5E8F7A22124DDF851617203D1B
:104D520001227F5A909C831276F07F64E5166404E8
:104D6200700C909C9B12773312DD4602DE21909CE0
:104D72008F1276F07F6E7E0890A5F4127702121ED3
:104D82000312DD467515B87514047F6E7E20C224A9
:104D9200A815E82404F9C23DE7124E27203D06E695
:0A4DA20012D5088008E6128460E8CC
:104DAC00A815F60515EE2406FED514DA851716128D
:104DBC001E5112DD4610000510018D80F878B812D6
:104DCC000E8F86BC0886BD0886BE0886BF124EE6CE
:104DDC0012DF1C120E8FC23D75160078B87F4B7E09
:104DEC000890A5F41277027E20E5BC12D508124E6D
:104DFC001E7E26E5BD12D508124E1E7E2CE5BE1277
:104E0C00D508124E1E7E32E5BF12D508124E1E0278
:104E1C00DD46F608080808F618181824D0500524A2
:104E2C00F64001220516D23D2275C70375C6FE1247
:104E3C00766E124EE675C6FC75BC2675BD6475BEE5
:104E4C00A975BF70124EE675C6FB12766E124EE651
:104E5C0075C6FA75BC1475BD1475BE0075BF0C1201
:104E6C004EE675C6F975BC4E75BDBF75BE0075BFF7
:104E7C0019124EE675C6F875BC0A75BD7E75BE0076
:104E8C0075BF01124EE675C6F775BC0175BD23756D
:104E9C00BE4575BF67124EE675C6F675BC0275BD8C
:104EAC00AB75BE0175BF01124EE675C6F512766E76
:104EBC0075BE0275BF0A124EE675C6F412766E7593
:104ECC00BCE1124EE675C6F312766A124EE615C6B2
:104EDC00124EE615C6124EE615C675B90575B90221
:104EEC0022751500127D6775B901E5BC64816003FC
:104EFC001276510515E515242050E975C70375C6C2
:104F0C008075B90505C6E5C6241C50F5124F1E0266
:034F1C007BBDE476
:104F1F00F5C7F5C6742612766F75BD4E124F38124F
:104F2F004F35E4124F3512766F124EE605C6227FCB
:104F3F00357E00E54B12D4747E10E54C12D4747E8E
:104F4F0020E54D12D4747E30E54E12D474227F4684
:104F5F007E00E56C12D4747E10E56B12D4747E2043
:104F6F00E56A12D4747E30E57F12D4742220740166
:104F7F0022D24475A700758307E559C454F024075E
:104F8F00F582E0F51A244C40E7A3E0F512A3E0F513
:104F9F00131209208938120E67E5BDA2E0923BE596
:104FAF001A40069570500224B4F51A203B05D2061C
:104FBF0012CAA5E51A1250DFE5152437F51DE435A1
:104FCF0014F51CE5172437F51FE43516F51E85CCAF
:104FDF0012853813AC12AB137A0412536375380170
:104FEF0024FA401A05382402401405382401400ED3
:104FFF000538053824014006053805380538C3E55E
:10500F001A945A500224B4F51AC23BC23CC23D75E1
:10501F001B00A23B823C406D203B2CE51A75F0082B
:10502F00A4951BFBE5F0303D04940180029400FC35
:10503F005008EB24A0FBEC3405FC1250E6125095FF
:0A504F00923B40031250B8203C2CA5
:10505900E51A75F008A4251BF9E4303D010435F083
:10506900FAE994A0FBEA9405FC5004AB01AC0212E6
:1050790050E6125095923C40031250B8E51B253872
:10508900F51B5094203D04D23D808D22E51F251744
:10509900FEE51E35167016EE24914011E51D251505
:1050A900FFE51C35147006EF2491400122D3228EAE
:1050B900027C8A7B3B125371ED2402FE8F027C8AAB
:1050C9007B3B125371ED2439FF02DE611256CF800A
:1050D900311256C2804675F008A4ACF0FB75190070
:1050E900C3EB9468F9EC9401FA40080519AC02ABDA
:1050F9000180ED8C108B11531903E51920E0CD12B5
:1051090056C212513AAF05E51924FE50031255E66D
:105119008E168F17E51920E0B81256CF12513AAF03
:1051290005E5191460061460031255E68E148F15EF
:1051390022AC06AB07AA12A9130253DC125227208C
:105149003D4974857F227E0812D5087E0830173CB8
:10515900AC1EAB1FEB2418EC34FC402F125342E574
:105169001B60077F207E0812D5237F207E10E51A59
:0951790012D5237F237E17742E4A
:1051820012D5047F207E1BE51B7011E519C2E012C7
:10519200D523227F207E0E740A02D523E51975F0ED
:1051A200058475F005A402D523125227203D5E74B2
:1051B200857F227E3A12D508301753AC1EAB1FEB07
:1051C2002418EC34FC4046EC7033EB249C402E7ED9
:1051D2002D125219125585C0E07F2A7E2EEB12D570
:1051E200237E39D0E0C2E012D5237F347E3712DE2F
:1051F200611E12DE611F12DE610E02DE617E30125E
:105202005219125585EB7F2A7E3112CE47227F2A10
:105212007E39740A02D5237F2912DE910FBF34F939
:105222000EBE40F322D23D301266120E71E5BDF57C
:105232001C75F00AA4F824E15002781EE4FCFBFE7F
:10524200FFC23D12BE75125293203D44D8F8751D1F
:10525200CEE51C146009751D9C146003751D6AC29D
:1052620017EC30E705D2171255F68C018B00E9488E
:105272007003D23D22EE7008EF251D4003D23D227D
:10528200AC06AB077A1C1253711255158C1E8B1F7C
:1052920022203D07123C767003D23D22056D12BCDE
:1052A2003BE4F5F7C2B2C2B2ADF7F5F7C2B2C2B291
:0252B200E5F71E
:1052B400FAD2B230E4E3ED2FFFE43EFEE56D2408BC
:1052C400F56D12BC3BE4F5F7C2B2C2B2ADF7D2B28F
:1052D400EA30E508EB2DFBEC3400FC22C3EB9DFB2C
:0552E400EC9400FC2227
:0100030055A7
:10DF5C0069FC362E06FD69FC372F071169FD383038
:10DF6C0007FD69FD3931061169FE383107FD68FE80
:10DF7C003732091168FF373008FD68FF372D07115C
:10DF8C006800362909FE680036290C116801372B08
:10DF9C000CFF6801372F0A116802383009FF68023C
:10DFAC00372E08116803372C0AFE6803372E081128
:10DFBC006704373208FE67043633091167053535B7
:10DFCC0005FF6705353303116706362F02FF670619
:10DFDC00362B05116707362B07FF6707352F051101
:10DFEC006708353104FF6708332E0511670931289E
:10DFFC000700670931250A11670A35240B01670AE6
:10E00C003A240A11660A3C210801660B3D1E0B11CD
:10E01C00660B3D1E0C00660B3D200A11660C3B2165
:10E02C000CFF660C39220E11660C37231100660D9D
:10E03C0036240D11660D34260F01660E3226111191
:10E04C00660E32251401660F35251311660F37271E
:10E05C0016016610392918116610392B1502651135
:10E06C00392D11116511372E0C026512332F081141
:10E07C006512312F07026513302C0A1165132D29F7
:10E08C000E0265132A271011651429270E02651438
:10E09C002C290C1165153129080365153726071134
:10E0AC006515321F09036516411B09116516411CC4
:10E0BC0008036416461F081164164D2105046416E6
:10E0CC005922031164166425040563156A2407118B
:10E0DC0063156D23090663156C230D1163156C25EF
:10E0EC00130762146E2B151162146E2F1406621333
:10E0FC006E30161162136E30150761136F311211E9
:10E10C0061126F350F0761126F380D116011723A81
:10E11C000A086011763F0611601079420209600FFF
:10E12C007A3A0533600F7832040A5F0F742C01338E
:10E13C005F0E722B030A5F0E732E08115F0E743084
:10E14C00050C5F0D722C02135E0D6C2B010C5E0D19
:10E15C00622C05315E0D5F2B030D5D0D5E290833BE
:10E16C005D0D5F23030B5D0D5F1B01335D0D5A16B7
:10E17C00020A5D0D521B00115C0D4D26000C5C0E4D
:10E18C00462802335C0E3926040C5C0F2C2B08330A
:10E19C005C0F23320C0F5D0F172E0A335D0F0C2E04
:10E1AC0009105D0F043507335E0FB23C080F5F0F8B
:10E1BC00AB4209335F0EA43E070F5F0EA2430B3335
:10E1CC00600EA746120B600D9F490C73610C9C49A5
:10E1DC000F0C610B97460973610B8B440A0C610A97
:10E1EC008B420B336109843A080C6108823A043380
:10E1FC0061087934030C60086F2F063360086228BD
:10E20C00050C6008572505336008511F040D5F0885
:10E21C004E1B05335F08491B090D5F094120103760
:10E22C005F0938270D0D5F0A302F06335F0B2B3239
:10E23C00070F5F0B282F0A335F0B262E0E0E600C78
:10E24C0023361137600D1F3F160F600D18411277E2
:10E25C00610D0F320A13610D042B0633610D022E72
:10E26C00040E620D043A0231620E0343050D630D78
:10E27C00B1470113630DA94A000B640CA14D0511A4
:10E28C00640C9B44070E650B99490911650A944768
:10E29C00090D65098E49021365088848060D650845
:10E2AC0081400E336407793B130F6407722F187784
:10E2BC0064076D231A106407692911776407651CBC
:0DE2CC00080F63075D180B33630751190D30
:10E2D9000D630746220E336308402B110F6308387C
:10E2E900291837630932271B0D6309312B1477620B
:10E2F9000A372C0F0A620A3C280973620A441E0B6A
:10E309000C620A48150E33620B46190C0A620B4758
:10E31900260D33610B4C280C0B610B54251037610A
:10E329000B5E24170C600B63291A77600A66361492
:10E339000A600A68390B735F0A6C2C100A5F09724C
:10E349002015775F097422120A5F0873300F775F0F
:10E35900087639140A5F077D3816775F0785370F06
:10E36900095F068D3B0D735F058B4410075F048BB6
:10E37900490C735F048E3F0C075F03863604335FD5
:10E389000394280708600299300E1160029E400527
:10E39900076102A34A0C336101AA4810086201B15E
:10E3A90042127762020131150A6202062B13776362
:10E3B900020830110C63020B361277630310331114
:10E3C9000C6403182B147764032223110A640426AE
:10E3D90023107764042226110A64051C2715776423
:10E3E900051D251508640521271277640628270FBE
:10E3F9000764062F1D11776406350F140764063E5E
:10E409000A19776406401216086407431B117763DB
:10E41900074A22120663075228127763075A2713FD
:10E429000662075E2314776206612011076206649B
:10E439001E0E7362066A1E0E076206742110376289
:10E44900057828130661057A2F157761047A332038
:10E459000661047A301B7761037A281B0761037F01
:10E4690023187761028429160661028832177761B9
:10E47900018D371305610193340C7362009A2E09DB
:10E489000562009D2E043362009D370C0663FFA0D0
:10E4990040103763FFA844140564FFAF4612776440
:10E4A900FF014511056500043F12776500053E101F
:10E4B900076600073F117766000B430D07670110D8
:10E4C9003D117367011539120767021A321277670E
:10E4D900021A2C12076702192C107768031B2E0FDA
:10E4E9000668031F2C117768042729100468042E75
:10E4F9002A0F776705322F130467053330127767C0
:10E5090006362D140567063B291677670643231B34
:10E51900046706471E16776607491E150366074CEA
:10E529001B157766074C2217046607522214776574
:10E53900075B26150265066229157765066D291799
:10E549000165067529137765057D281A0265058217
:10E5590028187765047F1F160265048F2A117765CD
:10E5690003953211006602993D157766029C401C9D
:10E57900FF6602A13E1F776701A43F1CFF6701A741
:10E589004314776801AB4710FF6901B1490F7769F7
:10E5990001024911026A0207490D736A020B480C0C
:10E5A900056B030F480B336B03144A0D026B0419F7
:10E5B9004914376B051F491CFE6C06224824776CE9
:10E5C90006233F21FC6C07203023776C0721272184
:10E5D900FC6C07262420776C08292812FC6C082873
:10E5E9002C0F776C0927230CFF6C09251802316C55
:10E5F90009350F05FC6C094C1401116C09561D01F4
:10E60900FC6B095F2003136B086B2108FB6B087413
:10E619002509336B08772507FC6B0778210D336BC8
:10E62900077A1E0AFB6B077F220C336B06832E0ABF
:10E63900FA6B05853C09336B0489410EF96B048C2F
:0DE649003E10376B038D3C0FFA6B038D40C4
:10E6560013776B02904112FA6C01934110776C01AB
:10E66600984410F86C009B471A776D009F461EF879
:10E676006DFFA24519776EFFA14019F86EFFA640FF
:10E6860014776FFEAA4417FA6FFEAF4A127770FE30
:10E69600B34D18FA70FF024B1B7771FF054718FD43
:10E6A60071FF0942177772000E4012FD7200163D87
:10E6B6000C7372011B3510FA7201232E1577720244
:10E6C60029321AF872032C371D7772032F3014F88B
:10E6D600720336210F77710346190DF87103502026
:10E6E6000B33710353290EF87003572B143770033D
:10E6F600612712F870036F2911777002793017F7C6
:10E706007001803722777001843D1FF67000883FC4
:10E71600197770FF8D3F11F670FF933D0C7371FEF4
:10E72600973D0EF571FE9B3E0C3372FD9F4310F62E
:10E7360072FDA448127773FDAB4C13F573FDB14F10
:10E74600167774FD034F14F775FE074C127775FEA6
:10E756000A4510F975FE0E400F7776FF124111F843
:10E7660076001745167776001C4614F67601214288
:10E7760017777602263D17F3760229382177760336
:10E786002A3315F276032B3009737604302A07F004
:10E79600760439220A337604472110F07504512590
:10E7A60012777504552416F1750459210F777504EF
:10E7B6005F2111F0740463231477740468240EF245
:10E7C600740370230933740379270AEF74028030C7
:10E7D6000B33740185360DEF74018B3913377400D2
:10E7E600903D1BF075FF94441E7775FF984823EF04
:10E7F60075FE9B46207776FE9F4221F076FEA13F6E
:10E80600177777FDA44313EF77FDA747157778FDB4
:10E81600AA4915EF78FDAD4C157779FDB04D19EE87
:10E826007AFDB34D1C777AFD024E19F07BFD054F3C
:10E836001B777BFE094F24F37CFE0D531D777CFF6F
:10E84600114619F37CFF173F12777C001F3810EF33
:10E856007C00263613777C012B3115ED7C012F2B9E
:10E8660015777C02332513ED7C02392214777C025E
:10E87600402110EE7C0249210B737B02531F0FEBE4
:10E886007B02601E15777B026A2214EA7B017428DC
:10E8960019777B017B2D1AEA7B00833122777B0077
:10E8A6008A3320EB7BFF91371A777BFE953C1FEA74
:10E8B6007CFE983C26777CFEA74621EC7CFD9939A8
:10E8C60023777CFC9A3B1FEA7DFC9A3F1C777DFBF5
:10E8D6009A401EE87DFB9B3F20777EFA9B3F1FE612
:10E8E6007EFA9C431A777EF99E4717E57FF8A04A81
:10E8F6000E737FF8A34A0AEA80F8A548073380F822
:10E90600A94402EA81F8AE46041182F8B24C00E747
:10E9160082F80351021183F8085304EA83F90E4D75
:10E92600061183F914430CEC84FA1A400E1184FB89
:10E93600203F0AE884FC2540061384FC2B4008E6A9
:10E9460084FD3039073383FD36300EE483FE3C2BDD
:10E95600193783FE402A1EE783FE3D25187783FE7E
:10E96600371B16E783FF3114137783FF35170FE440
:10E9760083FF3E220D738200412C15E58200432C55
:10E986001A77820046251BE782004C201577810006
:10E99600552116E581005E2510778100682718E469
:10E9A60081FF72291E7780FF7A2E22E580FE7E3057
:10E9B600277780FE812B22E680FD85251C7780FD4A
:0DE9C600882618E281FC8A2F187781FC8DCD
:10E9D3003821E181FB903F287781FA924025E0813D
:10E9E300FA943D237782F9973C18E082F99A3F1510
:10E9F3007782F89E4412E083F8A347107783F8A741
:10EA03004A0CDF84F8AA4D133785F7AC5214E2851C
:10EA1300F7AF56107786F7B2580DE087F802560223
:10EA23003387F8055002E388F8094C051188F90C7F
:10EA33004E02E489F91052011189FA155004DF8955
:10EA4300FB1D45041389FB233304DE89FB292306BD
:10EA53003389FC2B1F05DE89FC2F23093389FD3302
:10EA6300280ADC89FD3B23103788FD471E0EDD880D
:10EA7300FD511E0E3388FD53200CDD88FD54210B00
:10EA83003387FD57200DDD87FD5C20093387FD5D4E
:10EA93002403DE87FD5B29013386FD592C04DE86C2
:10EAA300FD5D2C093385FD622F0CDC85FD652D0B87
:10EAB3003385FC672908DF85FC6722093385FC6BF6
:10EAC300210CDD84FC72280A3384FB783005DD8455
:10EAD300FA7C37073384FA7E390ADC84F9813B06F2
:10EAE3003384F8843F05DB84F8873F023384F78A55
:10EAF3003C04DB84F78D390A3384F6903908D985D1
:10EB0300F5923F113785F595430FD985F498440A5B
:10EB13007386F49B440AD986F39C440C3386F39C96
:10EB23004507DA87F29C47063387F19E4C0AD9885A
:10EB3300F1A251103788F1A65516D989F0A7571FAE
:10EB4300778AF0A9541BDA8AF0AA4D12778BF0ACBE
:10EB5300460DDB8BF0AC4906338CEFAB4D05DB8CFC
:10EB6300EFA95002318DEEA85209E28DEEA7530EA4
:10EB7300118EEEA75316E58EEDA44A20118FEDA05A
:10EB83004423E28FEC9C4821118FEB9A4A22E090B8
:10EB9300EB95411D1190EA8E391DDF90EA893621EC
:10EBA3001190E9873223E590E9852C2C118FE87DBC
:10EBB3002A26E08FE8762124118FE8662122E08F50
:10EBC300E856221F118EE947201DE08EE9392116F0
:10EBD300118EE9302518E28EEA2D2917118EEB30BC
:10EBE3003213E18EEB333711118EEC373C10E18E8B
:10EBF300ED393E07138DED3B4203DD8DEE3B3E09C0
:10EC0300338DEE3B310DDE8DEE392812378DEF3823
:10EC13002319DC8DEF382A18778DF0372A12DC8D13
:10EC2300F0382214778DF0361B0EDC8DF1361B0C79
:10EC3300338CF1371F0DDB8CF136250E378CF23414
:10EC4300270CDC8CF22A270D338DF31F2A0CDC8D65
:10EC5300F3173409338DF4143A08E48EF4123A0CA2
:10EC6300338EF4103D11EA8FF50E411A778FF50CB0
:10EC73004917EA90F50A50157790F5054F13E79178
:10EC8300F5B24F107792F5AD5408E492F4AB5A0104
:10EC93003393F4AB5C05E893F4A9500A3394F3A4DB
:10ECA300450CE094F3A041093394F29A3A05E295B6
:10ECB300F29734043395F1913208DC95F19E310DCE
:10ECC3003395F08A320CDA95F0872D0B3395EF806C
:10ECD300250EDE94EF73220C3394EF6C2412DD9433
:10ECE300EF6928157794EE6B2812DF93EE69280EEF
:10ECF3007393EE64270DDF93EE5C260B3392EE578E
:10ED0300270EDB92EE5828123792EE5E2610DB9226
:10ED1300EE64240D7391EE6C2108D991ED722304F6
:10ED23003391ED782904D991EC7C320A3391EB7F4E
:10ED33003A08D891EB833D093391EA883C0CD7918B
:0DED4300E98D3B103791E9903E12D792E820
:10ED50009143137792E794420ED792E7993E073397
:10ED600093E7A03901D993E7A63B0A1194E6A83F9F
:10ED70000CD794E6AB490E1195E6AE4F07D695E653
:10ED8000004D011396E6034601D996E6033E0811AD
:10ED900097E7043D0ED997E70740151198E70C4314
:10EDA00012DA98E812460F1198E918490CDA98E936
:10EDB0001D44081198EA243D05D898EB293A03111F
:10EDC00098EB2C3707D898EC2D38093398ED2E3D69
:10EDD0000ADC98ED2E3E0A3398EE2D3F0BDB98EFC0
:10EDE0002C420C3398F02B430ED998F02B3D113761
:10EDF00098F12D3710D898F130340D7398F23433E0
:10EE00000FD698F237330F7798F339331CD597F331
:10EE10003C32167797F43E2F11D797F440280973A8
:10EE200097F4422109D797F4461F0AB396F44B2171
:10EE300008D796F45325083396F45C2505D796F445
:10EE40006723023395F4722503D695F3782B0231AC
:10EE500095F37B3102D695F27E31063395F1832FFF
:10EE600004D695F18A2F023395F0913201D596F0B0
:10EE70009638061196EF9A3F02D497EF9D450213FC
:10EE800097EE9F4704D497EEA247073398EEA64427
:10EE900008D398EEAA430B3399EEAD440CD499EE07
:10EEA000B1400D339AEE013F11D39AEE054512772A
:10EEB0009BEE064A15D59BEE064712779CEF05425E
:10EEC00012D79CEF063E0F779DEF084111D39DEFBF
:10EED000094619779EF00B4718D39EF00D431C7717
:10EEE0009FF10F4015D69FF1114113779FF2134602
:10EEF0000ED9A0F2174A0B33A0F31C4A08D4A0F491
:10EF000023420333A0F42A3305D3A0F53127071198
:10EF1000A0F5382300D29FF53D2702339FF6442900
:10EF200003D39FF64F2808119EF55E2807D19EF562
:10EF30006C2D04119EF4752F01D09EF47C2D0433AA
:10EF40009EF3822B04D09EF3872E05119EF28B3503
:10EF500007D09EF2903D01119FF1954203D09FF0A2
:10EF600094400333A0F09F3F0BD0A0F0A13D0F379A
:10EF7000A0EFA33C0DD1A1EFA43C0C33A1EFA43C26
:10EF80000AD0A1EEA53D0533A2EEA63C00D1A2EE2B
:10EF9000A8390211A3EEAA3C04D0A3EEAD3F05119F
:10EFA000A4EEB24008D0A4EE03410C11A5EE064138
:10EFB0000AD2A5EE08450711A6EF094A05D2A6EF29
:10EFC000094C0111A7EF0A4807D3A7F00B420B1118
:10EFD000A8F00B420DD4A8F00D461311A9F111466B
:10EFE00014D9A9F1173F1B11A9F21E381ADAA9F397
:10EFF00021381811A9F31F3A17DFA9F41839151190
:10F00000AAF4163A1DDCAAF5183C1A11AAF51C3A06
:10F010001AD9AAF61F391A11ABF6203615D9ABF753
:10F0200021341711ABF8203B19D9ABF81E3F17114B
:10F03000ACF91D4011D9ACF91E3F0E11ACFA1F40BE
:10F040000CD6ACFB22410D11ACFC23450FD6ADFC18
:10F0500023490B11ADFD214A0DD6ADFE2047091104
:10F06000ADFE21450CD6ADFF22430E11AE00224568
:10F070000CD8AE01214B0A11AE0220500DD7AF03C0
:10F080001D4F0B11AF031A5109D9AF04174A0D11C7
:10F09000B00418470BDBB0051A500A11B0061C5516
:10F0A0000ED7B1071C560B11B10719470ED9B1087D
:10F0B000173C0C11B208183D0CDCB2091C490E11AA
:0DF0C000B20A1E4E0AD9B30B1D500B11B33E
:10F0CD000C1A5109D9B30C174F0711B40D17490B71
:10F0DD00DBB40D17480D11B50E19490ADCB50F1922
:10F0ED004F0B11B50F185605DBB61017550711B696
:10F0FD0011174C0ADBB61116430B11B711173F0D43
:10F10D00DDB71219430C11B7131A480BDCB8131ADB
:10F11D00450F11B81419410DDCB81418400B11B975
:10F12D001518430DDBB91618470F11B91618490DEF
:10F13D00DBBA1718470A11BA1717450CDBBB1814A1
:10F14D00460F11BB18134C0EDBBC1912510A11BC22
:10F15D001A125007DBBC1A12470B11BD1A10400DC5
:10F16D00DCBD1B10400A11BE1B124509DCBE1C156F
:10F17D00490B11BE1D184A0ADBBF1D1B4A0811BFE2
:10F18D001E1B480CDBBF1F1A470E11BF1F1A490B60
:10F19D00DBC0201B4B0D11C0211C4910DBC0211DF4
:10F1AD00470F11C1221D4711DBC1231C4B0F11C18C
:10F1BD00231B4B0EDBC22419441111C224193D0F20
:10F1CD00DBC2251B3B1011C2261D3F0DDAC2261EC8
:10F1DD00411011C3271D3F12DAC3271C3D0F11C368
:10F1ED00281B3D10DBC4291C401111C4291C450FDF
:10F1FD00DCC42A1C460E11C42A1B4510DCC52B1974
:10F20D00431111C52C184511DDC62C164A1011C617
:10F21D002D174A11DEC62D18491211C72E19471088
:10F22D00DEC72F1A460E11C72F1C4410DFC7301F23
:10F23D00471111C731214B0CDBC832224D0E11C8BD
:10F24D0032224A10DAC83321471111C83420460F33
:10F25D00D9C83520461111C93521430CDBC93623D8
:10F26D003F0F11C937253D11DBC93725400E11C997
:10F27D0038254211DCC93925431311C939254312EB
:10F28D00DCC93A25431111CA3B24400DDCCA3C248C
:10F29D00411011CA3C23400EDCCA3D22401111CA57
:10F2AD003E20420FDECB3E20451011CB3F204714B0
:10F2BD00DECB4021441211CB40213F10DFCB412248
:10F2CD003C0D11CB42234011DFCC42233E1111CC1A
:10F2DD0043202F0EE0CC4319221211CC43122011E2
:10F2ED00E3CC4311250E11CD43132B10E3CD441266
:10F2FD002D1111CD440F2B0FE3CD44092B1211CE3F
:10F30D004404320FE2CE4401360E11CF44B3370D13
:10F31D00E0CF44B3330E11D04401370EE0D0440595
:10F32D003D0D11D0450A3B0CE3D14512330D11D1E2
:10F33D00451A2D0EE3D1461E2B0F11D1461D2E0F52
:10F34D00E4D1471D300F11D1471E320EE3D24821B3
:10F35D00330F11D248233510E2D24923350F11D284
:10F36D004A20360EE3D24A1D360E11D24B1B3410F5
:10F37D00E3D34B1B320F11D34B1B300EE4D34C1B7D
:10F38D00340D11D34C1B3A0DE5D44D1A3B0E11D44F
:10F39D004D1B360AE6D44E1D340E11D44E1E360DBD
:10F3AD00E5D44F1F360C11D5501F350EE5D5501F26
:10F3BD00340D11D5511E340EE5D5511E370C11D516
:10F3CD00521E390EE5D652203B0F11D653223C0F5B
:10F3DD00E4D65423391111D654243710E3D65524CD
:10F3ED00360F11D655253310E3D65626330D11D6CB
:10F3FD005627350BE2D657273A0C11D658273C0F16
:10F40D00E2D75827391011D75927370FE2D75A2786
:10F41D00381011D75A283B0FE2D75B293C1111D771
:10F42D005C2B3C12E2D75C2D391111D75D2C3910B4
:0DF43D00E3D75E2B3C0F11D75E293B0EE399
:10F44A00D75F27371011D75F26360EE3D760273CE0
:10F45A000E11D761284310E3D76229451111D762EB
:10F46A00293F0FE4D763283A1011D763293A11E4E8
:10F47A00D7642A3E1011D7652C4211E4D7662E4272
:10F48A001011D7662D3F11E4D7672F3A1011D768AC
:10F49A002D3B0CE4D7682E3D0711D7692E4204E4B0
:10F4AA00D76A2E470111D76B2E4702E4D76B2D403E
:10F4BA000513D76C2B3503E4D76C2A2B0711D76DAC
:10F4CA002B2909E5D76D2B300611D76E2A3A04E4A9
:10F4DA00D76F28400611D76F283E08E4D77027381F
:10F4EA000C11D87026320DE6D871252F0911D87162
:10F4FA0024310AE9D87221340811D8721B3A08EA71
:10F50A00D9730D420A11D973104909EADA730C4505
:10F51A000811DA730A3B06E8DB74093D0211DB7451
:10F52A000A4003E9DB740B3C0213DC75103406EA6B
:10F53A00DC7517350333DC761A3F06EADD771C469D
:10F54A000433DD771F4001E8DD7824360731DD78A2
:10F55A002C3206E7DC7933320413DC79373409E7D5
:10F56A00DC7A3A340C33DC7A3C3508E7DC7B3D370D
:10F57A000233DB7C3C3A05E7DB7C3C3D0333DB7D35
:10F58A003B3A04E7DB7D3B320331DA7D3E2D09EA63
:10F59A00DA7E43270D11DA7E4D230AE9DA7E5726F1
:10F5AA000B11D97D5E2C0BE9D97D61300C11D97D07
:10F5BA00632F08EAD87D662F0511D87C683005EAE2
:10F5CA00D87C6D330611D77B733608E9D77B7C3834
:10F5DA000511D77A853A04E8D8798B3B0711D8798F
:10F5EA008E3809E9D8788F371011D878903B0BE814
:10F5FA00D87791420D11D976954A08E7D976984974
:10F60A000411D9759D4008E8DA75A23A0B33DA7508
:10F61A00A53C0AE8DB75A8430031DB74AA4603E976
:10F62A00DC74AF460213DC74004A02EADD75054C4D
:10F63A000333DD75084D00EDDE75084B0533DF76C3
:10F64A00064902EDDF76044A0131E076044902EA0E
:10F65A00E076044C0513E176045006EAE176014DA2
:10F66A000D33E276B1450FEAE276AD3F1077E375E6
:10F67A00AB3F0DEAE375AC430A33E475AE4604EAE0
:10F68A00E475B0400131E575B23908EAE575013C27
:10F69A000611E675054607ECE6760A4B0311E7768E
:10F6AA000F4604EEE777163B0611E778203405EC9F
:10F6BA00E77827350611E7792D3409ECE7793234F2
:10F6CA000B11E77A3B260AECE67A45250B11E67A16
:10F6DA004D230BEAE67A56250711E67A5F270AEAEE
:10F6EA00E579672A0C11E579731F0AEBE578792E1B
:10F6FA000811E578843302EAE5778D3B0313E67651
:10F70A00954104EAE676993F0733E6759A3801EAA5
:10F71A00E67595310531E6748F3202EAE6748E3564
:10F72A000111E773923301EAE77398310413E77220
:0AF73A009D3304EBE872B4370911A7
:00000001FF
